:020000040800F2
:10000000000004207D880008012E0008052E00084D
:10001000092E00080D2E0008112E00080000000017
:1000200000000000000000000000000085E0000863
:10003000152E00080000000011E100086DE1000825
:10004000CD880008CD880008CD880008CD8800083C
:10005000CD880008CD880008192E0008212E000840
:10006000CD880008CD880008710A000851180008E2
:1000700079180008A1180008CD880008C9180008E0
:10008000D5180008CD880008CD880008CD88000864
:10009000CD880008CD880008CD880008F53100081B
:1000A000CD880008CD880008CD880008CD880008DC
:1000B000CD880008CD880008CD8800089D1700086D
:1000C000A9170008B5170008C1170008CD170008C8
:1000D000D9170008CD880008E5170008CD8800086A
:1000E000292E0008CD880008CD880008A92E000818
:1000F000C12E0008D92E0008CD880008FD18000880
:1001000000000000CD880008CD880008CD880008D8
:100110000000000000000000CD880008CD88000825
:10012000251900083119000865190008ED2E00088E
:10013000CD880008CD880008CD880008CD8800084B
:10014000CD880008CD880008CD880008CD8800083B
:10015000CD880008F92E0008711900080118000860
:10016000CD880008CD8800080000000000000000D5
:10017000000000000000000000000000000000007F
:10018000CD880008CD8800080000000000000000B5
:10019000CD880008CD8800080000000000000000A5
:1001A000000000000000000000000000000000004F
:1001B000CD8800080000000000000000CD88000885
:1001C000CD88000802484FF4DC310BF0E3BD00BFDE
:1001D000380100204FF0C043C0B21880704700BF04
:1001E0004FF0C0435880704741B100EB41014FF0E0
:1001F000C04230F8023B53808842FAD1704700BFBA
:1002000041B100EB41014FF0C042538820F8023B5E
:100210008842FAD1704700BF30B50024A1B0214612
:10022000682206A80194029403940494059410F0A3
:1002300076FC23462246144914480BF08DF90546F6
:100240000AF09CFAF022114620460AF035FAF02214
:10025000114620460AF018FA204603210BF036F822
:1002600001A928460AF0AFF9094A0A4B0A4C119431
:10027000CDE90E23094A1592094B0A4A06A92846D8
:100280000AF0BFF921B030BD7056010828550108A9
:10029000D5010008E1010008E90100080102000899
:1002A000CD9F0008319900084FF0FF30704700BF24
:1002B00030B58BB01E4B00220192196B41F0080142
:1002C0001963196B01F00801019101990292196BF0
:1002D00041F040011963196B01F04001029102994C
:1002E0000392196B41F0200119631B6B4FF40060FE
:1002F00003F0200303930490012304A90D48059300
:100300000224CDE90624039D04F0E6FC0822002324
:1003100004A90948CDE9042304F0DEFC20220123CE
:10032000064804A9CDE9042304F0D6FC0BB030BD87
:1003300000380240000C0240001802400014024045
:100340002DE9804800F2644783B00446384600F047
:1003500039FB04F27C4302211846019300F0ECFBC8
:10036000B8466FF04049404600F052FB404600F06E
:1003700057FB0121404600F077FBB4F888E4D4F83D
:100380009474D4F884C40EF1FF35A9EB050502215D
:1003900007EB85050EFA01F6654538BFAD190CEB84
:1003A000060B0246D4F88C642D68C4F89074D20908
:1003B000164407F1040A761BC4F894A4C4F88C64AC
:1003C000DA453A6018BFD4F894C4D4F88C24019864
:1003D000B2FBFEF20023C4F894C492B200F0C2FB58
:1003E000D4F87C150139C4F87C150029BBD1202331
:1003F000C4F87C350222204602F0FEF9B1E700BFC6
:1004000038B560210446002501F0CCFA04F5936369
:100410002022C4F88434A4F88824C4F89034C4F8A2
:100420009434C4F87C25284684F88A5403F0CEFF1F
:100430002946204600F082FC2946204600F098FC20
:100440002046294600F09EFC204638BD08B50446EB
:100450000849002004F0B6F80749002004F0B2F87B
:10046000052204F264400223114600F06BFA204694
:10047000FFF766FF201301084C1301080078B0FA5B
:1004800080F04009704700BF01230370704700BF30
:10049000704700BF00207047704700BFFEE70000B4
:1004A000044A05491368002B08BF0B461844106026
:1004B0001846704738B90120C80D02200020704747
:1004C00010B5034B036004460DF0A2FB204610BD9F
:1004D0004415010810B5054B036004460DF098FB68
:1004E000204608210FF0C0F8204610BD4415010831
:1004F00090F88A3410B5044623B1D0F8840408B1CA
:100500000FF0B4F8204610BD10B5064A064B026045
:10051000044640F8783F0DF07BFB20460DF0A6FC2A
:10052000204610BD601501084415010810B5064AA3
:10053000064B0260044640F8783F0DF069FB204608
:100540000DF094FC204610BD60150108441501080B
:1005500010B5084A084B0260044640F8783F0DF099
:1005600057FB20460DF082FC204688210FF07CF8D6
:10057000204610BD601501084415010810B5084A51
:10058000084B0260044640F8783F0DF041FB2046DE
:100590000DF06CFC204684210FF066F8204610BD5B
:1005A000601501084415010808B5274C2368BFF3FE
:1005B0005B8FD90712D5254C2368BFF35B8FDA0711
:1005C0002FD5234C2368BFF35B8FDB0717D5214B57
:1005D00001221A700EF06EFC04F04CF82046FFF772
:1005E0004DFF0028E7D01C48FFF70AFF1B4A1C49B3
:1005F0001948FFF74FFF2046FFF746FFDBE720468D
:10060000FFF73CFF0028E2D01349164800F0F2F84B
:10061000124A15491348FFF73DFF2046FFF734FF04
:10062000D5E72046FFF72AFF0028CAD00A490F481D
:1006300000F0B2F8094A0E490C48FFF72BFF20469C
:10064000FFF722FFBDE700BF54BA0120C8B901205F
:1006500040B90120A8CE012058BA0120BD040008ED
:10066000F104000844B9012009050008CCB90120B3
:100670002D0500080446D0F8840008B500F59870F0
:1006800002F09EFD0BF004F81E480AF091FD1E4892
:10069000082278210AF032FE1C48C82278210AF08C
:1006A0002DFE1B48DC2278210AF028FE19481E2264
:1006B00078210AF023FE1848502278210AF01EFE05
:1006C000D4F884000122042102F096F8D4F88400C2
:1006D0000022042102F0B4F9D4F88400002204219D
:1006E00002F08AF80AF0D4FF0C481E2278210AF0A2
:1006F00005FE0B48502278210AF000FED4F8840051
:10070000FFF7A4FED448010890130108A8130108BC
:10071000AC130108C0130108CC130108E813010849
:10072000F413010808B50446D4F88000032102F050
:100730002FF84FF4FA7120460DF038FCF4E700BFB3
:1007400070B5541A82B00F2C0E460194054611D88C
:10075000012C006808D10B780370019C28686C603C
:100760000023035502B070BD5CB900236C600355D3
:1007700002B070BD002201A90EF084FF019B286029
:10078000AB602246314610F009FA019C28686C6083
:100790000023035502B070BD70B5134A86B00446FD
:1007A00002AE0D466846A2F10F010096FFF7C8FFA2
:1007B000032369464FF4806220460DF0D5FB009874
:1007C0000A4B2360B042C4F8805003D00299013133
:1007D0000EF04AFF064B2360C4F8845020460DF00B
:1007E0000BFB204606B070BD1714010874150108F4
:1007F0008815010870B5114A86B002AE04460D4650
:100800006846A2F10E010096FFF79AFF022369469F
:100810004FF4007220460DF0A7FB0098B04203D0C1
:10082000029901310EF020FF054B2360C4F880507F
:1008300020460DF0E1FA204606B070BD26140108EE
:100840009C15010810B5034B036004460DF034FA03
:10085000204610BDB015010810B5054B03600446D5
:100860000DF02AFA204608210EF0FEFE204610BDAB
:10087000B015010830B5044689B040F80C1B0223BE
:10088000A36060600822002110F049F900251D4B8B
:1008900000951A6B257542F002021A631A6B1A480A
:1008A00002F002020092009A01951A6B42F00402D3
:1008B0001A631B6B03F00403019301220123CDE9AA
:1008C000022302A9019B00220023CDE9042304F0A6
:1008D00003FA0E4B0E481022CDE9022302A902238F
:1008E0000122CDE9042304F0F7F92A4609210A2060
:1008F00003F01CFF01220448114604F007FB2046C8
:1009000009B030BD00380240000402400000211050
:100910000008024070B505460C46164622460021E6
:10092000286800F0A7F900222868114600F0A2F913
:1009300080B204B970BDB0424FF00A00FAD003F0A3
:10094000D1FEEBE7F8B51746002204460E460068D4
:1009500011461D4600F08EF900221146206800F075
:1009600089F945F2065211462046FFF7D3FF43F6B8
:100970004B020021206800F07DF97602002211462A
:10098000206806F47E4600F075F9002106F14D025C
:10099000206800F06FF900221146206800F06AF923
:1009A00005EB4712D2B2120200214E32206800F04D
:1009B00061F900222068114600F05CF901232375DB
:1009C000F8BD00BF10B540F24F3204460021006868
:1009D00000F050F900221146206800F04BF94FF466
:1009E0004C5211462046FFF795FF45F2055211463D
:1009F0002046FFF78FFF04480DF088F9034B4FF4B2
:100A000080621A6010BD00BFD8BF012000E100E085
:100A100002484FF0FF310DF06BB900BFD8BF012085
:100A200010B5044688B005A90E480190032303AA17
:100A30002068039101A90293049300F049F9039BF4
:100A40002068596802F01CF86268039B000A106075
:100A50009968206802F014F86368000A586008B0CA
:100A600010BD00BFB8150108436853F82100704756
:100A700000B5102083B004F055FA0A4801A90DF022
:100A800053F9019B012B09D14FF0E0234FF0805225
:100A9000C3F8042DBFF34F8FBFF36F8F03B05DF822
:100AA00004FB00BFD8BF012030B589B01E4B002524
:100AB00000951A6B016042F002021A631A6B02F091
:100AC00002020092009A01951A6B42F004021A6326
:100AD0001B6B03F004030193144B4FF48042CDE9E8
:100AE00002230446012202A911480223CDE904236E
:100AF000019B04F0F1F82A460921282003F016FE94
:100B000001220123CDE9022302A902230022094880
:100B1000CDE9042304F0E0F801220648114604F070
:100B2000F5F9204609B030BD003802400000211020
:100B3000000402400008024010B5032384B0C943FA
:100B4000194080228DF806208DF8051000688DF878
:100B5000043001AC02AA0121CDE9024300F0CCF837
:100B600004B010BD10B584B013443031032202929A
:100B7000C3F3072C8DF80C1000688DF80DC003AC82
:100B800001AA012101948DF80E3000F0B5F804B0EF
:100B900010BD00BF0160704708B500220121054863
:100BA0000DF0CCF8BDE80840034A04490148FFF7BE
:100BB00071BC00BFD8BF0120BD0400084508000873
:100BC00070B5064C064EA4F1280544F8086D204681
:100BD0000DF072F8AC42F8D170BD00BF50C50120D5
:100BE000B015010810B50648064C40F8084F0DF046
:100BF00063F803480460BDE810400DF05DB800BF25
:100C000050C50120B015010810B50648064C40F843
:100C1000084F0DF051F803480460BDE810400DF096
:100C20004BB800BF60C50120B015010810B50648DB
:100C3000064C40F8084F0DF03FF803480460BDE84B
:100C400010400DF039B800BF70C50120B015010883
:100C500010B50648064C40F8084F0DF02DF8034833
:100C60000460BDE810400DF027B800BF80C501202A
:100C7000B015010800B585B0019279B904230DEBD8
:100C8000030103AA0E4806F091FF4FF0FF310D4813
:100C90000DF02EF8039805B05DF804FB022201A9BF
:100CA000094806F015FF41F234234FF0FF310748A1
:100CB00003930DF01DF8039805B05DF804FB00BF29
:100CC000F8C5012098C50120A0C5012090C50120CC
:100CD00008B54B681268096805489B009BB206F08E
:100CE00065FFBDE8084003484FF0FF310DF000B844
:100CF000F8C5012098C5012008B51368928851B93C
:100D000019460A4806F0E4FEBDE8084008484FF0DE
:100D1000FF310CF0EDBF1946064806F0D9FEBDE8DC
:100D2000084005484FF0FF310CF0E2BFF8C5012044
:100D300098C50120A0C5012090C5012010B50B4623
:100D40000848094AC45C525C08484FF4806104F0CA
:100D5000DDF822460548BDE810404FF4005104F08C
:100D6000D5B800BFC4150108C81501080014024019
:100D70000A1E034818BF0122202104F0C7B800BF93
:100D8000001002400A1E034818BF0122402104F04F
:100D9000BDB800BF0010024000B58BB0264B00224A
:100DA0000092196B41F008011963196B01F00801F9
:100DB000009100990192196B41F010011963196BB0
:100DC00001F01001019101990292196B41F020018B
:100DD0001963196B01F020010291029903921A6BB9
:100DE00042F040021A631B6B4FF44050012103F0A4
:100DF00040030022CDE90401039304A90F48002316
:100E0000CDE90623039B03F067FF602304A90C4888
:100E1000049303F061FF42F20C4304A909480493D0
:100E200003F05AFF4FF498430748049304A903F0D2
:100E300053FF0BB05DF804FB00380240000C024089
:100E40000010024000140240001802402DE9F04F4B
:100E500091B04FF0000BBD4CCDF80CB0236BBC48EB
:100E6000BC4D43F001032363236B03F001030393A1
:100E7000039BCDF810B0636C43F480536364636CE0
:100E800003F48053A022022604930AA94FF003081A
:100E90004FF00509049B0A920127CDE90C680B96D7
:100EA000CDF8389003F018FF10221223A8480C97B1
:100EB0000AA9CDE90A2303F00FFF4023A4480A93AF
:100EC0000AA9CDF830B003F007FFA34B2B604FF415
:100ED00082736B604FF48023AB610823EB6128467B
:100EE0000A23C5F808B0C5F80CB0C5F810B06F619A
:100EF000C5F820B0C5F824B0C5F828B0EB6206F0FC
:100F0000A5FD002840F01F810590236BDFF86CA23F
:100F1000924A43F480032363236BCAF80C0003F462
:100F200080030593059BCAF814004023CAF80830D3
:100F3000CAF81800CAF81C00CAF82C00CAF8300019
:100F4000CAF800204FF480634FF080624FF4003104
:100F50004FF0040B5046CAF80420CAF82880CAF89B
:100F60001030CAF82010CAF824B003F0B1FC0246D1
:100F7000002840F0E880394601903A2003F0D6FB83
:100F80003A2003F00FFCC5F848A0CAF83850DFF843
:100F9000F0A1019ACAF80820CAF80C20CAF8142057
:100FA000CAF81820CAF81C20CAF82C20CAF8302029
:100FB0006B4ACAF800204FF0C0624FF48063CAF851
:100FC000042050464FF44032CAF824B0CAF810301A
:100FD000CAF82880CAF8202003F07AFC834600284B
:100FE00040F0B18002463946382003F09FFB38209C
:100FF00003F0D8FB5A4631462320C5F84CA0CAF866
:10100000385003F093FB232003F0CCFBCDF818B04D
:10101000236B43F002032363236B03F00203069365
:10102000069BCDF81CB0236B43F004032363236BB2
:1010300003F004030793079BCDF820B0236C43F41F
:1010400080432364236C0B960AAD082003F480438D
:1010500029460A9008934348089BCDF83890CDE97B
:101060000C6803F039FE4FF4005329463E480A93BA
:10107000CDF830B0CDF8389003F02EFE4FF480520A
:1010800012233948CDF838902946384D0C97CDE9D0
:101090000A2303F021FE0820354BE8614FF48272E9
:1010A0000A206A60E8624FF480222B6028464FF4E1
:1010B0000043AA61C5F80CB02E61C5F814B0C5F89C
:1010C00020B0C5F824B0C5F828B0AB6006F0BEFC6F
:1010D000002838D10990236B43F400132363236B5A
:1010E000244C03F400130993099B60604FF4806360
:1010F000402223614FF400311F4BE0606061A0612A
:10110000E0616062E06220632046C4F82880A2604B
:101110002162236003F0DCFB8046A0B93946024619
:101120000F20AC64A56303F001FB0F2003F03AFB32
:1011300042463146242003F0F9FA242003F032FB22
:1011400011B0BDE8F08F03F095FA00BF00380240FF
:1011500000000240F8C50120003001404064024018
:10116000106402400008024000040240A0C50120B3
:101170000038004008C2012070600240C8C301204E
:1011800068C301202DE9F04F8FB0884C8848894E04
:10119000002503950A95236C43F400132364236C04
:1011A00003F400130393039B0495236C43F480031F
:1011B0002364236C03F480030493049B0595236B41
:1011C00043F002032363236B03F002030593C02261
:1011D00012234FF0020A4FF0040908A9CDE90823B1
:1011E000CDF82CA0059BCDF8309003F075FD724B27
:1011F000724AB560C6E900236E274FF4804330463B
:101200007561B561F5613562F760336104F028F905
:10121000002840F0C8800690226B694942F4001211
:101220002263226B02F400120692069A654A4FF47A
:1012300080659060D06050619061D06150621160B3
:101240004FF480384FF00071104651601561C2F8BC
:10125000208003F03DFB8346002840F0A480594ADB
:10126000B26396630C2102460B2003F05FFA5649E5
:10127000564AC1F804B0C1F80CB0C1F814B0C1F8B6
:1012800018B0C1F81CB0C1F820B0C1F824B00846AD
:101290004FF0400B0A600D61C1F808B003F018FB75
:1012A000024600287FD1484971638E6301900D2169
:1012B0000C2003F03BFA12233D48099308A90123AF
:1012C000CDF830900A93CDF82CA0089503F004FDDA
:1012D0004FF40073DFF80C913548089308A90923EF
:1012E0000C9303F0F9FC344BC9F804304FF48043FD
:1012F000019AC9F810304846354BC9F80C70C9F846
:101300000820C9F81420C9F81820C9F81C20C9F809
:101310002020C9F8003004F0A3F8002843D107903A
:10132000236B43F400132363236B2A4C03F4001351
:101330000793079B284BA060E0606061A061E061BB
:1013400060624FF060672046C4E90037C4F820802F
:10135000256103F0BDFA064628BBC9F83840C4F839
:1013600038901E4C02460C210D2003F0DFF91C4B77
:1013700067602046C4F808B0E66025616661A66132
:10138000E66126626662236003F0A2FA024650B963
:101390000C212F20C9F83440C4F8389003F0C6F966
:1013A0000FB0BDE8F08F03F065F900BF00380240D0
:1013B0000004024034C00120801A0600005400409E
:1013C0001060024048C10120A8C1012028600240ED
:1013D0000058004088C0012040600240E8C0012061
:1013E000B8600240E0BF01202DE9F0418AB000253D
:1013F0003F4E0195336B3F4C43F001033363336B36
:1014000003F001030193019B0295336C43F4003315
:101410003364336C03F4003302930C20022107235E
:10142000CDE90401029A344808930122032304A958
:10143000CDE9062303F050FC304AA5604FF4E133B8
:10144000C4E9002320460C23E56025616361A561A2
:10145000E56107F023F8002847D10390336B284D4E
:1014600043F400133363336BA86003F40013039356
:10147000244BE8606861A861E861286268624FF007
:10148000006828464FF48067C5E90038039A2F6149
:1014900003F01EFA064640BB02460D21102065638C
:1014A000AC63194D03F042F9102003F07BF940239F
:1014B000AB602846154BC5F80480EE602F616E6165
:1014C000AE61EE612E626E622B6003F001FA02469D
:1014D00058B90D2111202563AC6303F027F91120C1
:1014E00003F060F90AB0BDE8F08103F0C3F800BF73
:1014F0000038024028C301200000024000440040A0
:1015000068C2012088600240C8C20120A060024079
:101510002DE9F0478AB0604E00240094336B43F00D
:1015200004033363336B03F004030093009B0194C3
:10153000336B43F040033363336B03F04003019399
:10154000019B0294736C43F020037364736C40201E
:10155000022103F020030825CDE9040102934F483E
:10156000029B089504A94FF001084FF00309CDE94B
:10157000068903F0B1FB4FF4007202234848089536
:1015800004A9CDE90423CDE9068903F0A5FB4FF4B6
:1015900040520223CDE90423414808950022032349
:1015A00004A9404DCDE9062303F096FB3E4A3F4B8C
:1015B000AC60C5E900234FF400434FF44072EB6187
:1015C00028460C23AA61EC602C616B6106F066FF73
:1015D00000285FD10390336B354C43F480033363B1
:1015E000336BA06003F480030393324BE0604FF051
:1015F0002069C4E900396061A061E061E0622063B4
:101600004FF4003320464FF4806A4FF0040802275D
:10161000039AC4F810A02362C4F82480A76203F0E0
:1016200057F90646002835D10246062139206C6359
:10163000A563214C03F07AF8392003F0B3F8402376
:101640001E4AA36020464FF48033E6606661A661BF
:10165000E661E6622663C4F80490C4F810A0C4F8FA
:101660002480A7622260236203F032F9064688B91B
:101670000246062146202C63A56303F057F8462056
:1016800003F090F832460A21472003F04FF80AB0E1
:10169000BDE8F08702F0EEFF00380240000802408B
:1016A00000180240E8C401200014014080841E009C
:1016B00028C401202864024088C40120B864024084
:1016C00030B5044683B001F0B7FD40F20E2204F5B8
:1016D000AA70C4F850210021C4F84C0101250FF074
:1016E0001EFA02F0C5FF15490095802304F55972D2
:1016F000002002F085FF002811DA2046FFF74CFB9E
:101700002046FFF7A3FB2046FFF73CFD2046FFF7EE
:101710006BFE2046FFF7FCFE204603B030BD0849B3
:101720000095802304F57972284602F069FF0028AD
:10173000E3DB0449002002F045FFDEE7281401083E
:1017400038140108481401080268084913688842DF
:1017500023F04003136003D0054B984203D0704739
:10176000044801F037BB044801F034BBF8C5012040
:10177000A0C5012098C5012090C50120054B9842C5
:1017800000D0704702680448136823F040031360D8
:1017900001F020BBF8C5012098C50120014804F0E4
:1017A0004FBA00BF34C00120014804F0E5BE00BFBD
:1017B00034C00120014804F043BA00BFE0BF01205B
:1017C000014804F0D9BE00BFE0BF0120014806F087
:1017D00091BB00BFF8C50120014806F08BBB00BFDC
:1017E000A0C5012008B5044806F0CCFEBDE80840BD
:1017F000024801F0EFBA00BF28C3012080C50120D4
:1018000070B5104C94F83A5094F839302046EDB247
:10181000DEB206F0B7FE222D0BD0212E00D070BD17
:1018200094F83930202BFAD1BDE87040064801F019
:10183000D1BA94F83A30202BF1D1BDE8704003487A
:1018400001F0C8BAE8C4012078C5012070C50120A4
:1018500010B5074C204603F065F994F83530012B9C
:1018600000D010BDBDE81040024801F0B3BA00BF7F
:1018700048C1012060C5012010B5074C204603F087
:1018800051F994F83530012B00D010BDBDE810405F
:10189000024801F09FBA00BFA8C1012068C501201D
:1018A00010B5074C204603F03DF994F83530012B74
:1018B00000D010BDBDE81040024801F08BBA00BF57
:1018C00088C0012050C50120014803F02BB900BF9A
:1018D00008C2012010B5074C204603F023F994F804
:1018E0003530012B00D010BDBDE81040024801F09A
:1018F00071BA00BF68C2012080C5012010B5074C35
:10190000204603F00FF994F83530012B00D010BDBC
:10191000BDE81040024801F05DBA00BFE8C00120F8
:1019200058C50120014803F0FDB800BF68C301207D
:1019300010B5094C204603F0F5F894F83530012B2A
:1019400000D010BD054B06482022BDE8104083F8AA
:10195000392001F03FBA00BF28C40120E8C40120AB
:1019600070C50120014803F0DDB800BFC8C30120E5
:1019700010B5094C204603F0D5F894F83530012B0A
:1019800000D010BD054B06482022BDE8104083F86A
:10199000392001F01FBA00BF88C40120E8C401202B
:1019A00078C5012010B50446FFF78AFE214604F2EF
:1019B0006440FEF75FFF214604F27C40FFF774F8B5
:1019C000214604F59060FFF7E5F8204610BD00BF02
:1019D00038B5002201213048304C0CF0AFF9304AC4
:1019E00030492D48FEF756FD002201212E480CF00B
:1019F000A5F92B4A2B492C48FEF74CFD002201216A
:101A00002A480CF09BF90022012129480CF096F994
:101A1000234A28490020FEF73DFD002201212648E7
:101A20000CF08CF90022012124480CF087F91C4AA3
:101A300023490020FEF72EFD0022012121480CF051
:101A40007DF90022012120480CF078F9144A1F4941
:101A50000020FEF71FFD002201211D480CF06EF949
:101A6000002201211B480CF069F90D4A1A49002097
:101A7000FEF710FD04F1280520460022012108345C
:101A80000CF05CF9AC42F7D1BDE83840044A134988
:101A90000020FEF7FFBC00BF98C5012028C501202B
:101AA000BD0400084508000890C5012080C501203C
:101AB00088C50120510C000870C5012078C501209F
:101AC0002D0C000860C5012068C50120090C000824
:101AD00050C5012058C50120E50B0008C10B0008C6
:101AE000B420704710B4B328144C94BF84464FF010
:101AF000000CA4F800C0B329114C94BF8C464FF0E1
:101B0000000CA4F800C01418B42CDCBF02F1FF32A2
:101B1000801803EB0102D4BF80B2B320B42ADCBF2B
:101B200003F1FF33C918074C074B2080D4BF89B29B
:101B3000B3215DF8044B1980704700BF52C60120E5
:101B400050C60120020000200000002008B501F06E
:101B5000FFFC4FF6FF7008BDB420704708B5292080
:101B600001F082FDBDE80840382001F07DBD00BFD6
:101B700008B5282001F078FD142001F081FD102027
:101B800001F072FDBDE80840962001F079BD00BF6C
:101B900070B5C0B282B0002200F11E04A0F12F0384
:101BA0002A208DF805400E468DF804208DF8062079
:101BB0008DF8073001F058FD01AC254615F8010BF2
:101BC00001F04CFD02AB9D42F8D1F1B2A1F14D0301
:101BD0002B208DF805108DF8073001F045FD14F825
:101BE000010B01F03BFD02AB9C42F8D102B070BD8D
:101BF00038B5D50802F4784305F0FC051D441446B9
:101C0000ADB2FFF7C5FF2C2001F02EFD284601F0F4
:101C100025FDE00200F47840BDE8384001F01EBD2B
:101C20002DE9F8430546C60A05F01F08F6000846E8
:101C30001F4606EBC826C5F3451311464FEAC808F0
:101C400005F4784505EB830508EB8328FFF7A0FF33
:101C50002C20B6B2ADB21FFA88F801F005FD8FB1A5
:101C600007F1FF390024284601F0F8FC304601F066
:101C7000F5FC4C45404601D001F0F0FC0234A4B222
:101C8000A742F0D8BDE8F88338B504460D46FFF703
:101C90007FFF29462046FFF77BFF2E2001F0E4FC62
:101CA00001F0E8FC01F0E6FC044601F0E3FCC4F3BB
:101CB0008502C0F3C42303EB421304F478441819DB
:101CC00080B238BD2DE9F04F0446154683B02C2074
:101CD00025440F46994601F0C7FCA54219DD274E61
:101CE000DFF8A080DFF8A0A0254B4FF0000B328872
:101CF000A2420AD8B8F80020BA4206D8BAF80020A2
:101D0000A24202D31A88BA4206D20234A4B2AC422A
:101D1000EDDB03B0BDE8F08F39F81B10C80800F008
:101D2000FC0001F4784108444FEA4B0280B2019272
:101D300001F094FC019A39F81B000232C00239F814
:101D400002100192C90A00EBC10080B201F086FCCA
:101D5000691EA1420A4B02D10BF1020BD5E7019A91
:101D600039F80220D000C0B2520900EB822080B2C4
:101D700001F074FC0BF1020B014BC6E752C60120C7
:101D80000000002050C6012002000020354B2DE944
:101D9000F04F354C1B8824885588958801331B1BD0
:101DA000324C1FFA83FE324BB4F800C01B880CF192
:101DB000010CACEB030C5389948911FA8CFC9BB297
:101DC0008C4587B043EA044348D9D718C3B203F11E
:101DD0001E0A2F3B0CF1FF39DBB25FFA8AFA00933F
:101DE0001FFA89F64FEA4E0B4FF00008CDF804E0D9
:101DF00002900391009B8DF814802A208DF815A085
:101E00008DF816808DF8173001F02EFC05AC2546B4
:101E100015F8010B01F022FC06ABAB42F8D1F2B28F
:101E20008DF815202B204D3A8DF8172001F01CFC61
:101E300014F8010B01F012FC06ABA342F8D13B46AB
:101E40003146019A0298FFF73DFF039B013E9945F9
:101E5000B6B25F4402D909F1FF39CBE707B0BDE85C
:101E6000F08F00BF0200002052C6012000000020B9
:101E700050C601202DE9F04F01EB030B594587B007
:101E8000894641D2C3B203F11E0A2F3BDBB2009355
:101E9000109E029053005FFA8AFA01930027039282
:101EA000009B8DF814702A208DF815A08DF81670FF
:101EB0008DF8173001F0D8FB05AD1FFA89F4A8465C
:101EC00018F8010B01F0CAFB06AB9845F8D15FFA90
:101ED00089F28DF815202B204D3A8DF8172001F04E
:101EE000C3FB15F8010B01F0B9FB06AB9D42F8D11D
:101EF0003346039A02982146FFF7E4FE09F10109EF
:101F0000019BD9451E44CBD307B0BDE8F08F00BF7D
:101F10002DE9F04F0C4685B01146064620469A46FC
:101F20001546FFF735FE2C2001F09EFBBAF1000F9D
:101F300047D0F30806F4784203F0FC031344E4B2FC
:101F4000F6029BB204F11E0B4D3D00932F3CB3B241
:101F50000026EDB201935FFA8BFBE7B2B0462A2070
:101F60008DF80C808DF80DB08DF80E808DF80F7007
:101F700001F07AFB03ACA14619F8010B01F06EFBEE
:101F800004AB9945F8D105F14D032B208DF80D30A8
:101F90008DF80F5001F068FB14F8010B01F05EFBA7
:101FA00004ABA342F8D12C2001F05EFB009801F0B5
:101FB00055FB0136019801F051FB01355645EDB254
:101FC000CDD105B0BDE8F08F30B583B001F0C0FAD7
:101FD000352001F049FB002001F040FB3A2001F0E0
:101FE00043FB062001F03AFBB02001F03DFB01204D
:101FF00001F034FBFE2001F031FBB12001F034FB95
:10200000DE2001F02BFB212001F028FBB72001F09E
:102010002BFB052001F022FB332001F01FFBB82031
:1020200001F022FB052001F019FB332001F016FB23
:10203000C82001F019FB042001F010FB032001F07F
:102040000DFBC92001F010FB5E2001F007FB08200A
:1020500001F004FBCA2001F007FB0A2001F0FEFAA0
:102060000C2001F0FBFA022001F0F8FACC2001F07C
:10207000FBFA032001F0F2FA042001F0EFFAD0207D
:1020800001F0F2FA0C2001F0E9FAB32001F0ECFAC9
:10209000022001F0E3FAC02001F0E6FA532001F03B
:1020A000DDFAC52001F0E0FA002001F0D7FA452062
:1020B00001F0D4FAC22001F0D7FA032001F0CEFAE1
:1020C000122001F0CBFADD2001F0CEFA002001F061
:1020D000C5FAB42001F0C8FA112001F0C5FA962023
:1020E00001F0CEFA1C4B01932A2001F0BDFA01AC9D
:1020F000254615F8010B01F0B1FA02ABAB42F8D15D
:102100000022B3232B208DF805208DF8073001F035
:10211000ABFA14F8010B01F0A1FA02AB9C42F8D122
:10212000362001F0A1FA832001F098FA292001F06D
:102130009BFA382001F098FA2C2001F095FA4BF622
:10214000D854002001F08AFA013CFAD1142003B0DF
:10215000BDE8304001F094BA001E00D1F020704775
:1021600010B4EF28144C94BF84464FF0000CA4F830
:1021700000C0EF29114C94BF8C464FF0000CA4F81E
:1021800000C01418F02CDCBF02F1FF32801803EB02
:102190000102D4BF80B2EF20F02ADCBF03F1FF338D
:1021A000C918074C074B2080D4BF89B2EF215DF8D6
:1021B000044B1980704700BF56C6012054C6012049
:1021C0003E0000203C000020F020704708B501F0E0
:1021D000BFF9042001F048FA01F04CFA01F04AFA84
:1021E000C0B208BD08B5292001F03EFABDE808409C
:1021F000112001F039BA00BF08B5BD2001F034FA52
:10220000FE2001F02BFA102001F02EFABDE8084064
:102210000A2001F035BA00BF70B5C3B282B0002207
:10222000A3F111042A208DF807400E468DF80420F2
:102230008DF805308DF8062001F016FA01AC254620
:1022400015F8010B01F00AFA02AB9D42F8D1F1B288
:10225000A1F111032B208DF805108DF8073001F046
:1022600003FA14F8010B01F0F9F902AB9C42F8D122
:1022700002B070BD10B51446FFF7CEFF2C2001F060
:10228000F3F92046BDE8104001F0E8B970B50C46FE
:102290000646114620461D46FFF7BEFF2C2001F0E2
:1022A000E3F935B100243046013401F0D7F9A542F5
:1022B000F9D170BD2DE9F04F0446154683B02C20AE
:1022C00025440F46994601F0CFF9A54219D9124E7F
:1022D000DFF84880DFF848A0DFF848B000233288F4
:1022E000A2420BD8B8F80020BA4207D8BAF80020AA
:1022F000A24203D3BBF80020BA4205D20134A54262
:10230000EDD803B0BDE8F08F39F81300019301F068
:10231000A5F9019B0133F1E756C6012054C60120FF
:102320003E0000203C000020344B2DE9F04F344C9F
:102330001B8824885588958801331B1B314C1FFA54
:1023400083FC314BB4F800B01B880BF1010BABEBF5
:10235000030B5389948911FA8BFB9BB28B4587B091
:1023600043EA044347D95FFA80FAD7180BF1FF3BE1
:10237000AAF111094FEA4C035FFA89F91FFA8BF6AB
:1023800000934FF00008CDF804C0029003912A207A
:102390008DF814808DF815A08DF816808DF81790A3
:1023A00001F062F905AC254615F8010B01F056F96C
:1023B00006ABAB42F8D1F2B28DF815202B20113AC2
:1023C0008DF8172001F050F914F8010B01F046F9CF
:1023D00006ABA342F8D13B463146019A0298FFF77B
:1023E00069FF009B1F44039B013E9B45B6B202D987
:1023F0000BF1FF3BCBE707B0BDE8F08F3E000020BC
:1024000056C601203C00002054C601202DE9F04FA3
:102410000E4619448E4287B03FD25FFA80FBABF183
:10242000110A5300109F00935FFA8AFA4FF00008D8
:102430000191029003922A208DF814808DF815B036
:102440008DF816808DF817A001F00EF90DF1140922
:10245000B4B24D4615F8010B01F000F906AB9D42F0
:10246000F8D1F2B28DF815202B20113A8DF81720F3
:1024700001F0FAF819F8010B01F0F0F806AB9945F4
:10248000F8D13B46039A02982146FFF713FF009BC1
:102490001F44019B01369E42CDD307B0BDE8F08FAB
:1024A00038B504460D46FFF7B7FE29462046FFF72C
:1024B000B3FE2E2001F0D8F801F0DCF801F0DAF8D4
:1024C000044601F0D7F8C4F38502C0F3C42303EB3C
:1024D000421304F47844181980B238BD2DE9F04F46
:1024E00085B0884601901146404699461446FFF74C
:1024F00093FE2C2001F0B8F8B9F1000F38D05FFA44
:1025000088F8A8F1110B113C00265FFA8BFBE5B2AD
:1025100037462A208DF80C708DF80D808DF80E70DE
:102520008DF80FB001F0A0F803ACA2461AF8010B29
:1025300001F094F804AB5345F8D105F111032B20B9
:102540008DF80D308DF80F5001F08EF814F8010B56
:1025500001F084F804ABA342F8D12C2001F084F8F8
:102560000136019801F07AF801354E45EDB2D0D12F
:1025700005B0BDE8F08F00BF70B584B000F0E8FF93
:10258000102001F071F80A2001F07AF8012001F022
:102590006BF8C82001F074F8112001F065F878207C
:1025A00001F06EF8362001F05FF8002001F056F8D7
:1025B0003A2001F059F8052001F050F8212001F0EF
:1025C00053F84FF06F432A20009301F04DF86E4608
:1025D00001AD6C4614F8010B01F040F8A542F9D1A9
:1025E0002B2001F041F8344614F8010B01F036F8C5
:1025F000AC42F9D1332340F60C42B220ADF80020B2
:102600008DF803308DF8043001F02EF8751D344636
:1026100014F8010B01F022F8A542F9D1B72001F01E
:1026200023F8352001F01AF8BB2001F01DF81F2017
:1026300001F014F8C02001F017F82C2001F00EF87A
:10264000C22001F011F8012001F008F8C32001F0C8
:1026500005F8C42001F008F8202000F0FFFFC62094
:1026600001F002F80F2000F0F9FFD02000F0FCFF8D
:10267000A42000F0F3FF22482249234A0292CDE928
:10268000000142F62953E020ADF80C3000F0ECFFD9
:102690000DF1FF340D36254615F8010F00F0DEFF71
:1026A000AE42F9D140F206631022ADF8043040F694
:1026B000513344218DF80220ADF80830162243F240
:1026C0002F13E1208DF807108DF80A20ADF80C309B
:1026D00000F0CAFF14F8010F00F0C0FFA642F9D1C4
:1026E000292000F0C1FF112000F0BEFF352000F0CE
:1026F000BBFF002004B0BDE8704000F0AFBF00BFDA
:10270000D00811080C1539335036131430B5012890
:1027100083B00BD002280BD06024362000F0A4FF39
:10272000204603B0BDE8304000F098BF0024F4E735
:102730000D4A009200233320ADF8043000F094FFDE
:102740006C460DF1060514F8010B00F087FFA54259
:10275000F9D1372000F088FF002000F07FFF5020E3
:1027600000F07CFFC024D8E7000001F070B5064CF3
:10277000064EA4F1280544F8086D20460BF09CFA9B
:10278000AC42F8D170BD00BF40C70120B0150108B0
:1027900010B539B301291AD0154A164832F811106C
:1027A000C16000234FF4486242600361836005F01A
:1027B000DFFD0246D0B90E212C2001F0B7FF0D48F5
:1027C00005F08CFCBDE810402C2001F0EBBF03208D
:1027D00000F0FCFD2C2001F0F3FFBDE8104005489F
:1027E00005F08CBC032000F0FDFDF3E701F042FF93
:1027F000E0150108C4C70120032970B525DD274D68
:10280000012AA5F10C0411D0022A29D0002A42D1B4
:10281000234EB05C00F0E6FDA54206D054F8042B30
:10282000B05C00F0DFFDA542F8D170BD00231C4E66
:10283000F05C00F0CBFDA542F7D054F8043BF05C0F
:1028400000F0C4FDA542F8D170BD012A1DD0022AB6
:1028500015D002BB124BBDE87040585C00F0C2BD01
:1028600000220F4EB05C00F0C9FDA542DDD054F847
:10287000042BB05C00F0C2FDA542F8D170BD084B3E
:10288000BDE87040585C00F0B9BD054BBDE8704034
:10289000585C00F09BBD01F0EDFE00BFDC150108A7
:1028A000DC1501084FF06043F0B44FF0E02CD3F892
:1028B000004E154E154F012000FA02F224EA0205DF
:1028C0002243DCF8FC4D124844F08074CCF8FC4DF7
:1028D000013900244FF0020CC3F8B07FC3F8005E4A
:1028E0000C4FC3F8804E0C4DC0F8F0C001614FF49E
:1028F0008071C3F8404E3760C0F80413C3F8805E9F
:10290000F0BCC3F8002E7047001000E055CEACC5F7
:10291000000004E0FE0300400D000100F0B5A5B08A
:10292000364A374B00240194106C40F080501064FC
:10293000126C02F080520192019A02941A6842F4D9
:1029400040421A601B68119103F440430D204FF47C
:10295000A021022401220425CDE9080102934FF4AD
:10296000800608A8CDE90E46CDE91245029B0A92E1
:102970000D921095149404F057FD00283BD14FF4AC
:102980008053059007900F27032103A80693039710
:10299000049404F00DFB034668BB032218921D93B8
:1029A0004FF48072229368231C9215934FF00062BB
:1029B000482315A8199416951F92179304F0DAFB73
:1029C0000446C0B93146024604F068FA04F0B6FA8B
:1029D00004F088FB0B4BA3FB0030800901F0FEFEE6
:1029E000284601F069FF224639464FF0FF3001F0DA
:1029F0009DFE25B0F0BD01F03DFE00BF0038024055
:102A000000700040D34D621038B505462D200C46AD
:102A100001F0D6FE002001F0D9FC44B930BF2D20D2
:102A200001F0C0FEBDE83840012001F0CFBC01211B
:102A3000002003F071FE60212846FFF76FFFEEE7EC
:102A400010B50C461146FFF7DFFF04484FF0FF3189
:102A500000EBC400BDE810400BF04AB918C70120D4
:102A6000132908B501D9022008BD04F01DFF00207C
:102A700008BD00BF132901D90020704704F01ABF18
:102A800008BA704730B589B0194C00250095236B02
:102A900043F010032363236B03F0100300930F2014
:102AA00001210122CDE90201009B124802A9002365
:102AB000CDE9042302F010F9284600F093FC012030
:102AC00000F090FC022000F08DFC032000F08AFC56
:102AD0000195236C084A094943F080032364236C61
:102AE000116003F080030193019B09B030BD00BF6A
:102AF0000038024000100240C4C70120001C004002
:102B000010B584B001F086FE194B01244FF000523D
:102B10006846CDE902340192ADF8004001F098FE1C
:102B200013234FF0006106228DF808306846002319
:102B300001918DF80B208DF80C308DF8014001F0DB
:102B400087FE1C234FF08041022268468DF8083032
:102B5000032301918DF801208DF80B308DF80C4086
:102B600001F076FE042001F063FE04B010BD00BF4A
:102B7000110000032DE9F0438BB03D4B002500957B
:102B80001A6B42F002021A631A6B02F00202009200
:102B9000009A01951A6B42F020021A631A6B02F038
:102BA00020020192019A02951A6B42F040021A63C8
:102BB0001A6B02F040020292029A03959A6B42F05D
:102BC00002029A639B6B03F002030446002603276C
:102BD0000393C022274802234FF0090904A9CDE935
:102BE00004234FF00A08039BCDF82090CDE9066737
:102BF00002F072F84FF4407202231E48CDF8208094
:102C000004A9CDE90423CDE9066702F065F80422A2
:102C100002231948CDF8209004A9CDE90423CDE979
:102C2000066702F059F8402202231448CDF82080AC
:102C300004A9CDE90423CDE9066702F04DF8042389
:102C40000F49A3631022172321636563E2632364A2
:102C50006564A564E564256504F1300003F024FE95
:102C600020B901F07BF90BB0BDE8F08301F002FD63
:102C700000380240001402400004024000180240E4
:102C8000001000A000B583B00B4B002201925A6BDC
:102C900042F040025A635B6B084A40F87C2F03F015
:102CA00040030193019B04F077FD10B903B05DF878
:102CB00004FB01F0DFFC00BF0038024000080650B2
:102CC00030B589B00025184B02951A6C42F4807219
:102CD0001A641B6C03F480730C46029301A903A8C9
:102CE000029B04F025FA04F003FA1049104A0A6026
:102CF00040F2E732CA600F4A0D614300A2FB032392
:102D00009B0C013B08464B608D6005F031FB0422B3
:102D100021462D2001F00AFD2D2001F043FD03483E
:102D200005F0DCF909B030BD0038024040C7012091
:102D30000020004083DE1B4338B504460D4601F0F9
:102D400011FB214B1A6842F400721A601A6842F4AF
:102D500080621A601A6842F480721A60032001F0DF
:102D6000D3FC0F212046FFF7ABFF29462046FFF793
:102D7000D5FD04F0E3F8002208212046FFF792FD7C
:102D8000012000F047FBFFF77DFE2046FFF7F2FE33
:102D90002046FFF777FF0D4A0D480121C2F83C1E7F
:102DA00000237F21FF22C4E90003A160E2602361C8
:102DB0006361A361204604F00BFD18B9FFF7A0FE84
:102DC000204638BD01F056FC003C0240000047425E
:102DD0000028004000B583B001A90AF0A5FF58B152
:102DE000019B4BB14FF0E0234FF08052C3F8042D0C
:102DF000BFF34F8FBFF36F8F03B05DF804FB00BFCD
:102E0000FEE700BFFEE700BFFEE700BFFEE700BF32
:102E1000FEE700BF704700BF012002F083B800BF8B
:102E2000022002F07FB800BF08B54FF4804002F0E6
:102E300079F8BDE808404FF4004002F073B800BFD5
:102E4000102808B525D008D8012811D0022821D192
:102E5000BDE808401048FFF7BDBFB0F5804F13D064
:102E6000B0F5004F16D1BDE808400C48FFF7B2BFDF
:102E700000F058FB0A4B003818BF012003EBC000DC
:102E8000BDE80840FFF7A6BFBDE808400548FFF7CA
:102E9000A1BF08BD01F0EEFB38C7012030C70120FB
:102EA00018C7012028C7012008B5034805F046F9D6
:102EB000024B01221A7008BD84C7012080C701207F
:102EC00008B5044805F03AF9BDE80840032000F0D1
:102ED00095BA00BFC4C7012008B5034805F02EF914
:102EE000BDE8084001F0ECBB40C70120014801F0FB
:102EF00019BE00BF58C60120014801F013BE00BF33
:102F0000B8C6012038B5094C04F128052046002236
:102F1000012108340AF012FFA542F7D1BDE838407C
:102F2000034A04490020FDF7B5BA00BF18C70120C5
:102F3000BD0400086D27000810B54FF6FF7000F0C3
:102F400097FD002000F082FC4FF6FF7000F084FC3B
:102F5000084800F087FC084A01236421002000F0A3
:102F600001FDBDE81040054A01237821002000F052
:102F7000F9BC00BF80000020901401089C140108D7
:102F800070B504460D46204601F0ACF850B9A5B91D
:102F90002378642043B301F0A5FB204601F0A2F89A
:102FA0000028F5D0642001F09DFBECE701F09AFBCE
:102FB000204601F097F80028F4D1012D4FF064006D
:102FC000F4D12378013B012B4FF064000CD901F0C0
:102FD00089FB204601F086F80028E3D12378013BE5
:102FE000012B4FF06400F2D801F076FB86B2204648
:102FF00001F078F80028FAD1237845B153B964205C
:1030000001F070FBBDE87040642001F06BBB013B38
:10301000012BF4D901F060FB6438B0424FF064003A
:1030200003D9BDE8704001F05DBB01F05BFBDEE75A
:10303000F8B5174D35F81150044600201E461746C6
:1030400000F004FC29461422284600F0C3FD4FF688
:10305000FF7000F0FBFB0A222946284600F0BAFD6B
:1030600020460121FFF78CFF63883B80E388338093
:1030700000212046FFF784FF4FF6FF7000F0E6FBCB
:10308000294628461422BDE8F84000F0A3BD00BF41
:10309000EC15010838B500210446C068FFF7EAFCCA
:1030A00000283ED0030C6082A382E0680121012544
:1030B000FFF7E0FC00283BD12046FFF73DFF00F082
:1030C000B5FB054600F0BAFB012281B2A8B200F0C0
:1030D000DDFF0546002833D12346014603F8140BD3
:1030E00004F112022046FFF7A3FF638AA28AE06878
:1030F00043EA02422946FFF7B3FC2346012103F8C5
:10310000185B04F116022046FFF792FFE38A228B38
:10311000E068012143EA0242FFF7A2FC012020748B
:1031200038BD05460121E068FFF7A4FC0028C3D0A4
:10313000030CE0822383002DBED00120207438BD13
:103140004FF6FF7000F088FB4FF4784000F07EFBF4
:10315000164A01239121002000F004FC144A0123A7
:10316000A021002000F0FEFB012D17D0022D0AD077
:1031700000F064FBA0F141010E4A012389B2002056
:1031800000F0F0FBCAE700F059FBA0F141010A4A48
:10319000012389B2002000F0E5FBBFE7074A2B4678
:1031A000AF21002000F0DEFBB8E700BFA814010843
:1031B000B014010804150108F0140108D414010822
:1031C00038B5054608F09EFA022000F071FD00F0C7
:1031D0002DFB044600F032FB022281B2A0B200F0C7
:1031E00055FF00B138BD2846FFF754FFBDE8384011
:1031F00001F01AB810B50E4B5C6982B0202001F0C6
:1032000091FEA30601D402B010BD0A4801A90AF03C
:103210008BFD019B012BF6D14FF0E0234FF0805244
:10322000C3F8042DBFF34F8FBFF36F8F02B010BDF3
:10323000003C014004C8012010B582B00446FFF7ED
:103240007BFD00210B4B01911A6B84F8401142F475
:103250008052C4F83C411A631B6B03F48053019302
:10326000019B0AF0BDFC042005F032FB204602B0B1
:1032700010BD00BF0038024008B5002201210548FA
:103280000AF05CFDBDE80840034A04490148FDF727
:1032900001B900BF04C80120BD04000845080008AA
:1032A00030B5474B474C83428BB04FF0000545D0BB
:1032B0000295236B444843F002032363236B03F01E
:1032C000020302934FF480621223CDE9042300220B
:1032D0000223CDE9062304A90423029A089301F0EE
:1032E000FBFC4FF40072092304A9374804920893A9
:1032F00001F0F2FC0395236C43F480032364236CF8
:1033000003F480030393039B236A43F48003236243
:10331000236A23F4800323622A460F21212001F02F
:1033200005FA212001F03EFA2A460F21222001F061
:10333000FDF9222001F036FA0BB030BD0095236B69
:10334000214843F002032363236B03F0020300933D
:1033500040221223CDE9042300220223CDE90623D3
:1033600004A90423009A089301F0B6FC802304A961
:103370001548049301F0B0FC0195236C43F400134D
:103380002364236C03F400130193019B236A43F429
:1033900000132362236A23F4001323622A460F21B9
:1033A0001F2001F0C3F91F2001F0FCF92A460F216C
:1033B000202001F0BBF9202001F0F4F90BB030BD62
:1033C0000CC8012000380240000402400246034BB2
:1033D000034833F82210002201F098BD18160108A6
:1033E000001002400246034B034833F8221001222A
:1033F00001F08CBD18160108001002400246034B74
:10340000034833F8221001F085BD00BF18160108EB
:10341000001002402DE9F04300228DB00223DFF8B6
:1034200000813B4D3B4FCDE9082306464446A4EBC3
:103430000803052B4ED8DFE803F040331C074D038B
:1034400000200DB0BDE8F083334B002204921A6BCC
:1034500042F020021A631B6B03F020030493049BC9
:1034600037F8023B0693AEB1012E40D0043501344B
:10347000DDE7294B002203921A6B42F020021A6307
:103480001B6B03F020030393039B37F8023B069367
:10349000002EE9D12868079606A901F01DFCE5E792
:1034A0001D4B002202921A6B42F040021A631B6B02
:1034B00003F040030293029BD2E7174B00220192D4
:1034C0001A6B42F001021A631B6B03F001030193B4
:1034D000019BC5E7104B002205921A6B42F0400297
:1034E0001A631B6B03F040030593059BB8E70B4B76
:1034F0002868079306A901F0EFFB94F900900022D9
:1035000048460F2101F012F9484601F04BF9ADE7AA
:1035100004160108F81501080038024000002110C7
:10352000F015010870B5084E084D002435F8021B4F
:1035300056F8040B01F0E4FC20B90134052CF5D158
:10354000204670BDE0B270BD04160108F8150108F0
:1035500010B53D49AEB04FF020400124CDE91A012D
:103560002421CDE90C140222022309201021CDE9E7
:103570000E23CDE91623CDE90A04344A1F91072012
:103580004FF480410023149026914FF480504FF463
:103590000011CDE91C33CDE92033CDE9223310935E
:1035A000159318931E932593279328932B93299370
:1035B00001932490CDE912442A91916B21439163A8
:1035C000916B2140019101990293116B41F0080127
:1035D0001163116B01F00801029102990393116BC1
:1035E00041F010011163116B01F010010391039977
:1035F0000493136B43F020031363136B07940221AE
:1036000003F020030493069103210C2204980891EF
:103610004CF2B37305A90E480992059301F05CFBC7
:103620004FF6807305A90B48059301F055FB05A9DA
:103630000948059401F050FB12AA0AA91AA804F03F
:103640001FFD2EB010BD00BF040100A000380240D5
:10365000000C024000100240001402404FF0C04332
:103660005880BFF34F8F70474FF0C0431880BFF3AF
:103670004F8F70474FF0C043588880B2704700BFEB
:1036800001F030B810B50E4C204603F041F8034667
:10369000A0B90C480C49A360C4E900014FF4804272
:1036A0002046E36022616361A361E3612362FFF767
:1036B000F7FD2046BDE8104001F0D2BE10BD00BFAE
:1036C0000CC8012000540040A086010010B586B04F
:1036D0004FF47A73944602930A46012301460DF192
:1036E00017000090019313488DF817C001F098FF60
:1036F00008B906B010BD0F4801F078FF0D4803F07F
:1037000007F803460028F4D10A4C0B490B48A36084
:10371000C4E900014FF480422046E3602261636106
:10372000A361E3612362FFF7BBFD204601F098FE31
:1037300006B010BD0CC80120A08601000054004056
:1037400010B586B00A46002101234FF47A748DF833
:10375000171001460DF117000090029414480193D0
:1037600002F008F818B99DF8170006B010BD10480F
:1037700001F03CFF0E4802F0CBFF03460028F2D1D7
:103780000B4C0C490C48A360C4E900014FF4804283
:103790002046E36022616361A361E3612362FFF776
:1037A0007FFD204601F05CFE9DF8170006B010BDBD
:1037B0000CC80120A08601000054004010B584B060
:1037C0004FF47A74CDE9002302940A46012301469E
:1037D000134801F0CFFF044610B9204604B010BDD5
:1037E0000F4801F003FF0E4802F092FF0346002845
:1037F000F3D10B480B4A0C4942604FF48042016000
:103800008360C360026143618361C3610362FFF748
:1038100047FD034801F024FE204604B010BD00BF60
:103820000CC80120A08601000054004008B5024BDE
:103830001B689B6A984708BD60C8012008B5024B09
:103840001B68DB6A984708BD60C80120014B1860FF
:10385000704700BF68C80120014B5860704700BF27
:1038600068C80120014B9860704700BF68C80120FC
:103870002DE9F04F394B9C6887B0B4F8049004915F
:10388000A2F12003E188256809F107028446D010DF
:1038900001FB03F3C9EBC00200FB03F3D2B2002922
:1038A00045D01D4409F1FF38DFF8B4A005919044DC
:1038B0002B4600224D460146E14604981E7800EB57
:1038C000020B01291FFA8BFB07D0022932D11E7887
:1038D000587846EA002676BAB6B20024012701914C
:1038E0000293039206E013B11C4A128898470134F0
:1038F000A54214D9A8EB0402DAF8003007FA02F264
:1039000009EB040032425B6980B25946EBD1002BCF
:10391000EDD0124A013492889847A542EAD8039A1A
:1039200005980199029B013290420B44C5D107B022
:10393000BDE8F08F35B15878360446EA002698780D
:103940000643CAE70598013290420B44EFD0049831
:103950001E7800EB020B1FFA8BFBB6E768C801204C
:1039600060C801202DE9F047174612F8014B0646C2
:1039700088461D461CB110460DF01EF9441CDFF8A8
:103980009090DFF890A0D9F800309B6A9847DAF859
:103990000830012D9B88B0FBF3F031D0022D29D0E7
:1039A00033B2002B07F1FF37D8BF0126002409E00E
:1039B0003A78FFF75DFFDAF808309B88013433442A
:1039C000A4B29EB2D9F8003017F8015F9B6A003D9F
:1039D00018BF01259847DAF808209288034602FBB1
:1039E00014339BB293424146304601D3002DDFD1C0
:1039F000BDE8F087001B10FB03F39B1B9EB2CFE7D3
:103A0000001B00FB03F306EB53039EB2C8E700BFA5
:103A100060C8012068C801202DE9F047DFF84CA0FC
:103A2000DAF800502C6A07468846164644B10E4A1A
:103A300033461088A4460A463946BDE8F047604739
:103A40007AB1DFF8249001E0DAF800506B69381998
:103A5000414680B213B1B9F8002098470134A6421C
:103A6000F2D1BDE8F08700BF68C8012060C801201E
:103A70002DE9F041DFF838800C4ED8F80030376877
:103A8000DB6A30609847054660B10024D8F8003002
:103A90009B6A9847A1B2024601340020FFF7BCFFA1
:103AA000AC42F3D1BFB23760BDE8F08168C80120F5
:103AB00060C801202DE9F04F530087B0C3F1030324
:103AC000CDE90001404F414E029392464FF000096C
:103AD0000CE0029BA9EB0A020A330AF1FF3A09F152
:103AE000010903EB8203CA4502936AD33B685B6911
:103AF000002B59D0009A01991FFA89F41FFA8AF510
:103B000002EB040BA1EB05081FFA8BFB1FFA88F8E8
:103B100032885846414698473B68009A5B69121BB9
:103B200090B23288002B3FD0414603909847009ACC
:103B30003B68AA1891B2084601995B693288091B53
:103B400089B2002B30D00591049098473B68009AC9
:103B50005B69A2EB05081FFA88F8328823B3059940
:103B6000404698473B6801995B6932880D44ADB285
:103B7000D3B15846294698473B6832885B699BB168
:103B80002946039898473B6801995B6932880C4441
:103B9000A4B24BB10498214698473B6832885B69D0
:103BA00013B1214640469847094BB360029B002B56
:103BB0008FDA063303EB890309F10109CA45029341
:103BC00094D207B0BDE8F08F60C8012068C801201A
:103BD000780000202DE9F04FDFF8CC9083B0B9F8E1
:103BE0000030C9F80030550082468846C5F103050B
:103BF000164600240192CEB9A4BB002D05F10603A0
:103C00004EDBA31B0A3505EB8305013E0134A642BA
:103C1000F1D2019FB9F80030C9F800303A46414668
:103C2000504603B0BDE8F04FFFF744BF1FFA86FBD4
:103C3000A3B2AAEB0B004FEA4B0B03EB080187B2D0
:103C40001FFA8BFB5A4689B238460093FFF7E4FE11
:103C5000009BA8EB03015A4689B23846FFF7DCFE09
:103C6000002CCAD01FFA84FBB3B2AAEB0B004FEAB8
:103C70004B0BA8EB030187B21FFA8BFB5A4689B2A4
:103C800038460093FFF7C8FE009B03EB08015A4635
:103C900089B23846FFF7C0FE002D05F10603B0DA01
:103CA00003EB8405B2E700BF68C8012000000000F4
:103CB0009FED2B7B70B52C4D2C4BAB6085ED007BC5
:103CC0000446FCF7F5FA2A482A4E0122202101F089
:103CD0001DF900224FF40061274801F017F9052073
:103CE00000F000FD01224FF40061234801F00EF9BD
:103CF0000A2000F0F7FC00224FF400611E4801F09A
:103D000005F9142000F0EEFC01224FF400611A487E
:103D100001F0FCF80A2000F0E5FC7368984785285C
:103D200010D0164C636898474FF6FF73984201D045
:103D3000012070BD124A236814609847114BAB6094
:103D4000002070BD0E4A3368166098470CB1022CF3
:103D5000F4D12046FEF7DAFCF0E700BFAFF30080B5
:103D600000000000FFFF000068C80120880000205C
:103D70000014024040000020000C0240040000201B
:103D800060C801207800002030B595B09FED127B0F
:103D90000521002203460124069110204FF0807176
:103DA000CDE90E21CDE91222CDE902040D920B924C
:103DB000119200924FF480756A4606A908480C9546
:103DC0008DED047B019402F061FE003818BF0120E4
:103DD00015B030BDAFF300800000000000004000CF
:103DE00074C801200000000010B594B04FF480703A
:103DF000062100230C90069119480D9341F2883258
:103E000006A9CDE90E33CDE912330B93119302F0DD
:103E1000CFFD10B1012014B010BD9FED0F7B01222A
:103E20000392022310200522CDE90033029006926E
:103E300006A94FF0807441F288336A4608480F940F
:103E40008DED047B02F022FE003818BF012014B073
:103E500010BD00BFAFF30080000000000000400074
:103E600074C8012070B58AB0384B394800240094DA
:103E70009A6B42F002029A639A6B02F0020200927D
:103E8000009A9A6942F002029A619A6922F002024B
:103E90009A6101941A6B42F040021A631A6B02F0A5
:103EA00040020192019A02941A6B42F002021A63D4
:103EB0001A6B02F002020292029A03941A6B42F009
:103EC00020021A631B6B03F020030393402202239A
:103ED000CDE904230A26012204A90323CDE9062300
:103EE0000925039B089600F0F7FE042304A919484E
:103EF00004930694089500F0EFFE4FF4807304A934
:103F000015480493089600F0E7FE04A94FF40073E7
:103F100011480493089600F0DFFE802304A90E48A0
:103F20000493089500F0D8FE402304A90A4804939E
:103F3000089500F0D1FE22460F215C2000F0F6FB30
:103F40005C2000F02FFC0AB070BD00BF00380240BA
:103F500000180240000402400014024070B5494CB1
:103F6000494B90B02046236002F00EFD054610B18B
:103F7000012010B070BD01462046FFF773FF0422F8
:103F80001023A260E36065604FF0807696FAA6F396
:103F9000B3FA83F3013B4FF48062204623616261F0
:103FA000A561E561256202F07FFC0028E0D1CDE942
:103FB0000A00CDE90E004FF4807566230990079042
:103FC0000D9041F2883202A920460895029302F032
:103FD000EFFC10B1042010B070BD992341F288327B
:103FE00002A92046029302F0E3FC0028F2D141F23C
:103FF0008830FFF7C9FE0028ECD18523CDE90A06F9
:10400000CDE90E0002930990012307900D9041F233
:10401000883202A9204608950C9302F0C9FC0028BA
:10402000D8D141F288320DF10701204602F0A2FEFC
:104030000028CFD1FFF7D8FE0028CBD181230293EF
:10404000F02292FAA2F29DF807300A20B2FA82F228
:1040500000FA02F203F00F03134302A941F288327F
:1040600020468DF8073002F0A3FC0028B2D141F2BF
:1040700088320DF10701204602F0F0FD00283FF4E0
:1040800078AFA7E774C80120001000A070B5114CEC
:10409000114E23683078154698476368702098471A
:1040A000CD2801D0032070BD8DB1022D0CBF082199
:1040B0000C210A4A0A4DA3681170702030702C60E0
:1040C00098472B683078DB689847002070BD062140
:1040D000EFE700BF94000020D0C80120900000202E
:1040E000D4C801202DE9F04FDFF8E0B0344ADBF806
:1040F000003005461B69107883B098472870002867
:1041000059D001AADFF8C8802E4F6E46AA464FF05C
:1041100000091446DBF80030294A5B691078314603
:1041200022469847284B34F8020B1A7836F8023B9F
:10413000110706D5194626F8020C24F8023C03465E
:104140000846910704D5C3F1EF039BB226F8023C61
:10415000520704D5C0F1EF0080B224F8020CD8F861
:104160000020D7F800E093421FFA82FC1FFA8EF17C
:104170008CBFA3EB0C02ACEB030270458CBFA0EB31
:10418000010EA1EB000E92B21FFA8EFE7244052AB8
:1041900004DDC8F80030386001469C462AF802CF9A
:1041A000AAF804102B7809F101094B4508F104081D
:1041B00007F10407AED8002003B0BDE8F08F00BFC0
:1041C000D0C80120C0C8012090000020D4C8012020
:1041D000C8C801200000000000B589B0104B11488C
:1041E000002201921A6B42F040021A631B6B9FED92
:1041F0000A7B03F0400301930122022302A9CDE9C7
:1042000004238DED027B019B00F066FD09B05DF893
:1042100004FB00BFAFF3008020000000000021106D
:10422000003802400018024008B5FFF7D5FF0F2103
:104230000022172000F07AFA172000F0B3FA044B9E
:10424000044A1B6810789B699847002008BD00BF8E
:10425000D4C80120D0C80120704700BF002070479B
:1042600010B50446FFF70EFAA821E0B2FFF768FA8E
:1042700010BD00BF10B582B000240221C0B28DF87D
:104280000740FFF75DFA8DF807009DF8073003F04F
:104290000F038DF807309DF80730022B88BF8DF88B
:1042A00007409DF80710044B9DF807005970002245
:1042B0009A7002B010BD00BFD8C8012070B5164C6E
:1042C0001546A37862789A4282B00E461FD903B38E
:1042D000012B0CBF0921002104230DEB0302C0B206
:1042E000FFF76CFA9DF804309DF805209DF8071043
:1042F0001B0203F470631A439DF8063032801B02E0
:10430000A27803F470631943531C2980A37002B090
:1043100070BD0321E0E700BFD8C801200122A4211D
:10432000C0B2FFF7D3B900BF0022A421C0B2FFF78B
:10433000CDB900BF064A1378834204D05178884231
:1043400001D013B101B170470123D054FFF79AB9DE
:10435000DCC80120704700BF0022A421C0B2FFF7D3
:10436000B5B900BF10B4174A116885B04FF0E0230B
:10437000490400910099D3F8244D2143C3F8241D2A
:104380001168890401910199D3F8244D2143C3F8A0
:10439000241D12680C4912010292029AD3F8144D9E
:1043A0002243C3F8142D0A686FEAC2020392039AEB
:1043B000D3F8141D0A40C3F8142D05B05DF8044B62
:1043C000704700BF304401082C440108012882B026
:1043D0000BD00B4B1B684FF0E022DB430093009B9C
:1043E00011690B40136102B07047064B4FF0E02299
:1043F0001B680193019B11690B43136102B0704765
:104400002C440108304401082DE9F041C468876854
:104410000546164600202B699C4223D2013B1A1BFD
:104420003B1BB34228BF3346934228BF1346184470
:104430006A68F61A03EB04085BB1013C02EB040C5A
:104440000B4411F801EB0CF801EF8B42F9D1AF6886
:104450001946B84514BF44460024EC60002EDAD15A
:10446000BDE8F0815A1E3A44121BD9E7F0B4C36884
:1044700086684468F71A974203EB020523440BD978
:104480003AB1013B0A4411F8014B03F8014F914244
:10449000F9D1C560F0BC704747B1013BCC1911F8A8
:1044A000012B03F8012FA142F9D14468AD1BF0D0D4
:1044B000631E4C1911F8012B03F8012FA142F9D109
:1044C000C560F0BC704700BF10B5154A154C1648C2
:1044D0001649C4E906209FED107B4FF480602062EE
:1044E00010200023C4E91821A0661149A362042208
:1044F000E01D6362E3622367E366636784ED047B28
:104500000CF04CFB0B4B93E803002022A2712060BF
:10451000A18010BDAFF30080030000000300000085
:104520001C150108F0CC0120F0C80120E0C80120D2
:10453000281501082C15010838B5214B00EB400463
:1045400003EBC40E0130DEF82C4000EB4000012CE0
:104550008C46154603EBC00015D0022C0FD034BB9F
:10456000DEF82830DEF8242093429CBFDEF82010CD
:104570005B18013B9A1A95421CD9204638BDBDE80C
:104580003840FFF741BFDEF82830DEF82440A34270
:104590009CBFDEF820105B18013B1C1B944228BF17
:1045A000144622466146FFF761FF204638BD0024CD
:1045B000204638BD2A466146FFF758FF2C46DCE707
:1045C000F0CC0120F8B5054608460C460CF0F4FA8C
:1045D0000A4B1B7806466BB1EFF311874FF02001B1
:1045E00081F31188324621462846FFF7A5FF87F35D
:1045F0001188F8BDFFF768FFEEE700BFF0CC01209F
:104600002DE9F041194D1E462B7804468846174681
:1046100033B32B69A34226D9EFF3118C4FF020015D
:1046200081F3118854B92246131905EBC305069B83
:10463000EB628CF311880020BDE8F081601C00EB78
:104640004000C00004EB440305EBC30345F80080C1
:1046500028440021476062001E6299625962E3E7C4
:10466000FFF732FFD5E74FF0FF30E5E7F0CC012050
:10467000FFF72ABFFEE700BF38B50E4A0E4B12788F
:10468000054618684FF47A73B3FBF2F3B0FBF3F00E
:1046900000F0A4F8044608B90F2D01D9012038BD57
:1046A000024629464FF0FF3000F040F8034B204609
:1046B0001D6038BDBC000020C4000020C0000020E8
:1046C000034A044B11681B780B441360704700BF0A
:1046D00098CD0120BC000020014B1868704700BF36
:1046E00098CD012038B50446FFF7F6FF631C054658
:1046F00002D0044B1B781C44FFF7EEFF401BA04286
:10470000FAD338BDBC0000200749CA6803024FF63F
:10471000FF0003F4E0630240134343F0BF6343F43C
:104720000033CB60704700BF00ED00E01B4BDB683F
:10473000C3F3022300B5C3F1070EBEF1040F03F16A
:10474000040C28BF4FF0040EBCF1060F1CD9A3F1D6
:10475000030C4FF0FF3303FA0CF322EA03024FF08D
:10476000FF3303FA0EF321EA030303FA0CF31343B6
:104770001B010028DBB20ADB00F1604000F561405C
:1047800080F800335DF804FB00229446E7E7044A12
:1047900000F00F00024413765DF804FB00ED00E02A
:1047A000FCEC00E0002807DD4109044A00F01F008E
:1047B0000123834042F82130704700BF00E100E050
:1047C000002808DD4309044900F01F0001222033BE
:1047D000824041F82320704700E100E00138B0F149
:1047E000807F10B403D301205DF8044B70474FF075
:1047F000E023074C58614FF0F00C84F823C00022EE
:10480000072110469A615DF8044B1961704700BF9B
:1048100000ED00E0BFF35F8F044B5A6A002122F4E1
:1048200080325A62C3F89410704700BF00ED00E078
:10483000064B40F00100C3F894005A6A42F48032FB
:104840005A62BFF34F8FBFF36F8F704700ED00E0E8
:104850001849437800B5C1F8983002781AB3436814
:10486000C1F89C30C37A90F80CC090F80FE01B069A
:1048700043EA0C7390F80AC0134343EACC4390F820
:104880000DC0827B43EA8C4343EA424390F809C05F
:10489000027A43EA0E4343EA0C2343EA4203C1F897
:1048A000A0305DF804FBC1F89C20C1F8A0205DF8A1
:1048B00004FB00BF00ED00E04FF0E0220428136984
:1048C0000CBF43F0040323F004031361704700BFDF
:1048D00038B50446FFF700FF0546002C6AD0236870
:1048E000022284F835201A68002122F0010284F89F
:1048F00034101A6005E0FFF7EFFE431B052B37D895
:1049000023681A68D107F6D4A0686268E16825694F
:1049100002430A436169A0692A430A43E1691D68A9
:1049200002430A4331492940256A2A430A43616AFE
:10493000042924D01A605A6922F007021143D8B220
:104940002B4A59611038A2FB0052120929496FF312
:104950000903895CE1655F2888BF04333F228A40F0
:10496000A36500209A600123606584F8353038BD66
:10497000032320226265184684F8353038BDE56A85
:10498000216B2943114319605969A26A21F007017B
:10499000114341F00401002DD1D068B9012A21D082
:1049A00032F00202CBD1EA01C9D54022012362656F
:1049B00084F83530012038BDB0F5005F04D0022AFC
:1049C000F3D9032AEFD0BAE7032AB8D801A050F8E8
:1049D00022F000BFAB490008A7490008AB49000816
:1049E000E5490008B5F1C07FA9D1DEE73F8010F0AE
:1049F000ABAAAAAA3444010870B490F83440856D7B
:104A0000012C0AD090F835404FF0010C644580F835
:104A100034C005D0002380F83430022070BC7047C9
:104A2000022680F83560046800264665266826F46C
:104A30008026266063608368402B0EBFA260A16061
:104A4000E260C26D08BFE1603F239340AB60236822
:104A5000026C43F0160323601AB1236843F0080385
:104A60002360236843F001030020236070BC70477B
:104A700070B50446866DFFF72FFE94F83530022B93
:104A8000054606D080220023626584F83430012078
:104A900070BD23681A6822F016021A605A6922F063
:104AA00080025A61226C32B31A6822F008021A603E
:104AB0001A6822F001021A6005E0FFF70DFE431BA1
:104AC000052B0FD823681B6813F00103F5D1E16DA6
:104AD0003F228A400121B260184684F8343084F8BD
:104AE000351070BD032020220023626584F8343025
:104AF00084F8350070BDA26C002AD5D1D8E700BF7C
:104B000090F83530022B03D0802343650120704795
:104B10000268052380F83530136823F00103002074
:104B200013607047F0B583B0674A876D166800233D
:104B30000193C36D3D6808229A402A42044603D07F
:104B400001680868400778D401229A402A4203D0BD
:104B50002168496908066AD404229A402A4203D08F
:104B60002168096889075CD410229A402A4203D040
:104B700021680868000741D420229A402A4214D0B4
:104B800021680868C00610D5BA6094F83520052A57
:104B900063D00B6813F4802F0B687ED0190340F1AB
:104BA0008980E36B0BB120469847636D23B3636D37
:104BB000DA071AD522684549052384F83530136889
:104BC000A1FB061623F00103B60A136002E0136886
:104BD000DB0704D5019B0133B3420193F7D90022CF
:104BE000012384F8342084F83530E36C23B1204667
:104BF00003B0BDE8F040184703B0F0BDBA600A68E2
:104C000012F4802F0A6822D1D20503D40A6822F058
:104C100008020A60226C002AAED020469047E36D5D
:104C2000AAE7BA60626D42F0040262659CE7BA606E
:104C3000626D42F0020262658EE7086820F00400AF
:104C40000860BA60626D42F0010262657CE71103A0
:104C5000E0D5A26C002AE0D18EE70A6822F01602A5
:104C60000A604A6922F080024A61226C3AB30A68FB
:104C700022F008020A603F2202FA03F3216DBB60B2
:104C80000022012384F8342084F835300029B3D081
:104C9000204603B0BDE8F040084713F4807380D18C
:104CA0000A6822F010020A60012284F8343084F885
:104CB000352076E7636C002B7FF475AF75E7A26C47
:104CC000002AD4D1D7E700BFC4000020B5814E1B15
:104CD00090F83500704700BF2DE9F04F00230D68B4
:104CE00083B04FF0010803E00133102B00F09480F3
:104CF00008FA03F232EA050402EA050AF4D14C6824
:104D00008E684FEA430E24F0100C06FA0EF90CF1EF
:104D1000FF3B032606FA0EF6BBF1010F6FEA06060B
:104D20007DD9C268324042EA0902C2600268164078
:104D300004F0030202FA0EF232430260E200D3D51D
:104D4000674E00220192726C42F480427264726C6F
:104D500002F480420192019A23F0030202F18042A0
:104D600003F0030C0F2702F59C324FEA8C0C07FA74
:104D70000CFE5C4F9668B84226EA0E0623D007F573
:104D80008067B84200F08B80574FB84200F08C80AB
:104D9000DFF85CE1704500F08E80DFF858E1704587
:104DA00000F08F80DFF850E1704500F09180DFF86F
:104DB0004CE170450CBF4FF0060E4FF0070E0EFA97
:104DC0000CFC46EA0C069660484A1268E7036FEA54
:104DD0000A06464F54BF32404AEA02023A607A68F5
:104DE000A703424F54BF32404AEA02027A60BA68CF
:104DF000E7023E4F54BF32404AEA0202BA60FA6804
:104E0000A40203F10103394C54BF32404AEA0202C2
:104E1000102BE2607FF46CAF03B0BDE8F08FD0F8E8
:104E200008B0CF680BEA060B07FA0EFA4AEA0B0A3B
:104E3000C0F808A0D0F804A02AEA020A22099A4081
:104E400042EA0A024260C268324042EA0902BCF108
:104E5000020FC26008D004F00302046802FA0EF2E6
:104E60003440224302603FE70CFA0EFC4FEAD30EB7
:104E700000EB8E0E0C69DEF8209003F00702920022
:104E80000F27944007FA02F229EA02021443CEF8EF
:104E90002040026832404CEA0202026024E708FA2D
:104EA0000CFC46EA0C068EE74FF0020E0EFA0CFCE4
:104EB00046EA0C0687E7032707FA0CFC46EA0C06CD
:104EC00081E74FF0040E0EFA0CFC46EA0C067AE776
:104ED0004FF0050E0EFA0CFC46EA0C0673E700BF15
:104EE000003802400000024000080240003C01403F
:104EF000000C024000100240001402400018024062
:104F000000690840003818BF0120704702B9090441
:104F100081617047436931EA030308BF0904816175
:104F2000704700BF044A5169014208B500D108BD6D
:104F30005061FDF785FF08BD003C01402DE9F843B5
:104F40000F46804616461D464FEA1149B9F1010F3A
:104F5000D8F8003002D111E0691C19D19C696FEAC0
:104F6000040CCCF3400C8CF0010C5FFA8CFC664511
:104F7000F2D00020BDE8F8836A1C09D15C6927EAF9
:104F80000404A4B2B4FA84F46409B442F4D0F0E79F
:104F9000FFF7A2FB089BC01AA84201D8002DD5D16B
:104FA00000222023C8F8302088F83D3088F83E20C1
:104FB000D8F8403088F83C2043F02003C8F840304F
:104FC0000120D7E72DE9F84307460E46904699465B
:104FD0003D686C6926EA0404A4B2002C3ED06B69DB
:104FE0005B050FD4B8F1FF3F03D023E06B695A058E
:104FF00008D46B6926EA03039BB2002BF6D118464E
:10500000BDE8F8832B6843F400732B600022202353
:105010006FF4806169613A6387F83D3087F83E201C
:105020003B6C43F004033B64002387F83C300120D1
:10503000BDE8F883FFF750FBA0EB0900404502D81C
:10504000B8F1000FC4D1002320223B6387F83D2034
:1050500087F83E303B6C13433B64E5E72046CFE7DF
:1050600070B504460D4616462068436913F04003A8
:1050700018D14269D20617D4FFF72EFB801BA84235
:1050800001D8002DF0D100232022236384F83D2095
:1050900084F83E30236C13432364002384F83C30AF
:1050A000012070BD002070BD6FF010012022416111
:1050B000236384F83D2084F83E30236C2364ECE7BE
:1050C000036D5BB9C36C0268012B836C15D0C3F30D
:1050D00007231361036D013303657047036D012BD3
:1050E00003D0036D022B0ED07047836C0268DBB2D5
:1050F0001361036D013303657047DBB21361036D08
:1051000002330365704790F83D30222B0ED090F8A3
:105110003D30212BE8D1426A036812F8011B196166
:10512000438D4262013B9BB24385DDE70268136811
:1051300043F480731360704770B504460D461646FD
:1051400023685A6910062FD45A69510519D46A1C6C
:1051500011D0FFF7C1FA801BA84201D8002DEFD172
:1051600000232022236384F83D2084F83E30236C02
:105170001343236413E05A69150615D45A6956057A
:10518000F9D500226FF4806020215861226384F8F1
:105190003D1084F83E20236C43F004032364002375
:1051A00084F83C30012070BD002070BD70B504460D
:1051B0000D46164623685A6950072FD45A6951057F
:1051C00019D46A1C11D0FFF787FA801BA84201D8B6
:1051D000002DEFD100232022236384F83D2084F8A2
:1051E0003E30236C1343236413E05A69550715D4EA
:1051F0005A695605F9D500226FF480602021586164
:10520000226384F83D1084F83E20236C43F00403AD
:105210002364002384F83C30012070BD002070BD61
:105220002DE9F0479946036890461A6842F4807267
:1052300082B01A605A690A9E0B9FD20705468A46B9
:1052400010D4711C0BD0FFF747FAC01B86422B68A5
:1052500033D3002E31D05A69D00703D4F3E75C6909
:10526000E207FCD50AF0FE021A612A493B463246A3
:105270002846FFF7A7FED8B92B680190596901911C
:105280009B6901933A4631462846019BFFF754FF3C
:10529000044650B9B9F1010F2B6826D15FFA88F2A4
:1052A00020461A6102B0BDE8F0872B6C042B2BD08E
:1052B0000124204602B0BDE8F087002120222963A6
:1052C00085F83D2085F83E102A6C85F83C1042F0A8
:1052D00020022A641B68DC0502D54FF400732B649E
:1052E0000324204602B0BDE8F0874FEA1820186179
:1052F0003A4631462846FFF71FFF0028D5D12A68D5
:105300005FFA88F31361D4E72A68136843F40073E3
:105310001360CDE7020001002DE9F04704689946CB
:10532000236843F4806384B0236023680C9E0D9F40
:1053300043F4807323606369DB0705468A46904621
:1053400010D4711C0BD0FFF7C7F9C01B86422C6824
:1053500052D3002E50D06369D80703D4F3E76369B2
:10536000DA07FCD50AF0FE0323613B493B4632468F
:1053700028465FFA8AFAFFF725FE002838D12B6805
:105380000390596903919B6903933A463146284635
:10539000039BFFF7D1FE40BBB9F1010F2B6842D14F
:1053A0005FFA88F21A613A4631462846FFF7C4FE92
:1053B000D8B902462868016841F48071016033461B
:1053C00000974FF001112846FFF7B8FD2A68002822
:1053D0003ED14AF001032049136128463B4632463C
:1053E00004B0BDE8F047FFF7EDBD2B6C042B29D0CE
:1053F000012004B0BDE8F087002220232A6385F84D
:105400003D3085F83E202B6C85F83C2043F020038E
:105410002B642368DC0502D54FF400732B64032052
:1054200004B0BDE8F0874FEA18221A6131463A46C7
:105430002846FFF781FE0028D7D12A685FFA88F353
:105440001361B0E72A68136843F400731360CFE771
:105450001368DB05E3D5DFE702000100704700BFFA
:1054600070B50446002800F09B8090F83D3003F0B2
:10547000FF02002B00F096802368242284F83D2050
:105480001A6822F001021A601A6842F400421A6097
:105490001A6822F400421A6001F02AFE4D4B61683E
:1054A00099424DD84C4B98427AD922684B4D4900CD
:1054B000A5FB0035431EB3FBF1F3516821F03F011A
:1054C00041EA95415160116AAE0C013621F03F016D
:1054D00031431162D06940F6FC7C013320F44F4027
:1054E00013EA0C0F20F0FF0061D104230343D361C2
:1054F0001168206AE36921F0C00103430B43136084
:105500009168E068236921F40341034321F0FF011E
:105510000B439360D168A069636921F0FF010343E5
:105520000B43D3601168002341F00101202011607A
:10553000236484F83D002363184684F83E3070BD30
:10554000274B98422CD92268244B5668A3FB003C79
:1055500026F03F0646EA9C4656604FEA9C45431EAD
:105560004FF496761F4806FB05F5A0FB0505106A6B
:10557000AD0920F03F00013505431562D069A568EB
:1055800020F44F4020F0FF00A5B901EB4101B3FB2F
:10559000F1F30133C3F30B03CBB143F40043A5E7AD
:1055A000012070BD80F83C20FFF758FF64E7C3F38B
:1055B0000B039BE701EB810101EB8101B3FBF1F3ED
:1055C0000133C3F30B0313B143F440438EE70123CC
:1055D0008CE700BFA08601007F841E0083DE1B4392
:1055E000FF083D00D34D6210704700BF10B5044660
:1055F000A0B10268242380F83D30136823F0010332
:105600001360FFF7F1FF00232364184684F83D3050
:1056100084F83C30236384F83E3010BD012010BD77
:105620002DE9F04F044683B09946BDF834A00E9E94
:105630000F469046FFF750F894F83D30202B054672
:1056400008D0022003B0BDE8F08FFFF745F8401BFB
:1056500019287BD8206883696FEA030C1CF0020BC1
:10566000F3D094F83C30012BEBD003680122DB0728
:1056700084F83C2078D53946076827F4006707602E
:105680000C98606221200195009684F83D0040202E
:1056900084F83E0000202064A4F82AA0608D2085B4
:1056A0003348E0624B4642462046FFF7B9FD0028EA
:1056B00048D1238D5BB32A4631462046FFF73CFD97
:1056C000002837D1676A2068B4F828C039460CF141
:1056D000FF3211F8013B0361638D013B9BB263858F
:1056E000D0F814E0616293B21EF0040F2385E1D07C
:1056F0006BB17A780261628DACF1020C013A1FFA4B
:105700008CF3023792B2676223856285D2E72A461C
:1057100031462046FFF74AFD60B922681368202110
:1057200043F40073136084F83D1084F83C0084F85F
:105730003E0087E7236C042B04D12268136843F4EE
:1057400000731360012003B0BDE8F08F2023C4F87C
:1057500030B084F83D3084F83EB0236C84F83CB01F
:1057600043F0200323646CE703681343036082E77C
:105770000000FFFF2DE9F04F044687B09946BDF8C1
:1057800044A0129E0F469046FEF7A6FF94F83D30C7
:10579000202B054609D00227384607B0BDE8F08F18
:1057A000FEF79AFF401B192849D8206883696FEAE1
:1057B000030C1CF0020BF3D094F83C30012BEAD020
:1057C00003680122D90784F83C2046D5394607688A
:1057D00027F4006707601098606222200195009608
:1057E00084F83D00402084F83E0000202064A4F8A6
:1057F0002AA0608D20858248E0624B4642462046C2
:10580000FFF78AFD0746A8B9238D22684BBB02909B
:105810005369029393690293029B136843F40073E4
:1058200013600023202284F83D2084F83C3084F863
:105830003E30B1E70127384607B0BDE8F08F20239E
:10584000C4F830B084F83D3084F83EB0236C84F85E
:105850003CB043F0200323649DE7036813430360D7
:10586000B4E7012B00F0BC80022B00F08280059091
:105870005169059192690592059A032B4DD8012B28
:1058800000F0A180022B5F49009533464FF00002E3
:1058900020467DD0FFF752FB02460028CAD123687C
:1058A000196821F4806119601969636A1970616A65
:1058B000638D01316162013B218D9BB263854B1E7B
:1058C00023855049009533462046FFF737FB0028D3
:1058D000B0D12368616A1A6842F400721A601B69C9
:1058E0000B70638D626A2168013B9BB26385531C18
:1058F00009696362238D013B23855170238D628D7D
:10590000616A013B013A01319BB292B26162238527
:105910006285002B85D0032BB1D92A46314620461B
:10592000FFF79EFB002885D12268636A12691A700E
:10593000628D2068238D616A013A92B26285426964
:10594000013B9BB201F1010C52072385C4F824C02E
:10595000DFD503694B70628D238D013A92B2628567
:10596000626A013B9BB2013223856262002BD2D175
:1059700057E7116821F480611160116841F40061FA
:10598000116004905169049192690492049A74E739
:10599000FFF7D4FA00287FF44DAF2368616A1A68D4
:1059A00042F400721A601B690B70638D626A013BDE
:1059B0009BB26385238D013B23852368511C1B69A2
:1059C00061625370C7E72A4631462046FFF748FB1D
:1059D00000287FF42FAF23681A69636A1A70BAE748
:1059E000116821F4806111600390516903919169FC
:1059F00003910399116841F4007111603DE700BF04
:105A00000000FFFF04000100704700BF704700BFA7
:105A1000704700BF704700BF704700BF704700BFAE
:105A2000704700BF704700BF704700BF704700BF9E
:105A3000806B38B5416B90F83D400368826B5FFA2C
:105A400084FC39B30024CC63EAB11D68D46325F427
:105A500080651D6044850C65002111651A6822F07F
:105A600001021A6090F83D20602A28D00CF028042A
:105A7000282C17D02022002380F83D2080F83E30CB
:105A8000FFF7D2FF38BD1C6824F480641C60428597
:105A90000A65E3E7EAB11C68D16324F480641C6002
:105AA0004185D9E71A6842F001021A601A6800219C
:105AB00042F480621A60016380F83D40E0E7002311
:105AC000202280F83D2080F83E300364FFF7AEFFCF
:105AD00038BD196821F4806119604285BEE700BFB6
:105AE00090F83D2090F83E100368102910B5D2B20E
:105AF00004464AD002F02801282941D059680805F7
:105B000038D50022226384F83E205A6812F40062DD
:105B10001FD05A68606B22F400625A6090F83530EA
:105B2000012B52D0444B0365FEF7EAFF002869D1F0
:105B3000236C190704D02268536823F4E063536090
:105B400094F83D30226C5207DBB201D5282B65D08A
:105B500010BD94F83D10602921D05A69500605D532
:105B6000626A1B691370636A013363622046FFF740
:105B70005BFFDDE7602AC4D0202284F83D20C0E727
:105B80000022226384F83D10BFE7222AB2D11A68AE
:105B900022F400621A605A681205B2D4ECE72021A0
:105BA00084F83D1022645A69520606D5626A1B6960
:105BB0001370626A2368013262621A6822F001027D
:105BC00020461A60FFF732FFB2E7A06B1A4B03655D
:105BD000FEF796FF0028ABD023685A69510606D518
:105BE000626A1B691370626A2368013262621A6812
:105BF000A06B22F0010220211A60036D84F83D1091
:105C0000984795E72268606B1368202123F0010311
:105C10001360036D84F83D10984789E70023074916
:105C2000E16220222363204684F83D2084F83E3040
:105C3000FFF7F4FE10BD00BF315A00080000FFFF5F
:105C400070B5036804465868E56A94F83E1094F805
:105C50003D2010298CB0D2B25FFA81FC21D0BCF17A
:105C6000400F1ED0216C002900F0CB80596900251F
:105C700011F0020600F08B80860540F18A80226CCC
:105C800002B19D6994F83D2002F02802282A00F014
:105C900027826FF002010022596184F83C200CB089
:105CA00070BD99695A69D6071AD4B5F52A0FF6D08E
:105CB000B5F12A4FF3D012F0080538D0850539D553
:105CC000626C616BD2B21A61002900F0F981CA6B73
:105CD000002A00F076825A6842F400625A60DEE7D9
:105CE000860527D5E26AB2F52A0F00F0EE81E26A56
:105CF000B2F12A4F04BF0822E26294F83E20402A03
:105D000000F0E6812269B2F5804F00F0FE81226D3D
:105D1000002A00F06081226D012AC0D1626CC2F3BA
:105D2000C81202F0060242F0F1021A61B7E79607C4
:105D300000F13D8111F0040F596865D00905AED41A
:105D4000160602F0040140F14F81450540F14C81F7
:105D5000002940F04C8194F83D20208D94F83E10AD
:105D6000E56AD2B2C9B2002840F09A82212A00F036
:105D70008583402993D1222A91D1628D92B2002A43
:105D800040F0A7835A6822F480625A6087E7CD0604
:105D900063D402F0F702212A01F0040500F0B98073
:105DA0004E0640F1F580410540F1F280002D40F0B3
:105DB000F28094F83D10628D92B2C9B2002A3FF48D
:105DC0006EAF626A1B691370638D626A013B9BB29E
:105DD0006385638D01329BB26262002B7FF45FAFFB
:105DE0002A297FF45CAF226853682225282123F4F6
:105DF000806353602046256384F83D10FFF70AFE58
:105E00004DE79D69596933E709053FF548AF5606E7
:105E100002F0040100F1FF8000293FF440AF820549
:105E20007FF53DAFE06A628D616A92B2042A00F0AC
:105E30000E82628D92B2032A00F04482628D92B289
:105E4000022A00F08D821B690B70638D626A013B30
:105E500001329BB26262638521E7850599D594F88A
:105E60003D505A6822F4E0625A600B965A690B92D0
:105E70001A6842F001021A600B9A1A6822F48062D2
:105E80001A605A681005EDB200F1EA80638D9BB28A
:105E900013B323685A6951070AD5626A1B691370E4
:105EA000628D636A013A591C92B22368616262850D
:105EB0005A69520609D5626A1B691370638D626A5A
:105EC000013B01329BB262626385638D9BB21BB161
:105ED000236C43F004032364236C002B40F0EA801E
:105EE0002A2D00F07D8194F83D30282B00F06B8145
:105EF000236B222B02D0222D7FF4D1AE002320224F
:105F00002363204684F83D2084F83E30FFF782FD6D
:105F1000C5E60E0627D5410525D53DBB94F83D00C5
:105F2000618D89B2C0B200293FF4B9AE616A11F83F
:105F3000015B1D616162618D013989B26185618D8D
:105F400089B200297FF4ABAE29287FF4A8AE596846
:105F5000282521F4806159602046226384F83D5051
:105F6000FFF756FD9BE6002D3FF499AE82057FF5C5
:105F700096AE628D92B2002A3FF491AE626A12F838
:105F8000011B1961638D6262013B9BB2638586E6EA
:105F9000002D3FF484AE82057FF581AE628D92B212
:105FA000002A3FF47CAE626A1B6913704DE78605D8
:105FB0007FF5C0AE94F83E20E06A266B94F83D1061
:105FC0002229D2B200F0E2800A955A690A929B69AE
:105FD0000A930A9B63E6626CC2F3C81202F00602DF
:105FE00042F0F0021A615AE600293FF458AE8005EB
:105FF0007FF555AEE16A94F83D20212A00F02E810C
:1060000094F83E30402B7FF44AAE20460CB0BDE8F9
:106010007040FFF755B845057FF5FEAE00297FF4C7
:10602000FEAE94F83D20222A7FF439AE628D92B202
:10603000032A40F2FB81626A1B691370638D626AF6
:10604000013B9BB26385638D9BB20132032B62627D
:106050007FF425AE2268536823F4806353601EE604
:1060600005F0F702222A70D0606B0268526892B283
:106070006285628D92B21AB1226C42F004022264EF
:106080005A6822F400625A60FEF722FE012808D006
:10609000606B944B0365FEF733FD10B1606B036DCD
:1060A0009847638D9BB2002B7FF4F3AE236C002BDB
:1060B0003FF419AF20460CB0BDE87040FFF710BDAB
:1060C000A26B002A7FF403AEE9E50122E26214E646
:1060D000226D002A33D1626C02F0FE021A61DEE505
:1060E0005A682E0622F480625A60C5F3800154BFBC
:1060F000E268A269002381F00101C9B284F83C3052
:1061000092B22046FFF788FCC9E594F83D20212A89
:10611000626C16BF42F0010202F0FE02D2B21A61B6
:10612000626B1AB1D26B002A7FF4D5ADA26B002A44
:106130003FF4B5ADD26B002A7FF4CDADAFE5626C14
:1061400042F00102D2B21A61A9E5A06B026852685E
:1061500092B26285628D92B21AB1226C42F0040250
:1061600022645A6822F400625A60FEF7B1FD0128E9
:106170003FF48CAEA06B5B4B0365FEF7C1FC0028BF
:106180003FF484AEA06B036D98477FE6216D09B99B
:10619000402A7ED0226D22B92169B1F5404F00F02E
:1061A0008380628D92B25ABB03925A6903929A69B4
:1061B0000392039A1A6842F400721A60002323655E
:1061C0006DE5A26BB6E700234749E1622022236315
:1061D000204684F83D2084F83E30FFF71FFC5EE542
:1061E00028222363204684F83D20FFF713FC94F80F
:1061F0003D30282BE7D0236B222B7FF450AD7DE67A
:10620000628D92B2012A73D0628D92B2022A00F09E
:10621000EA801A6842F480621A605A6815050ED541
:10622000202800F28881072840F281812F4A08380F
:10623000C240D00703D55A6842F480525A60002207
:1062400009925A6909929B690993099BB6E75A68B2
:1062500022F480625A601B690B70F6E5628D92B27F
:10626000002A7FF48BAE082963D0202961D011F574
:10627000803F5ED0596821F4E061596011202023ED
:10628000206384F83E20204684F83D30FFF7BCFBB5
:1062900005E501915A6901929B690193019BFEE416
:1062A000212A7FF466AD68E502925A6902929A69E2
:1062B0000292029A1A6842F480721A60236D0133C6
:1062C0002365ECE45A68042822F480625A603FF4A3
:1062D000BAAD02283FF4B7AD1A6822F480621A60A2
:1062E000B1E500BF315A00080000FFFF01010001C5
:1062F00010F5803F00F0F380082800F0DA802028B5
:1063000000F0D780122E00F02A81102800F2298197
:10631000964A0241D60700F124811A6842F480624D
:106320001A60002206925A6906929B690693069BA0
:1063300044E7596821F4E06159601968002220207F
:1063400041F400711960226384F83D0094F83E30F6
:1063500084F83E20402B204698D1FFF761FB9EE455
:1063600001380F2809D8DFE800F03934083408086C
:10637000080808080808080808391A6842F4007272
:106380001A601B690B70638D626A2168013B9BB2C6
:1063900063850B69511C61625370638D2168626A69
:1063A000013B9BB263854B68013223F4407320208C
:1063B00062624B6084F83D0094F83E30402B55D02B
:1063C0000022122384F83E2020462363FFF71EFBA1
:1063D00065E41A6842F480621A60D2E71A6822F40F
:1063E00080621A60CDE7102800F28D80604AC240BA
:1063F000D50740F188801A6842F480621A605A68B2
:1064000012050BD5072840F2A6805A4A0838C24028
:10641000D60703D55A6842F480525A600022089287
:106420005A6908929B690893089BC7E6E16A0229AA
:106430003FF435AC012A3FF632AC1A68606A22F4A8
:1064400080621A605A6822F4E0625A601B69037025
:10645000638D626A013B9BB22021638584F83D1005
:1064600094F83E300132402B6262A9D1002384F8B7
:106470003E3020462363FFF7D5FA10E4082D3FF4A1
:1064800058AF202D3FF455AF15F5803F3FF451AF85
:106490005A6822F4E0625A60112000212023206310
:1064A00084F83E10204684F83D30FFF7ADFAFFF740
:1064B000F6BB1A68002122F480621A6007915A69BB
:1064C00007929A690792079A1A6842F400721A6052
:1064D00074E694F83E20402A7FF450AD95E51A68A2
:1064E00022F480621A605A6812F4006228D01A6896
:1064F000002122F480621A6004915A6904929B6917
:106500000493049B5AE61A6822F480621A601A689F
:1065100042F400621A605A6811057FF57FAF2028A7
:106520007FF670AF10F5803F7FF478AF72E70128F7
:106530007FF485AE7FE610F5803F7FF480AE7AE68B
:1065400005925A6905929A690592059A1A6842F469
:1065500000721A6032E601287FF460AF5AE7012822
:10656000A7D11A6822F480621A60DAE6EBFFFEFF18
:106570001400010001010001F0B503685C6959686D
:1065800090F83E20E60583B0D2B204F400750CD535
:10659000CF0504F480660BD56FF480715961002D2E
:1065A0003FD1002E6DD0012508E01DB1C9051BD4D7
:1065B00003B0F0BD66052ED5C905F9D5418D90F81B
:1065C0003D60076B202A89B2F6B237D06FF4806144
:1065D000102A596145F0040127D0402A25D027050B
:1065E00021D541F008050BE0022504F480666FF424
:1065F00000715961002EE1D1270504D545F0080549
:106600006FF400625A61036C2B43036403B0BDE86E
:10661000F040FFF765BA2405CAD5CA05C8D50825D4
:10662000EEE70325E3E70D46EDE71A68260542F499
:1066300000721A60F7D545F00C05E1E7D9B906F00C
:10664000F702212A03D0282E15D1212F13D190F83B
:106650003D20C16A0829D2B219D0202917D0212A99
:1066600004F4006434D06FF480625A61002CC5D108
:10667000002DC8D19CE76FF480625A6145F0040197
:10668000ADE7250501D50925BAE70125BBE7282A8D
:10669000E5D11E4AC2625A68019022F4E0625A6053
:1066A0006FF480625A611A6822F480621A600023D3
:1066B0002022036380F83D2080F83E30FFF7AEF9DA
:1066C00014F4006F0198D3D0036845F0080597E7EC
:1066D0000E49C1620263202280F83D20002280F82A
:1066E0003E205A68019022F4E0625A606FF48062A2
:1066F0005A611A6822F480621A60FFF789F90198DA
:10670000002CE1D1002D7FF47EAF51E70000FFFFA8
:1067100090F83D00704700BF10B40D4C0D4A23683F
:1067200023F00303034323601369012943F00403A7
:1067300013610AD040BF20BF20BF064A5DF8044B5A
:10674000136923F004031361704730BFF5E700BFFE
:106750000070004000ED00E04B6A2DE9F04133B1DC
:10676000B2F1406F03D08C6A0568013C2C618C69E2
:106770000E6AD1F81C804CB343EA040C4B690068E4
:10678000CF6A0D6B4C6B4FEA834E4CEA020C0B68E0
:10679000002E4CD04CEA060C8E68C6610E69B8F12A
:1067A000000F4DD043EA08033B432B4323433343BD
:1067B000CC68234343EA0E0343EA0C03B2F1406F73
:1067C000436146D04B688361BDE8F081F6B14C6906
:1067D0000068CF6A4D6B43EA060C8B68C3610E6B91
:1067E0000B694CEA020CA404B8F1000F3DD043EA57
:1067F00008033B4333432B43CD682B43234343EAF6
:106800000C03B2F1406F4361DCD122E0B8F1000F1C
:1068100034D1F3B1CC6A006823430C6B1343234398
:106820004C6B4A69234343EA8243436111E0B8F168
:10683000000F10D043EA08033B432B432343B7E741
:106840003B432B432343334343EA0E0343EA0C0306
:106850004361BDE8F0813B432B43234343EA0E03EE
:1068600043EA0C034361BDE8F0813B4333432B43D0
:10687000234343EA0C034361BDE8F081CC6A00681E
:1068800043EA0803134323430C6B23434C6B23431A
:10689000CC6823434C69B2F1406F43EA84434361BF
:1068A00090D1D6E7704700BF70B50446FDF714FFDE
:1068B0000546002C59D094F8413003F0FF02002B1C
:1068C00049D0A66C2268A1681368013923F4F853F3
:1068D00043EA0123136093689B060CD5711C33D0E7
:1068E000FDF7FAFE401BB04241D8002E3FD022688F
:1068F00093689806F4D4E569E368116860682B43EF
:10690000256A21F07F412B4343EA006321F0D00147
:106910000B431360A5696369506819492B432569C6
:10692000014043EA05430B4353601368002143F0E1
:1069300001034FF0010C13600846616484F841C004
:10694000002384F8403070BD93689B06D3D59368CC
:106950009B06F9D4CFE784F840202046FFF7A2FF3A
:1069600041F288331E46A364ACE7012070BD0423C6
:1069700084F84130636C012003436364E0E700BFA7
:10698000FEF8E0FF704700BF10B5044670B1026822
:10699000136823F001031360FFF7F4FF002363641F
:1069A000184684F8413084F8403010BD012010BDF5
:1069B0002DE9F84304460D461746FDF78DFE94F881
:1069C0004030012B804638D0012384F8403094F8C1
:1069D0004130012B5FFA83F907D04FF00209002301
:1069E00084F840304846BDE8F88300236364266895
:1069F000022384F84130B368980611D57A1C0CD074
:106A0000FDF76AFEA0EB0800874237D3002F35D090
:106A10002668B3689906F3D402E0B3689B06FCD4F9
:106A2000002229462046FFF797FE6B6A53B10123E7
:106A300084F841304FF00009D1E74FF00209484691
:106A4000BDE8F883B368990710D47A1C0BD0FDF722
:106A500043FEA0EB08039F4210D37FB12668B368C2
:106A6000980703D4F3E7B3689B07FCD50222012300
:106A7000F2604FF0000984F84130B0E7042384F855
:106A80004130636C43F001036364A8E72DE9F84FDC
:106A900081461E468A469346FDF71EFE99F8403011
:106AA000012B074666D0012389F8403099F8413020
:106AB000012B5FFA83F807D04FF00208002389F812
:106AC00040304046BDE8F88F0023C9F84430D9F87B
:106AD0000040422389F84130A368990611D5731C00
:106AE0000CD0FDF7F9FDC01B864248D3002E46D0DE
:106AF000D9F80040A3689A06F3D402E0A3689D0683
:106B0000FCD4DBF80030A362DBF804306362DBF80E
:106B10000830E3622568DBF8103025F4400C4CEABD
:106B2000030C4CF48002DBF80C3022604846CAF8B3
:106B300028304FF000625146FFF70EFEA368180799
:106B400010D4721C0BD0FDF7C7FDC01B864216D3B4
:106B5000AEB1D9F80040A368190703D4F3E7A368DE
:106B60001B07FCD508220123E2604FF0000889F8DA
:106B70004130A3E74FF002084046BDE8F88F0423F8
:106B800089F84130D9F8443043F00103C9F8443062
:106B900094E700BF70B50446FDF79EFD94F84130C0
:106BA0009907054638D50022236884F840201A68E2
:106BB00052073AD41A6842F002021A609A6896079D
:106BC0000DD4A66C711C29D0FDF786FD401B8642B2
:106BD0003AD3002E38D023689A689007F4D5022261
:106BE000DA609A68920610D5A66C711C0AD0FDF77F
:106BF00073FD401B864227D336B323689A689006FC
:106C0000F5D402E09A689206FCD45A69012122F078
:106C100040625A6184F84110002070BD9A6896075E
:106C2000DDD49A689607DAD4F8E71A68E06B22F0A8
:106C300004021A60FDF71CFF23680028BAD0626CBA
:106C400042F004026264B5E7042384F84130636CC7
:106C500043F001036364012070BD00BF2DE9F843D8
:106C6000044689461546FDF737FD94F84030D4F8C0
:106C70000080012B064664D0012384F8403094F84C
:106C80004130012BDFB206D00227002384F84030C8
:106C90003846BDE8F88300236364B9F1000F5CD087
:106CA000122384F84130D8F810300133E362D8F869
:106CB0001030C4F824900133A362D8F8143023F0C4
:106CC0004063C8F81430E36A42460BB393685B072D
:106CD00010D4681C0BD0FDF7FFFC801B854234D319
:106CE000002D32D023689B685A0703D4F3E79368DA
:106CF0005907FCD5636A1B7888F82030E16A636A1B
:106D000022680139E162E16A013363620029DDD161
:106D1000936898070BD4691C24D0FDF7DDFC831B16
:106D20009D4212D38DB1226893689B07F5D502234B
:106D3000D3602046FFF72EFF0746012384F8413039
:106D4000A3E702273846BDE8F883042384F84130DE
:106D5000636C43F001036364EFE7636C43F0080383
:106D6000636492E793689B07E1D493689B07F9D526
:106D7000DDE700BF2DE9F843044615468946FDF7D7
:106D8000ABFCD4F80080D8F8182094F84030012BE0
:106D900006466BD0012384F8403094F84130012B33
:106DA000DFB206D00227002384F840303846BDE821
:106DB000F88300236364B9F1000F63D0222384F8C1
:106DC0004130D8F810300133A363D8F81030C4F83C
:106DD000309001336363D8F8143023F0406343F0FC
:106DE0008063C8F81430C8F81820A36B424623B358
:106DF000936813F0060F12D1691C0CD0FDF76CFCE0
:106E0000801B854236D3002D34D023689B6813F055
:106E1000060F04D1F2E7936813F0060FFBD0236B43
:106E200098F820201A70A16B236B22680139A163A6
:106E3000A16B013323630029DAD1936898070BD43F
:106E4000691C24D0FDF748FC831B9D4212D38DB1F1
:106E5000226893689B07F5D50223D3602046FFF78D
:106E600099FE0746012384F841309CE70227384603
:106E7000BDE8F883042384F84130636C43F00103D8
:106E80006364EFE7636C43F0080363648BE7936824
:106E90009B07E1D493689B07F9D5DDE770B5244ED5
:106EA00088B00D461446F8B90090336B43F00103E7
:106EB0003363336B069003F0010300934FF4807249
:106EC0000223CDE902231B480022032302A9CDE9B6
:106ED0000423009BFDF700FFB36823F0EC632B4312
:106EE0002343B36008B070BD00220192336B124897
:106EF00043F004033363336B069203F004030193FE
:106F00004FF400720223CDE9022302A900220323D9
:106F1000CDE90423019BFDF7DFFEB36823F078433E
:106F200043EA050141EAC401B16008B070BD00BF89
:106F3000003802400000024000080240014B0122DC
:106F4000DA64704700004742164908B58B6803F0C1
:106F50000C03042B1BD0082B01D0134808BD4A6832
:106F60004B68496813F4800302F03F0211D10E48C8
:106F7000C1F38811A1FB000108F0C4FB094B5B6859
:106F8000C3F3014301335B00B0FBF3F008BD0748D6
:106F900008BD0648C1F388110023A1FB000108F0D9
:106FA000B1FBEBE7003802400024F40000127A0045
:106FB0002DE9F0410D46044660B1454A136803F0DF
:106FC0000F038B4209D2CBB21370136803F00F0387
:106FD0008B4202D00120BDE8F0812368980714D5C8
:106FE000590704D53B498A6842F4E0528A601A077F
:106FF00004D538498A6842F460428A603549A068FD
:107000008A6822F0F00202438A60DF0721D56268B5
:10701000012A55D0931E012B2E4B1B684DD9990781
:10702000D8D52C4EB36823F003031343B360FDF7A8
:1070300053FB41F28838074604E0FDF74DFBC01BC7
:10704000404542D8B368626803F00C03B3EB820F8B
:10705000F3D11F4A136803F00F03AB4206D9EBB21A
:107060001370136803F00F03AB42B3D123685A07C0
:1070700006D51849E0688A6822F4E05202438A6023
:107080001B0707D5134A2169936823F4604343EA39
:10709000C1039360FFF758FF0E4A0F4C92680F49E7
:1070A000C2F303120346A25C0D48D34000680B6094
:1070B000FDF7E2FA0020BDE8F0819801B1D489E73C
:1070C000044B1B689E03ACD484E7032083E700BF16
:1070D000003C02400038024044440108C400002043
:1070E000C0000020014B1868704700BFC40000209A
:1070F000044B05499B68054A0868C3F38223D35CA7
:10710000D840704700380240C40000203C440108C9
:10711000044B05499B68054A0868C3F34233D35CB6
:10712000D840704700380240C40000203C440108A9
:107130000E4B0F2210B402609A680D4C02F003024D
:1071400042609A6802F0F00282609A6802F4E052AB
:10715000C2609B68DB0803F4E053036123685DF8B9
:10716000044B03F00F030B60704700BF0038024070
:10717000003C02402DE9F041036813F0010582B0A4
:1071800004460BD0A4494569D1F88C2022F0C06296
:107190002A43B5FA85F5C1F88C206D099E070CD5F8
:1071A0009D48A169D0F88C2022F0C0520A43C0F853
:1071B0008C20002908BF45F00105180700F19F80C9
:1071C0005F0705D5954B94F83820C3F8E021236874
:1071D000DE0608D59049606AD1F8942022F4400276
:1071E0000243C1F89420980603F0400134D58A4840
:1071F000A66AD0F8942022F000623243B6F1006F04
:10720000C0F8942000F0E180002900F0C08082499D
:10721000206AD1F8942022F080520243012DC1F857
:1072200094201FD0DA0508D57B49E06AD1F88C207C
:1072300022F000420243C1F88C209B0508D5764A13
:10724000216BD2F88C3023F400430B43C2F88C300E
:10725000002002B0BDE8F0810029D8D1012D01D075
:10726000802BDFD16E4B6C4E00229A66FDF734FA0C
:10727000054604E0FDF730FA431B022B3BD8336888
:107280001A01F7D4654B626BC3F8D8202268D30784
:1072900040F181806369002B7DD1E368A06861685B
:1072A0001B0643EA801320690B435B4943EA0073E2
:1072B000C1F8843010060CD5E368A06862682169C3
:1072C0001B0643EA80131343534A43EA0173C2F88F
:1072D0008430534B504E01229A66FDF7FDF9054666
:1072E00004E0FDF7F9F9401B022804D833681901BE
:1072F000F7D5236896E7032002B0BDE8F081464B3E
:10730000484E002201921A6C42F080521A641B6CA3
:1073100003F080530193019B336843F4807333601F
:10732000FDF7DAF9074604E0FDF7D6F9C31B022B97
:10733000E1D83368D905F7D5374EE369326F12F4D7
:10734000407203F4407112D08A4210D0336F344A35
:107350000121C2F8401E23F440730021C2F8401EF0
:107360003367336FDA0747D4E36903F44071B1F54B
:10737000407F36D028498A6822F4F8128A60264A6B
:10738000116FC3F30B030B431367236818E7012D39
:107390007FF448AF66E7970703D5A369002B3FF456
:1073A0007CAF960604D5A36AB3F1006F3FF475AFC6
:1073B00055067FF57FAF236A002B7FF47BAFA36A6E
:1073C000B3F1006F7FF476AF67E700293FF44AAF6F
:1073D000D0F89430226A23F080531343C0F89430DD
:1073E00040E70D48826823F0704122F4F81221F43E
:1073F00040710A438260C2E7FDF76EF941F28838B6
:10740000074605E0FDF768F9C01B40453FF673AF3E
:10741000336F9B07F6D5A7E70038024000104742BC
:1074200000004742007000402DE9F0410368DD078D
:1074300082B004462FD59F498A6802F00C02042AC4
:1074400000F0C2808A6802F00C02082A00F0B880BE
:107450006368B3F5803F00F0F980B3F5A02F00F02A
:107460004C81944D2A6822F480322A602A6822F4E2
:1074700080222A60002B40F0EE80FDF72DF90646B1
:1074800005E0FDF729F9801B642800F202812B68D2
:107490009B03F6D423689F0728D5864A916811F08C
:1074A0000C0F00F09F80916801F00C01082900F09A
:1074B0009580E368002B00F00F817F4B7D4E012209
:1074C0001A60FDF709F9054605E0FDF705F9401BCF
:1074D000022800F2DE8033689807F6D53368226907
:1074E00023F0F80343EAC203336023681A0716D572
:1074F0006369002B00F081806F4B6E4E0122C3F850
:10750000802EFDF7E9F8054605E0FDF7E5F8401B9C
:10751000022800F2BE80736F9B07F6D523685807D8
:107520002FD5644A136C13F0805377D00025634E37
:107530003368D90540F19D80A368012B00F0AD8030
:10754000052B00F019815B4E326F22F00102326789
:10755000326F22F004023267002B40F0A380FDF767
:10756000BBF841F28838074605E0FDF7B5F8C01BC7
:10757000404500F28E80336F9807F6D4002D40F01E
:10758000C680A369C3B14B4DAA6802F00C02082A59
:107590002FD0022B484B4FF000021A6600F0BD803E
:1075A000FDF79AF8044604E0FDF796F8001B022860
:1075B0006FD82B689B01F7D4002002B0BDE8F081A2
:1075C0004A6850027FF544AF3A4A126891037FF54A
:1075D00062AF6268002A7FF45EAF0AE0526856022A
:1075E0003FF567AF334A1268950723D5E268012A51
:1075F00020D0012002B0BDE8F0812F4A2D4EC2F804
:10760000803EFDF769F8054604E0FDF765F8401B8C
:1076100002283ED8736F9F07F7D47FE70193136C5E
:1076200043F080531364136C03F080530193019B68
:1076300001257CE71F4920690A6822F0F80242EA26
:10764000C0020A601A077FF56AAF51E7194A13684A
:1076500043F480331360FDF73FF8164E054604E00F
:10766000FDF73AF8401B642813D833689A03F7D51E
:1076700010E7336843F480733360FDF72DF8074655
:107680003368DA053FF558AFFDF726F8C01B02282E
:10769000F6D9032002B0BDE8F081064A136F43F02B
:1076A00001031367FDF718F8024F064641F28838C8
:1076B0000BE000BF0038024000004742007000406D
:1076C000FDF70AF8801B4045E3D83B6F9B07F7D5D1
:1076D000002D3FF456AF1AE02C4A2D4E1360FCF7F4
:1076E000FBFF054604E0FCF7F7FF401B0228D0D85B
:1076F00033689907F7D42368F8E6254B1A6842F4F3
:1077000080221A601A6842F480321A60A3E7204A85
:10771000136C23F08053136433E7FCF7DDFF064658
:1077200004E0FCF7D9FF801B0228B2D82B6899012E
:10773000F7D4216AE369626AE06A0B4343EA821381
:10774000A26A216B43EA0063520843EA0173013ADB
:107750000E4943EA024301226B600A66FCF7BCFF54
:107760000B4D044604E0FCF7B7FF001B022890D83D
:107770002B689A01F7D51FE7054B1A6F42F00402F8
:107780001A671A6F42F001021A678BE7000047423E
:1077900000380240704700BF10B50446A0B14379DD
:1077A00003F0FF0263B12168022363710B680022BA
:1077B00043F0040301200B6060711046A26010BD0D
:1077C0000271FFF7E7FFEEE7012010BD704700BF31
:1077D00038B50446002860D0437F03F0FF02002B39
:1077E0005DD0236853220220CA21607759625A6211
:1077F000DA6855063CD599686268256921F4E0018C
:1078000021F040019960616998682A430A43024364
:10781000E1689A6019611A69A16842EA01421A6135
:10782000DA6822F08002DA609A6891060DD51A6C47
:10783000A06922F480221A641A6C02431A64FF21A0
:10784000012259620020627738BDDA6822F0A00276
:10785000DA60FCF741FF054605E0FCF73DFF401B01
:10786000B0F57A7F14D82368DA689206F5D5DEE79A
:107870004FF0FF32DA60FCF72FFF05462368DA6825
:107880005006B8D4FCF728FF401BB0F57A7FF5D935
:107890002268FF21042351626377012038BD0277FB
:1078A000FFF794FF9DE700BF0368503343F82120A2
:1078B000704700BF0368503353F82100704700BF82
:1078C0002DE9F04106689846B36831EA03030CBF1E
:1078D00001230023934207460C4615460AD0B8F10F
:1078E000FF3F12D1B36834EA03030CBF0123002326
:1078F000AB42F7D10020BDE8F0819B6834EA030376
:107900000CBF01230023AB42F4D0FCF7E5FE069B3D
:10791000C01A40453B68F0D379685A68B1F5827F58
:1079200022F0E0025A6013D0BA6AB2F5005F07D1C4
:107930001A6822F400521A601A6842F400521A605F
:107940000122002387F8512087F850300320D2E726
:10795000BA68B2F5004F02D0B2F5806FE4D11A6870
:1079600022F040021A60DFE730B5174B174D1B6855
:10797000A5FB035C85B04FEA5C5C4FF47A7303FBB4
:107980000CF303934368B3F5827F044607D10CE000
:10799000039B2268013B039393681B0602D5039B5C
:1079A000002BF5D1002005B030BD00920B4600221F
:1079B0008021FFF785FF0028F4D0636D43F020039A
:1079C00003206365EFE700BFC4000020819F5E16BF
:1079D00030B50B4611464268B2F5827F83B004464B
:1079E00008D0009100220121FFF76AFF88B900202A
:1079F00003B030BD8268B2F5004F1ED0B2F5806F83
:107A00000ED00091002280212046FFF759FF002868
:107A1000EDD0636D032043F02003636503B030BDF8
:107A200005682A6822F040022A60009100220121A4
:107A3000FFF746FF0028DAD0EBE70068026822F083
:107A400040020260DDE700BF704700BF70B504462A
:107A500000283BD090F8513003F0FF02002B30D0CB
:107A600004F1080007C86368666A03430B43616951
:107A7000E06913430B432268216A022584F85150C0
:107A800003430B431168A069A56A21F0400111600E
:107A90002B43010C00F400700343136001F0040356
:107AA0003343B5F5005F536004BFE36A1361D369E4
:107AB000002023F400630121D361606584F8511034
:107AC00070BD80F85020FFF7BFFFC9E7012070BDEF
:107AD00090F85030012B70B504465ED090F85130CC
:107AE0000120834284F85000DDB205D00225002336
:107AF00084F85030284670BD0029F8D0002AF6D00E
:107B0000032384F8513000236365A363E286636432
:107B10002364A387E387A368A286B3F5004F226896
:107B2000216335D0A36AB3F5005F28D0A06C1C4E4A
:107B3000E38E06641B4EC6631B4EC66400260C32E1
:107B40009BB20665FCF758FF88B923681A6852068D
:107B500003D41A6842F040021A605A6842F02002C8
:107B60005A605A6842F0020200255A60BFE7636D0E
:107B7000012243F01003636584F85120B7E71368CE
:107B800023F400531360136843F400531360CDE7EC
:107B9000136843F480431360C4E70225284670BD90
:107BA000D97C00082D7D0008097D000838B5044601
:107BB00090F8500001287ED0012084F8500094F8FD
:107BC000510001285FFA80FC0ED06068B0F5827F1A
:107BD00004D00220002384F8503038BDA06800286B
:107BE000F7D1BCF1040FF4D1002962D0002A60D093
:107BF000002B5ED094F85100A38604281CBF0520FA
:107C000084F8510000206065A387E386E387A36AB8
:107C10002163B3F5005F2168A2632064606407D12B
:107C20000B6823F400530B600B6843F400530B60A4
:107C300094F85130E06C042B14BF204B204BC363ED
:107C4000204BC3644FF000030365E38F14BF1E4D48
:107C50001E4D05640C319BB2FCF7CEFE014608BBFD
:107C60002268A06C536843F001035360E38E016403
:107C7000C163C16401659BB2216B0C32FCF7BCFE91
:107C800080B923681A68520603D41A6842F0400289
:107C90001A605A6842F020025A605A6842F00202A2
:107CA0005A6097E7636D012243F01003636584F81F
:107CB000512001208EE7022038BD00BF517E000810
:107CC0009D7D0008097D0008F97C0008E97C00081A
:107CD000704700BF704700BF08B5806BFFF7FAFF21
:107CE00008BD00BF704700BF08B5806BFFF7FAFF03
:107CF00008BD00BF704700BF08B5806BFFF7FAFFF3
:107D000008BD00BF704700BF806B026808B55368AC
:107D100023F003035360436D012143F010034365D7
:107D200080F85110FFF7EEFF08BD00BF30B50546E3
:107D300083B0846BFCF7D0FC2B681B68DB05024624
:107D400021D42368586820F020005860586820F03B
:107D50000200586064212046FFF706FE18B1636DEB
:107D600043F020036365A36833B922680193D368A5
:107D7000019393680193019B01230022E28684F81A
:107D80005130636D23B92046F9F7DEFC03B030BDF6
:107D90002046FFF7B7FF03B030BD00BF70B5054602
:107DA00082B0846BFCF798FC2B681B68D9050646EB
:107DB00021D42368A16A5A68B1F5005F22F020023D
:107DC0005A6035D0A26852B35A6822F001025A6054
:107DD000324664212046FFF7FBFD08B1202363658E
:107DE000012223680021E18784F851209A68D20695
:107DF00006D4636D73B92046FFF76AFF02B070BD09
:107E0000626D4FF6EF7142F0020262659960636D38
:107E1000002BF0D02046FFF775FF02B070BD6268FE
:107E2000B2F5827FD0D15A6822F003025A60CFE7C0
:107E300001220090642311462046FFF741FD18B14E
:107E4000636D43F0020363652368DA68BAE700BF35
:107E500070B5054682B0846BFCF73EFC2B681B684E
:107E6000D905064622D42168A26A4B68B2F5005FA4
:107E700023F020034B602DD0324664212046FFF7CB
:107E800073FD18B1636D43F02003636523685A687E
:107E9000002122F0030201205A60E186E18784F884
:107EA00051009A68D20606D4636D73B92046F9F77B
:107EB00065FC02B070BD626D4FF6EF7142F00202D8
:107EC00062659960636D002BF0D02046FFF71AFFC2
:107ED00002B070BD01220090642311462046FFF7D6
:107EE000EFFC18B1636D43F0020363652368DB6840
:107EF000C2E700BF30B502685168936813F0400FC5
:107F000085B00446C3F3801519D113F0010F2FD1AA
:107F1000980745D49D0600F19180DB050DD58D06AF
:107F20000BD5636D002043F00803636503909368ED
:107F30000393039B636D002B5AD105B030BD13F042
:107F400002001AD008067CD413F020002CD18D0634
:107F5000F3D594F85150032D79D0656D45F00405A3
:107F600065650090D06800909068009000983AE0B5
:107F700011F0400FCCD0036C65E08D06DDD594F890
:107F80005150032D63D0656D45F004056565009083
:107F9000D0680090906800900098980623D515E06E
:107FA00008064ED49806B8D58806C6D575B194F89B
:107FB000510003284BD0606D40F004006065002044
:107FC0000090D0680090906800900098606D40F03C
:107FD000010060650020029090680290106820F017
:107FE000400010600298DB059BD4636D002BA4D089
:107FF0005368012023F0E0038D07536084F851009B
:108000002DD05368E06C23F00303536040B1164B4E
:108010000365FCF775FD18B1636D43F040036365BC
:10802000A06C002889D0104B0365FCF769FD00287F
:1080300083D0636D43F0400363657EE78806C5D453
:108040007BE7636C204605B0BDE83040184700234D
:108050000193D368019393680193019B6DE72046D8
:10806000FFF750FE69E700BF6D80000808B5806B20
:108070000023C387C386FFF745FE08BD704700BFD6
:1080800070B50E461546044618B390F8493003F013
:10809000FF02CBB1214651F8080B00F053FBA26858
:1080A0002068314600F08CFB236BA268606829468B
:1080B00000F0B2FB2268A16852F8213043F00103BE
:1080C00042F82130002070BD80F84820FFF7D6FF2D
:1080D000E0E7012070BD00BF704700BF0368DA68A9
:1080E00042F00102DA609A6802F00702062A03D021
:1080F0001A6842F001021A60002070470368DA68CB
:1081000022F00102DA601A6A41F211110A4208D122
:10811000196A40F24442114203D11A6822F0010266
:108120001A600020704700BF704700BF704700BF53
:10813000704700BF704700BF704700BF03681A69EF
:10814000910710B5044602D5DA6892075FD41A6920
:10815000500702D5DA68510746D41A69120702D5CA
:10816000DA6810072ED41A69D20602D5DA68D0066A
:1081700018D41A69D10702D5DA68D2075DD41A6912
:10818000100602D5DA6811065FD41A69520602D5C4
:10819000DA68500661D41A69910602D5DA68920647
:1081A00043D410BD6FF010021A61DB69082213F48A
:1081B000407F2277204664D0FFF7BAFF0022236871
:1081C0002277D6E76FF008021A61DB69042299076B
:1081D0002277204652D1FFF7A9FF2046FFF7AAFFDA
:1081E000002223682277BEE76FF004021A619B69C0
:1081F000022213F4407F227720463CD1FFF796FFFE
:108200002046FFF797FF002223682277A5E76FF04B
:1082100002021A619B6901229B07027725D0FFF7B2
:1082200087FF00222368227791E76FF02002204623
:108230001A61BDE8104000F0B7B86FF001021A6192
:108240002046FFF771FF236899E76FF080021A61FB
:10825000204600F0ABF8236897E76FF040021A6100
:108260002046FFF769FF236895E7FFF75FFF204689
:10827000FFF760FFD5E7FFF75BFFC4E7FFF758FFA5
:10828000AEE7FFF753FF2046FFF754FF96E700BF26
:10829000354A0368904210B44DD0B0F1804F34D0CD
:1082A000A2F57C42904230D002F5806290422CD000
:1082B00002F58062904228D002F5784290423AD08E
:1082C0002A4A904225D002F58062904221D002F5E0
:1082D000806290421DD0A2F59832904219D002F5EA
:1082E0008062904215D002F58062904211D08C6875
:1082F0000A68496923F080030B4303600123C462C9
:1083000082625DF8044B436170474A6823F0700352
:108310001343CC684A6923F44073234323F080035A
:1083200013438C680A6803600123C46282625DF8AB
:10833000044B436170474C68CA6823F070032343C1
:1083400023F4407313434A695DF8044B23F0800320
:10835000134303608B68C3620B6883620B6903631A
:1083600001234361704700BF00000140004001400D
:1083700010B50446B0B190F83D3003F0FF0263B190
:108380002146022351F8040B84F83D30FFF780FFAB
:108390000123002084F83D3010BD80F83C20FFF719
:1083A0009BFEEDE7012010BD704700BF704700BF86
:1083B0000268116938B50446C068A368256921F4CC
:1083C000405101431161D168E0692B43656921F493
:1083D00016412B4321F00C0103430B43D360536937
:1083E000A16923F440730B43B0F5004F5361284B50
:1083F00023D09A421ED003F580639A421AD0FEF72A
:1084000077FE636819219A00A0FB01019B0F07F01A
:1084100079F9204AA2FB00135B092168642404FB5C
:10842000130000013230A2FB00201B0103EB5013AC
:108430008B6038BDFEF76CFEE3E79A4225D003F56A
:1084400080639A4221D0FEF753FE62681921921888
:108450004FF000035B41A0FB010107F053F90D4A07
:108460002468A2FB00314909642303FB1103DB00EC
:108470003233A2FB0323C3F342121B0902EB0112A6
:1084800003F4F8731344A36038BDFEF741FEDCE744
:10849000001001401F85EB51704700BF38B50446FE
:1084A00050B390F8393003F0FF0203B3226824235D
:1084B00084F83930D36823F400532046D360FFF7A3
:1084C00077FF23681A6922F490421A615A6922F0F0
:1084D0002A025A61DA680025202142F40052DA604B
:1084E0002846E56384F8391084F83A1038BD80F8DE
:1084F0003820FFF7D1FFD9E7012038BD704700BF12
:10850000704700BF90F83A30222B10B522D1816815
:1085100002690468836AB1F5805F1CD0591C12BBE4
:10852000626881621A70C38D013B9BB2C3858BB9AF
:108530000368DA6822F02002DA60DA6822F48072D6
:10854000DA605A69202122F001025A6180F83A105B
:10855000FFF7D6FF10BD62B96268C2F3080223F8C4
:10856000022B8362DFE76268816202F07F021A7089
:10857000D9E76268D2B223F8012B8362D3E700BF48
:10858000704700BF03681A6870B51607DD6859693F
:1085900004460CD1960601D5A90671D4160601D55C
:1085A000280646D4510601D56A065ED470BD11F086
:1085B000010129D115F4907FF0D0D60709D5E8053F
:1085C00040F1A180E06B40F00100E063500764D50A
:1085D000F1B9960766D5100700F19280E16B00298A
:1085E000E4D0900602D5A90600F191805A69E16BAA
:1085F00002F0400201F0080152EA01055CD1204678
:10860000FFF7BEFFE56370BDD60742D450073BD5E8
:10861000E16B41F00201E163910737D5E16B41F075
:108620000401E1631107D9D5E16B41F00801E16371
:10863000D4E794F83920212AB8D1A168226AB1F58B
:10864000805F69D0511C216212785A60E28C013A35
:1086500092B2E284002AA9D1DA6822F08002DA60BC
:10866000DA6842F04002DA6070BDDA68202122F058
:108670004002DA60204684F83910FFF73FFF70BDF2
:10868000BDE87040FFF73EBF9007C7D41107CBD4B9
:10869000A4E7E80596D45607BAD4960702D5002970
:1086A00099D0BBE7160799D505F020000843BBD148
:1086B000E26B002A9AD170BDDA6822F49072DA6017
:1086C0005A69202122F001025A6184F83A105A694D
:1086D000520611D55A69606B22F040025A6158B1B6
:1086E000134B0365FCF70CFA00283FF45FAF606B97
:1086F000BDE87040036D18472046FFF741FF70BD8D
:10870000A90691D4D4E756073FF563AFC5E72046E5
:10871000FFF7F8FE236869E711882069C1F30801B3
:10872000596010B90232226290E7013222628DE76D
:108730003587000808B5806B0023C385C384FFF725
:108740001FFF08BD0A68F0B450F822301B4D8C683A
:10875000CE68CF6B1D404B68234333430E693343D0
:108760004E693343CE6933430E6A33434E6A334313
:108770008E6A3343CE6A33430E6B33434E6B896B41
:1087800033433B430B432B43082C08BF43F04003C8
:10879000B6F5801F40F8223006D012B103681943A5
:1087A00001600020F0BC7047002AFAD0036843F44F
:1087B00080130360036819430160F2E78004C0FF7F
:1087C0000B6900EB820203F1FF3C536810B58C6922
:1087D00003F0404E0B6823434C6843EA04138C6853
:1087E00043EA0423CC68496943EA044343EA0C534F
:1087F000023943EA016343EA0E0353600368DB0274
:108800004FEA0C5C05D5436823F470034CEA03037C
:108810004360002010BD00BFB3F5804F30B406D0D8
:108820006FF0704340F8223030BC0020704750F8A1
:1088300022300A4C8D691C400B682B434D6843EA7B
:1088400005138D68C96843EA052343EA01432343BE
:1088500040F8223030BC0020704700BF0000F0CF4D
:10886000054BD3F888204FF0006142F47002C3F842
:1088700088209960704700BF00ED00E0DFF834D039
:10888000002103E00C4B5B58435004310B480C4B68
:1088900042189A42F6D30B4A02E0002342F8043B06
:1088A000094B9A42F9D3FFF7DBFF08F051F9F7F7CC
:1088B0007BFE704700000420E870010800000020E3
:1088C0003801002038010020C80D0220FEE700001A
:1088D000024B1A6818601046704700BF700C0220E7
:1088E00008B5034610B103F025FA8369184608BDA0
:1088F00008B5034610B103F01DFAC369184608BD58
:10890000034B1B685A7C034B53F82200704700BF8F
:10891000D4000020480C022037B50D4658B151B1A3
:1089200003F012FA02AC294644F8040D00F0D5FA1F
:10893000204603F017FA03B030BD00000A4A0B4985
:10894000002313700A4A0B6013600A4A4B601360DD
:10895000094A13605360094A1360094A1360094ABF
:108960001360094A13607047C4CD0120580C0220DF
:108970009CCD01207C0C0220840C0220900C022053
:10898000440C0220700C0220800C0220F0B5054639
:1089900085B00C461646002D4CD0284603F0D4F97D
:1089A000876A0190BB0701463DD502AD26B1284636
:1089B000324602F0A5FB02E003C885E8030020462A
:1089C000294602F022FC70B317F0010F019B1ED163
:1089D0003EB1B3F90220B6F902309A42A8BF13465D
:1089E00001E0B3F90230B4F902209342B4F9062051
:1089F00006DDBDF80A3019B28A4214DB013B04E0FF
:108A0000BDF80E3019B28A420DDDE3800BE0DF695C
:108A10004FB1384621462A46FFF7B8FF384603F0E3
:108A200089F9076AF4E704A850F80C3D1D6A03F0C1
:108A300099F9B0E705B0F0BD2DE9FF4104460F46B6
:108A400090460025002C37D0204603F07DF9866A39
:108A50000190B207014628D502ACB8F1000F04D04E
:108A60002046424602F04CFB02E003C884E80300C3
:108A70003846214602F0C9FBB8B1F30705D4BDF86A
:108A80000C3001333B8001250FE0019BDE6966B1AC
:108A9000304639462246FFF7CFFF0028304618BF40
:108AA000012503F047F9066AF1E704A850F80C3DE8
:108AB0001C6A03F057F9C5E7284604B0BDE8F08109
:108AC000F0B5044685B00E461746002C31D020463E
:108AD00003F03AF9856A0190AA07014622D502AC53
:108AE00027B120463A4602F00BFB02E003C884E8B7
:108AF00003003046214602F088FB98B1EB0704D40E
:108B0000BDF80830013BB3800CE0019BDD694DB13D
:108B1000284631462246FFF7D3FF284603F00AF9DC
:108B2000056AF4E704A850F80C3D1C6A03F01AF932
:108B3000CBE705B0F0BD0000F7B507460D46284667
:108B400003F002F9836A02AC13F00206014644F80E
:108B5000040D04D1204603F005F9304616E03846EE
:108B600002F000FB019B9E69204656B903F0FAF81B
:108B7000074B1A68954208D058682B1A584258413A
:108B800004E003F0EFF83546D9E7012003B0F0BD6B
:108B9000480C0220F0B5044685B00D46002949D0A6
:108BA00003F0D2F80023036285610190284603F0A8
:108BB000CBF8019BC56902909F6A2DB9C46101A8D9
:108BC00003F0D0F802A833E0284603F0BDF804AE65
:108BD00007F0080746F8040D77B9836A1A070BD522
:108BE000019B1D62029B01A8DC6103F0BBF802A897
:108BF00003F0B8F830461BE002A803F0B3F83046A3
:108C000003F0B0F8284603F095F80390039B1D6A23
:108C10000DB91C620BE0284603F08CF8002FF4D14C
:108C2000836A1B07F1D5039B1C62019B1D6201A88F
:108C300003F098F805B0F0BD03460846B3F90220EA
:108C4000B3F9001002F006BB114B30B51C68626C22
:108C500085B00546BAB11068516802AB03C30D4B2D
:108C6000186800B9A06C03F06FF804AC02A944F8CE
:108C70000C0DFFF7E1FF204603F074F802A8294627
:108C800002F070FA02A801F0E7FC05B030BD00BFA9
:108C9000D4000020440C02201FB50E4B1B6893F833
:108CA00054200AB10C4811E0986C03F04DF8019083
:108CB00003C802AC84E8030001A803F053F8074B93
:108CC000196811B12046FFF737FF2046FFF7BCFFB8
:108CD00004B010BDD4000020A8CD0120440C022017
:108CE00013B5044600B303F02FF8826A019093078E
:108CF00017D5406A40B10D4B1B68A34204D000F069
:108D00005DFC019B00225A622046FFF7F1FD0446FC
:108D10003CB12046FFF7E4FF204603F00BF8046A5D
:108D2000F6E701A803F01EF802B010BD8C0C02207B
:108D3000B0F90020B0F904309A4208DCB0F9022002
:108D4000B0F906309A42CCBF0020012070470020C5
:108D500070470000F0B585B006460D46174602F094
:108D6000E9FF846A0190A30734D52846FFF7E0FFA6
:108D700000282FD040F601032340012B2AD0304693
:108D800002F0E2FF02AC024601902946204602F0C2
:108D9000B7F92046FFF7CCFFC8B1019B9E6A44F2A9
:108DA0002001314003F1080529B128462946224611
:108DB00002F060FA0BE094E803003E4385E803000C
:108DC0009E62054B1A8801321A8002F0E9F901A867
:108DD00002F0C8FF05B0F0BD600C02202022FFF7B2
:108DE000B9BFF0B50F4685B01546064648B302F048
:108DF000ABFF836A04AC9B07024644F80C0D03D416
:108E0000204602F0AFFF1CE002A8394602F078F9D4
:108E10000028F5D0204602F0A5FF304602A92A46D8
:108E2000FFF798FF3046FFF763FD04464CB120463C
:108E300002A92A46FFF7D5FF204602F07BFF046A0D
:108E4000F4E705B0F0BD2DE9FF41804617461D4609
:108E50000C46002930D0084602F076FF866A019061
:108E6000B307024625D502A8414602F049F900B3EE
:108E700040F601033340012B07D1019B02A89969F9
:108E80001A6A2B46FFF7DFFF04E0204602A92A46B4
:108E9000FFF760FF019BDC695CB1BC4209D0204652
:108EA00002A92A46FFF79DFF204602F043FF046A0D
:108EB000F2E701A802F056FF04B0BDE8F0812023DC
:108EC000FFF7C1BF1FB504AB019043F8101D694601
:108ED00003F0E8F905B05DF804FB00230B808288FD
:108EE0004B800388D31A8B80C2884388D31ACB80E7
:108EF0007047F0B50F4687B00546002833D002F022
:108F000023FF866A0190B2072AD503C804ACF30395
:108F100084E8030002D52846FFF7E2FE5FB1386817
:108F2000796802AB03C3019802A9FFF785FE2046CA
:108F300002A902F017F920462946FFF7FDFD78B196
:108F400040F601033340012B06D1019B204699696D
:108F50001A6AFFF7B4FF03E028462146FFF73EFFF9
:108F600001A802F0FFFE07B0F0BD0021FFF7C1BF6E
:108F700010B5044602F0DEFE80690028F9D1054BE9
:108F80001A68944205D05868844214BF4FF0FF30ED
:108F9000012010BD480C022008B5FFF7E9FF0028AA
:108FA00003DBBDE8084002F011B908BD0D4A1368A3
:108FB00070B59D6C0446164608B90B4A14689C644B
:108FC0002046FFF7E9FF01F005FF204602F0B2FE60
:108FD0003368B0F90010B0F90220D9641A65284648
:108FE00070BD00BFD4000020640C02202DE9F74FB3
:108FF0000C9D9B464B4B0746884692461E6865BBB8
:10900000494B1B8863B3494B1B685A7C484B53F848
:1090100022305A1C24D01BB31D46284602F094FE71
:10902000B0F90020B0F90230019017449844BAF129
:10903000000F05D1B0F904A0C2EB0A0A0AF1010A37
:10904000BBF1000F05D1B0F906B0C3EB0B0B0BF170
:10905000010B01A802F086FE02E06B1CDDD10025A9
:109060000F982C3003F088F80446002856D00D9B4A
:109070001E432D4B1A8801321A8002F065FE0E9BAA
:1090800003610DF108092B4B826A49F8080D334042
:109090000780A0F802805744D8441343013F08F1E9
:1090A000FF3883628780A0F80680684602F05AFE87
:1090B000214B186848B102F03DFE0746204602F0F9
:1090C00039FE7B6943617C6100E01C6029462046D3
:1090D000FFF760FDB50602D52046FFF767FFF007F2
:1090E00003D5164B1A6801321A60710602D5204664
:1090F00003F028F9B2070DD5204602F025FE836A59
:10910000009043F002038362684602F02BFE204683
:10911000FFF72BFF20460121FFF7D4FE204603B0C6
:10912000BDE8F08F700C0220400C0220D40000201B
:10913000480C02209F3F3F00640C0220900C02204C
:109140002DE9FF415D4F3B6893F85400002800F083
:10915000B2805B4B5A69012A1C4603DD013A5A6111
:109160000020A8E004F108061B6996E8030001331B
:1091700002AD236185E8030023B92388ADF80830E8
:10918000638811E0A3896289ADF80A2001339BB29C
:10919000B4F90420ADF808301BB29A4206DA2388ED
:1091A000ADF80830E3890133ADF80A30BDF90A2083
:1091B000B4F90630DFF808819A4204DD6369013BA7
:1091C0000020636177E03B68986C02F0BDFDBDF95B
:1091D0000820B8F9003001909A421CD1B8F8063046
:1091E000ADF80E30B8F80430ADF80C30334B1B68D6
:1091F0009A6C5AB1104602F09DFD80460022006A2A
:109200002946FFF7C3FBD8F81820F2E7019B29464F
:10921000D869FFF7BBFBBDF80830ADF80C303B68F0
:109220009A6C6AB1104602F085FD294680460022FC
:10923000006AFFF701FC0028EDD1D8F81820F0E70C
:10924000019B2946D869FFF7F7FB0028E3D1A388E3
:10925000BDF90820ADF80C301BB29A4207DD95E845
:10926000030086E8030001A802F07CFD97E73B6855
:109270009A6C52B1104602F05DFD07460022006A6A
:109280002946FFF71DFCBA69F3E704AF294657F8F2
:109290000C3DD869FFF714FC384602F063FD2369E2
:1092A00044F62062934289DC95E8030086E80300D7
:1092B000FFF7F2FC012004B0BDE8F081D4000020EB
:1092C000A0CD01202DE9F041394F3B6893F854209F
:1092D00086B0064612B9FFF7DFFC64E0354D6A69D7
:1092E0000132012A6A612C465DDC986C02F02CFD8B
:1092F0004FF0FF322A61304A009012782AB100F113
:10930000080302AA93E8030005E0826A12F002084B
:109310000AD003C802AA82E8030002AD66B128465B
:10932000314601F01FFF07E06B696846013B6B6146
:1093300002F018FD404637E03B68204E5A6CC2B13F
:10934000009B10685168019304AB03C3336833B1C9
:1093500001A802F007FD306802F0F6FC01900198C8
:1093600004A9FFF769FC284604A901F0FBFE01A847
:1093700000E0684602F0F6FC316819B12846FFF7B4
:10938000DBFB28B13B682846996CFFF7D5FB18B981
:109390006369013B636107E095E8030084E803002B
:1093A000FFF7CEFE00E0012006B0BDE8F08100BF6F
:1093B000D4000020A0CD01206D0C0220440C02201E
:1093C000024B1B68012283F854207047D400002010
:1093D00010B5044640682368E168172B0FD006DCFF
:1093E0000E2B0ED0142B14D1FFF796FA11E0222B7E
:1093F0000CD0282B0DD1BDE81040FFF7B6BDE060C2
:1094000010BD2146BDE8104002F086BF6FF07043EA
:1094100000E00023E36010BD03680E2B10B5044686
:1094200002D00F2B09D020E0C3685A68012A21D14D
:109430001868BDE8104001F005BF0F4A4368116885
:109440008B4206D05268934214BF4FF0FF33012382
:1094500000E00023094A52F823006FF0704398425D
:1094600003D001F0AFFE02F013F92046BDE8104032
:10947000FFF7AEBF10BD00BF480C0220740C0220E5
:1094800030B52B4B187885B01D4600284DD1294B9F
:109490001860294B1860294B1B685864284B1880AA
:1094A000284B04461880204601F0CEFFC0B14FF093
:1094B000FF3202238DE80C00002043F6FF72224B9E
:1094C0000293039013460146FFF790FD1F4B43F8AC
:1094D00024001F4B6FF0704243F82420FFF745FD36
:1094E0000134022CDFD11B4802F024FF1A4802F09D
:1094F00021FF1A4802F01EFF194802F01BFF19480D
:1095000002F018FF184802F015FF104B1868FFF71B
:109510004DFDFFF755FF01232B701448144B0360DA
:1095200005B0BDE8304002F0C3B805B030BD00BFA3
:10953000C4CD0120640C0220B8CD0120D40000204D
:10954000600C0220400C022019940008480C0220F4
:10955000740C0220B40D0220A40D0220940D0220F0
:10956000BC0D0220AC0D02209C0D0220BCCD0120C0
:109570003D89000813B550B102F0E6FB044602A88D
:1095800040F8044D02F0EEFB04F11800FFE702B0D2
:1095900010BD37B5054670B102F0D6FB036802ACCA
:1095A0001B6944F8040D9B68984701F078F905465B
:1095B000204602F0D7FB284603B030BD37B504463D
:1095C000D0B10E4B1B681B6E834201D101F014FE1B
:1095D000204602F0B9FB0190406908B103F0C8FAD7
:1095E00002AD55F8043D186801F03EFF284602F030
:1095F000B9FB204602F0D6FB03B030BDD4000020FA
:10960000F8B504460E46D0F88C302A211546984706
:10961000E16AD4F8903031442046C1F30F219847D5
:10962000E16AD4F89030B7B239442046C9B29847BD
:10963000E16AD4F8903031442046C1F30F219847B5
:10964000E16AD4F8903039442046C9B29847D4F83A
:109650008C3020462B219847216BD4F89030294438
:109660002046C1F30F219847216BD4F89030AEB259
:1096700031442046C9B29847216BD4F89030294430
:109680002046C1F30F219847216BD4F89030314424
:109690002046C9B29847D4F88C3020462C219847F0
:1096A000F8BD2DE9F041044688461F462A21D0F82E
:1096B0008C30069D16469847E16AD4F890304144B4
:1096C0002046C1F30F219847E16AD4F89030414415
:1096D0002046C9B29847E16AD4F890303944204610
:1096E000C1F30F219847E16AD4F8903039442046FD
:1096F000C9B29847D4F88C3020462B219847216B6B
:10970000D4F8903031442046C1F30F219847216BA3
:10971000D4F8903031442046C9B29847216BD4F830
:10972000903029442046C1F30F219847216BD4F88B
:10973000903029442046C9B29847D4F88C3020464E
:109740002C219847BDE8F08113B50D4A04465168B5
:1097500010686B4603C3D4F88C30204636219847F6
:10976000636BA18C02AA134421F0E00113F8083CBA
:1097700019432046D4F8903089B2984702B010BD02
:10978000E054010813B50446D0F80C312E20984758
:10979000216AD4F82831684603319847226A00AB21
:1097A00013441DF8022059789878D2088908D2020B
:1097B00042EA411242EAD00002B010BD1FB5044691
:1097C000D0F82C312E209847216AD4F848316846C9
:1097D00002319847236A00A901EB43023DF81300C8
:1097E000528802F47C41C2F3C40242EA511200F0F2
:1097F000F80042EA002004B010BD38B504460D461A
:10980000D0F80C31080A9847D4F80C31E8B29847E0
:1098100038BD08B5D0F82C310846984708BD08B5C2
:10982000D0F81031C8B2984708BD08B5D0F830312B
:109830000846984708BD0000082902D0102905D025
:109840007047064BC0F88C30054B03E0054BC0F861
:109850008C30054BC0F89030704700BFFB97000874
:109860001F980008139800082B980008F0B585B0E1
:1098700084680A9F0097BD1A581A013500FB0555E8
:10988000D4F8A8700B9E2046B847D4F80C312E208F
:109890009847D4F82831216A02A89847D4F828318B
:1098A00002A8032198479DF808309DF80920DB089D
:1098B0009208DB0243EA42139DF80A20013D43EA85
:1098C000D20326F8023BE9D105B0F0BDF0B587B070
:1098D00084680C9F0097BD1A581A013500FB055586
:1098E000D4F8A8700D9E2046B847D4F82C312E200D
:1098F0009847D4F84831216A02A89847D4F84831EB
:1099000002A802219847BDF80A3003F47C42C3F351
:10991000C40343EA5213BDF8082002F0F80243EAF8
:109920000223013D26F8023BE8D107B0F0BD00005C
:1099300010B5044600F0A6FDA368124AC3F8AC2097
:10994000114AC3F8A820114AC3F8B020104AC3F83E
:10995000B8200022C3F8BC20C3F8CC200D4A0E4921
:109960001268C3F8C420DA8C0968C3F8B41022F076
:1099700003020A49DA840A4AC3F8C810C3F89420DB
:1099800010BD00BF01960008A39600084997000883
:1099900085970008CC000020C80000206D980008C2
:1099A0003998000808B5D0F8B430984708BD08B514
:1099B000D0F8303188B2984708BD00002DE9F04F4B
:1099C0003D4F846882463868007C10F0010F85B0F6
:1099D0000E4615469846C1EB030945D04FEA490BA0
:1099E0000E98854265DCD4F8C4C0E76EBCF1000F68
:1099F00001D1B44607E08DE8A000504631462A4622
:109A00004346E04711E0C4450EDCD4F8EC30CDF815
:109A10000CC0614650462A469847DDF80CC027F82E
:109A2000020B0CF1010CEEE7E76EBB1E09F1010C15
:109A30005F44BB4205D0A26A59884A4023F8022FEE
:109A4000F7E700952A46D4F8A870CDF80CC0204658
:109A500031464346B847DDF80CC0D4F83831E06EE3
:109A6000614698470135BBE70E980090851AD4F8F7
:109A7000A8602046B0473B68A76EDB6B09F101097F
:109A8000D3F8008005FB0995012395B1FA2D34BF69
:109A90002E46FA262BB138461FFA88F1324601F0DD
:109AA0005BFAD4F83831384631469847AD1B00236D
:109AB000EBE705B0BDE8F08FD40000202DE9F04FB2
:109AC0008DB08568179F05937B1E012B0990089127
:109AD0000A920B9503D9042F01D0082F06D18F4B82
:109AE0001B681B7C03F00303022B10D00A9A169FFD
:109AF0001A9D0899059B3A442944013A0B9D00920E
:109B00000B44D5F8A8400A9A2846013BA047DDF847
:109B100028B00A9F169DC7EB0B03AB4280F251821F
:109B2000179F7B1E0F2B00F24582DFE813F0100019
:109B3000B70043024001430243024302D7014302FC
:109B40004302430243024302430243023D02734B7A
:109B5000099D1B68AC681B9D1B7C2F686D68079571
:109B6000DDF820A01A9D03F00303022BAA441BD0AA
:109B7000032B6ED0012B6CD0059EDDF8648098F825
:109B80000010D4F8303180222A41114216BF0799C3
:109B9000B8B288B201359847082D04BF08F1010812
:109BA0000025013EEBD105E2199D0695D4F86C9095
:109BB000DDF86880CDF80CA0002556462B46069FA0
:109BC0004FF0800C3A784CFA08FC12EA0C0C0BD0DF
:109BD00013B9D4F86C900396079FA9F8007001356B
:109BE00009F10209012317E0012B14D1CDF800B0CF
:109BF000CDF810C020460399D4F8A8705A46731EB9
:109C0000B847D4F83831E06E29469847DDF810C0DF
:109C10006546634600E0634608F10108B8F1080FA5
:109C200006F1010604D1069F013706974FF00008A0
:109C3000059A5244B242C2D1059F7B1E5344002D67
:109C400000F0B881CDF800B0D4F8A86003992046A0
:109C50003DE1DDF814801A9E199DDDF814902A78F4
:109C600080233341D1441A42C8EB09090DD0D4F8FE
:109C7000EC30099849465A469847A36AD4F8F070E0
:109C80004340494609985A46B8470136082E04BF52
:109C900001350026B8F10108DFD18BE1099D1B9F3A
:109CA000AC68002F00F086811C4B199D1B6895F84D
:109CB00000A01B7C13F0030311D0022B40F07A812B
:109CC0001A9DDDF82090E76E0397A944A846199DD8
:109CD00007950025CDF818904E462B4640E01A9D7A
:109CE000059E199FC5F103035B00C3F10602C02165
:109CF00041FA02F202EA0A02DA401B99D4F8303142
:109D000031F8220001359847042D03D197F801A0BE
:109D100000250137013EE5D14CE100BFD400002011
:109D200013B9E76E039706961B9F57F82C30039FD5
:109D30003B80023701350397012308F10108B8F190
:109D4000040F06F1010606D1079F97F801A001371D
:109D500007974FF00008059A4A44B24200F0AC80E1
:109D6000C8F103025200C2F106014FF0C00C4CFAD8
:109D700001FC0CEA0A0C3CFA02FCD1D1012B14D1F3
:109D8000CDF800B0CDF810C020460699D4F8A870E0
:109D90005A46731EB847D4F83831E06E29469847C2
:109DA000DDF810C065466346C7E76346C5E7099D11
:109DB0001B9FAC68002F00F0FD80834B199D1B6832
:109DC00095F800A01B7C13F0030311D0022B40F088
:109DD000F1801A9DDDF82090E76E0397A944A8460C
:109DE000199D07950025CDF818904E462B463CE06E
:109DF0001A9D059E199FC5F101039B00C3F1040242
:109E0000F02141FA02F202EA0A02DA401B99D4F880
:109E1000303131F8220001359847022D03D197F8EF
:109E200001A000250137013EE5D1C3E013B9E76E7B
:109E3000039706961B9F57F82C30039F3B800237F1
:109E400001350397012308F10108B8F1020F06F16B
:109E5000010606D1079F97F801A0013707974FF039
:109E60000008059A4A44B24226D0C8F10102920085
:109E7000C2F104014FF0F00C4CFA01FC0CEA0A0CA0
:109E80003CFA02FCD2D1012B14D1CDF800B0CDF8B0
:109E900010C020460699D4F8A8705A46731EB847D9
:109EA000D4F83831E06E29469847DDF810C0654691
:109EB0006346C8E76346C6E7059F7B1E4B44002DFB
:109EC00078D0CDF800B0D4F8A860069920465A465C
:109ED000B047D4F83831E06E29466AE0099D1B9FEF
:109EE000AC68002F66D0384B1B681B7C13F0030353
:109EF00009D0022B5ED1DDF82090D4F86C800026CA
:109F00004F46334622E0199D199B059F3B445B1B3E
:109F1000002B4FDD15F8012B1B9FD4F8303137F89B
:109F200022009847F0E713B9D4F86C80B9461B9D1E
:109F300055F82A30A8F80030013608F1020801234C
:109F4000089A059D01372A44BA421CD0199D0898E9
:109F50002A1A12F807A0BAF1000FE4D1012B10D190
:109F6000CDF800B0204649465A467B1ED4F8A8508A
:109F7000A847D4F83831E06E3146984756465346E4
:109F8000DEE75346DCE7089F6B1E3B4496B1CDF8F5
:109F900000B020464946D4F8A8505A46A847D4F8FD
:109FA0003831E06E314604E00B9D1998D5F8383110
:109FB00005999847199F189D2F4419970BF1010B8C
:109FC000A7E50DB0BDE8F08FD400002010B5044621
:109FD00000F058FAA468104BC4F8E4300F4BC4F8F2
:109FE000E8300F4BC4F8EC300E4BC4F8F0300E4B99
:109FF000C4F8A0300D4BC4F8A430D4F8C430C4F871
:10A00000FC302046D4F89430102198471023A363E5
:10A01000074B636410BD00BFBD9A0008BD990008DE
:10A02000D3A3000843A30008A5990008AF9900082E
:10A03000C8560108084670470068401A0138704742
:10A04000084670470068401A01387047104670474C
:10A050004068801A01387047104670474068801A7F
:10A060000138704710467047104670474068801AA4
:10A07000013870474068801A0138704708467047B9
:10A08000084670470068401A013870470068401A57
:10A090000138704710B58468D4F8F040A04710BD6F
:10A0A00008B58368D3F8EC30984708BDF7B5044687
:10A0B0000F4616468568FFF7F3FF0190DDF804E0D0
:10A0C000AB6A2046394632468EEA0303FFF7E2FFC9
:10A0D00003B0F0BD13B584680092D4F8E840A047FF
:10A0E00002B010BD13B584680093D4F8E8400B4665
:10A0F000A04702B010BD37B5069C85680094D5F81E
:10A10000E840A04703B030BD30B587B085680A9CF1
:10A1100000940B9C01940C9C02940D9C03940E9C47
:10A1200004940F9C0594D5F8E440A04707B030BDD7
:10A130007047000073B5079E84680C4D76B128689F
:10A1400088B906980090D4F8A8602046B047D4F8A3
:10A15000A8302B60064BC4F8A83004E02B6813B17C
:10A16000C4F8A8302E6002B070BD00BFC8CD012079
:10A1700031A1000808B5026CD0F8D4309069984736
:10A1800008BD08B5026CD0F8D8309069984708BD72
:10A190002DE9F7430A9D8468009517462046D4F8B8
:10A1A000A86099468846ED1BB047216CD4F8DC3096
:10A1B00088690B99C8EB09086A1C08FB02229847BA
:10A1C00003B0BDE8F0832DE9F7430A9D846800954C
:10A1D00017462046D4F8A86099468846ED1BB0473C
:10A1E000216CD4F8E03088690B99C8EB09086A1C27
:10A1F00008FB0222984703B0BDE8F0830139172914
:10A2000024D8DFE801F01023232323232323230C66
:10A21000250E1523232323232323231F1A210D482F
:10A2200070470D48704703689B68D3F8FC0070477F
:10A2300003689B68D3F8F400704703689B68D3F801
:10A24000F800704705487047054870470020704780
:10A2500004487047B3A5000855A50008B9A4000834
:10A2600035A100089FA50008013980680D2923D871
:10A27000DFE801F0090B0D0F22222211072525131B
:10A28000181D00207047006870474068704780685C
:10A290007047C0687047806B704788B1406B00F0B2
:10A2A0000100704760B1406BC0F34000704738B1A7
:10A2B000406BC0F3800070474FF0FF3070470120C3
:10A2C0007047836801290CBF586C00207047836871
:10A2D00000220A804A801A685B68013A013B8A8042
:10A2E000CB807047F0B5104D2E4607460FCE91B08B
:10A2F0006C460FC496E80F00203584E80F000FCDA0
:10A3000008AC0FC495E80F0084E80F007B6B10AA1F
:10A3100002EB830353F8402CC7F8002153F8203C8C
:10A32000C7F8043111B0F0BDE854010807B58069E1
:10A330008DE8060003216A46F5F7B6FF03B05DF825
:10A3400004FB2DE9F74384689846E38C9B07894614
:10A35000174632D5D4F8003120469847D4F8045136
:10A3600006463A4620464946A8472369A2699E42C6
:10A37000ACBF002301239642D4BF1A4643F001022A
:10A3800063699842ACBF134642F00103054613B916
:10A39000E36998420ADD62682368013A009200216D
:10A3A000D4F8A87020460A46013BB847D4F8AC70F0
:10A3B000204631462A46B84703E0D4F8AC50204640
:10A3C000A847D4F8A43020464146984703B0BDE8DA
:10A3D000F083F7B58468E38C9B070F46164645D596
:10A3E000D4F8003120469847D4F804313246054667
:10A3F000394620469847D4F8983006461BB1204687
:10A400000121002298472369A2699D42ACBF002325
:10A4100001239542D4BF1A4643F0010263699E426C
:10A42000ACBF134642F0010313B9E3699E420ADD53
:10A4300062682368013A00920021D4F8A87020468F
:10A440000A46013BB8472946D4F8AC30204632468C
:10A450009847D4F8A03020469847D4F8983005465D
:10A460006BB1204600210122984708E0D4F8AC30B7
:10A4700020469847D4F8A0302046984705462846FD
:10A4800003B0F0BD38B58568044695B94FF4BA708D
:10A4900001F0A6FD4FF4BA72A060294600F08AFDD3
:10A4A000A3680222DA8401221A62024A1C64C3F8F9
:10A4B000082138BDE5A2000870B506460D461446D1
:10A4C000FFF7E0FFB368002B3BD0262D02D0272DED
:10A4D00016D070BD9A6B102A02D0122A08D070BD17
:10A4E000184AC3F8D440C3F8B820C3F8B42070BDEC
:10A4F000154AC3F8D840C3F8BC20C3F8C02070BDCB
:10A500009A6B102A02D0122A0ED070BD3CB10F4AAD
:10A51000C3F8DC40C3F8C820C3F8C42070BDC3F83A
:10A52000C840C3F8C44070BD3CB1094AC3F8E0401C
:10A53000C3F8CC20C3F8D02070BDC3F8CC40C3F81A
:10A54000D04070BD75A1000883A1000891A100084A
:10A55000C7A1000838B50546FFF794FFAC684FF473
:10A56000FA7001F03DFDA36BA0660733D810236895
:10A57000584301F035FD01210022E066A869F5F796
:10A5800093FED4F808310546204698472046D4F873
:10A59000B0309847002DD4BF0020012038BD70B5E1
:10A5A00004460D461646FFF76DFFA36883E860007A
:10A5B00070BD70B504460D461646FFF763FFA368ED
:10A5C0009D60DE6070BD38B505460C46FFF75AFF4A
:10A5D000AB682268DA6262681A63A2685A6352073B
:10A5E00007D593E806001A605960DA689968D9605F
:10A5F0009A60A2899A84226912B122EAE2721A62EE
:10A6000038BD2DE9F04104461F4616468846FFF73F
:10A6100039FFA5684146682205F5867006F0BEFA46
:10A620002046B0472046B84723699B689847A862F0
:10A63000BDE8F08110B5074C2368186B00F024FCCE
:10A6400000F042FC2368586B00F01EFCBDE810408F
:10A6500000F056BCD400002037B5094C23685A7C62
:10A66000084B054653F82200C2686946126B9047B2
:10A67000206829466A46083000F042FD03B030BD2C
:10A68000D4000020C40C022037B50D46144600F05B
:10A69000DBFE019008B901200CE0C3680A215B6A67
:10A6A00001A8984703460028F5D00198294622467C
:10A6B0009847002003B030BD37B50D46144600F072
:10A6C000C3FE019008B901200CE0C3680B215B6A4E
:10A6D00001A8984703460028F5D00198294622464C
:10A6E0009847002003B030BD37B50D46144600F042
:10A6F000ABFE019008B901200CE0C36810215B6A31
:10A7000001A8984703460028F5D00198294622461B
:10A710009847002003B030BD012810B50C4608DC76
:10A7200000F092FE20B1C36821469B6A984710BD95
:10A7300010BD002010BD38B5044621460120FFF7AA
:10A74000EBFF214605460020FFF7E6FFA842B8BF11
:10A75000284620EAE07038BD0821FFF7DDBF092157
:10A76000FFF7DABF0E21FFF7D7BF0000024B1B68CF
:10A77000587CFFF7F4BF00BFD4000020024B1B68D9
:10A78000587CFFF7EFBF00BFD400002008B5044B92
:10A7900053F82000C36808219B6A984708BD00BF92
:10A7A000C40C022008B500F04FFE20B1C36802219E
:10A7B000DB6A984708BD08BD024B1B68587CFFF751
:10A7C000F1BF00BFD4000020024B53F820301B69BA
:10A7D00058687047C40C0220024B53F820301B69A4
:10A7E00018687047C40C02200120FFF7A4BF0220A4
:10A7F000FFF7A1BF024B1860024B1960704700BF02
:10A80000D0CD0120CCCD0120014B1868704700BF8E
:10A81000D0CD0120014B1868704700BFCCCD01207E
:10A8200000283BD030F0010329D030F0030328D0BA
:10A8300030F0070327D030F00F0326D030F01F038D
:10A8400025D030F0FF0324D020F4FF7323F0010360
:10A850000BB320F47F6323F00F03E3B120F4FF4335
:10A8600023F07F03BBB1030C1B04A3B1830C9B0437
:10A870009BB110F07F4F0CBF1820202070470120A3
:10A88000704702207047032070470420704705205E
:10A89000704708207047102070471220704708B595
:10A8A000FFF7BEFF01280FD0831E062B09D9A0F1A8
:10A8B0000903072B07D91138102834BF20200020A6
:10A8C00008BD082008BD102008BD000070B5084B69
:10A8D0001B681A7C80EA0201490705D59C6BD96B7D
:10A8E00026680D6825600E601874104670BD00BFA4
:10A8F000D400002008B5024B1B689B68984708BD30
:10A90000D000002038B5144B1B680A46B3F90A1072
:10A910008A4204461EDBB3F90E108A421ADCB3F9F0
:10A920000810884216DBB3F90C10884212DC197C3F
:10A93000587C11F0010F094951F8200004D0C36878
:10A940002146DB69984738BDC168DB6B8D691B68A0
:10A950002146A84738BD00BFD4000020C40C022007
:10A9600038B5104B1C68B4F90A3099420D4617DB14
:10A97000B4F90E30994213DCB4F90810B4F90C3074
:10A980008842A8BF01469A42B8BF13468B4207DBF4
:10A99000607C054A52F82000C26894682A46A047A5
:10A9A00038BD00BFD4000020C40C022073B50E4691
:10A9B00012490C68B4F90810B4F90C508842A8BFC9
:10A9C0000146AA42B8BF15468D4214DBB4F90A20ED
:10A9D000B4F90E009642A8BF32468342A8BF034690
:10A9E000934208DB647C064850F82400C468009356
:10A9F00024692B46A04702B070BD00BFD4000020E0
:10AA0000C40C02202DE9F04FDFF8ACC18FB0DCF8A8
:10AA100000C009900E4615469B461C9CDDF87880C8
:10AA2000BCF1000F0DD0189D199E009501961A9F3C
:10AA30001B9D1D9E0297039504940596DCF800402B
:10AA400053E0189F199847EA0003012B4FD1584B48
:10AA50001868B0F90A20511A002908DDC1EB0B0370
:10AA6000002B40F3A2801B9F07FB014401E05B46E3
:10AA700032465E44B0F90E10013E761A002E03DD18
:10AA80009B1B002B40F391800999B0F90C6029447D
:10AA90000139891B099E0029C8BFC1EB0505C8EB18
:10AAA0000601B0F90860B1420CDAC1EB060C08EB04
:10AAB0000C078E1B2CF0070C354404EBE7046144B3
:10AAC00007F00708002D70DD467C3A481A9F50F8C1
:10AAD0002600C668019703941B9F1D9C0093029754
:10AAE000CDF81080059474682B46A0475DE01A9F4E
:10AAF000C7F108070C976746DC4556DA2C4B1998C6
:10AB00001B683044B3F90A200A90411E91420B9110
:10AB100045DBB3F90E309E4241DC4FF00008DDF812
:10AB200024900894C246AA4539DAB8F1000F05D13D
:10AB3000089A1778013208924FF008080C981A9971
:10AB40001B4A47FA00F3C1EB08088F4013F0FF01DE
:10AB5000FFB203D11068007C80071BD41268D26B4F
:10AB600010680D901D9810B150F8213000E0DBB254
:10AB7000189913604A1E4A440B9BCDF81CC04846E6
:10AB80003146FFF713FF0A4B0D9A1B68DDF81CC016
:10AB9000DB6B1A60189B0AF1010A9944C3E71B9EFC
:10ABA0000CF1010C34440A9EA6E70FB0BDE8F08F0B
:10ABB000D4000020C40C0220980C02202DE9F04F94
:10ABC000DFF80CC291B0DCF8009007920546884689
:10ABD0009B461C9E1E9CB9F1000F0CD01A9D1B9F1A
:10ABE000009501971D9D1F9F02960395049405975C
:10ABF000D9F8004081E01A9F1B9847EA0003012B17
:10AC00007DD1714B1868B0F90A20531A002B08DD6A
:10AC1000C3EB0B01002940F3D4801D9F07FB0344C5
:10AC200001E059464246D844B0F90E3008F1FF38E9
:10AC3000C3EB0808B8F1000F04DDC8EB01010029DF
:10AC400040F3BF80079BB0F90CC02B44013BCCEB19
:10AC50000303002B02DD079FFF1A0797B0F908C016
:10AC6000654533DA079FC5EB0C03FF1A082E0797DB
:10AC700027D00DDC022E14D0042E1AD0012E26D19E
:10AC800023F0070C04EBE304654403F007031EE024
:10AC9000182E18D0202E16D0102E18D104EB4304F5
:10ACA00013E023F0030C04EBA304654403F0030357
:10ACB0000DE023F0010C04EB6304654403F0010391
:10ACC00005E01C4401E004EB830465460023079F74
:10ACD000002F76DD90F811E03C481D9F50F82E00C3
:10ACE000D0F80CE003948DE842001F9C0493029777
:10ACF0000594DEF80440079B2946A04761E0C6F1B1
:10AD000008070E97CDF828900A9F5F4559DA2E4B19
:10AD10001B9F1B684744B3F90A200C97013F9742D9
:10AD20000D9746DBB3F90E30984542DC4FF0000A30
:10AD30000B94AC465746079887423ADABAF1000FAF
:10AD400006D10B9890F8009001300B904FF0080A54
:10AD50000E991D4A49FA01F313F0FF0109FA06F9A9
:10AD60005FFA89F9C6EB0A0A03D11068007C8007F4
:10AD70001BD41268D26B10680F901F9810B150F856
:10AD8000213000E0DBB21A9913604A1E624460462B
:10AD90000D9BCDF820C04146FFF708FE0A4B0F9AE5
:10ADA0001B68DDF820C0DB6B1A601A9B01379C44DE
:10ADB000C1E70A9FDDF8308001370A971D9F3C44A8
:10ADC000A2E711B0BDE8F08FD4000020C40C02202F
:10ADD000980C022008B5054B1968054B4A7C53F8BE
:10ADE0002200C36808311B6B984708BDD4000020BF
:10ADF000C40C022037B5FFF7EDFF02F0FFFB04465D
:10AE000000283DD10546284600F01EFB019048B1C0
:10AE1000C3680C215B6A01A89847034670B3019888
:10AE2000984704430135022DEDD14CBB02F002FCE2
:10AE30000124204600F008FB0190D0B1204600F02C
:10AE4000C5F90420FFF756FD43F6FF7200200146C6
:10AE50001346FFF7ABFD0020FFF74CFD02A80E21C3
:10AE600050F8043DDB685B6A9847034608B10198D7
:10AE7000984714F1FF34DCD2002002E0012000E00A
:10AE8000204603B030BD000008B5054B1B685A7C56
:10AE9000044B53F822301B691B68984708BD00BF5C
:10AEA000D4000020C40C022008B5054B1B685A7C56
:10AEB000044B53F822301B695B68984708BD00BFFC
:10AEC000D4000020C40C0220044B1B681A7C5207DB
:10AED0004CBF9B6BDB6B1860704700BFD400002039
:10AEE00008B5064B1B68196B814206D01863FFF743
:10AEF000CBFFBDE80840FFF7E7BF08BDD400002046
:10AF0000044B1B681A7C52074CBFDB6B9B6B1860B1
:10AF1000704700BFD400002008B5064B1B68596B72
:10AF2000814206D05863FFF7AFFFBDE80840FFF746
:10AF3000E7BF08BDD400002008B5024B1B685B6862
:10AF4000984708BDD000002008B5024B1B681B685D
:10AF5000984708BDD000002070B5840702D5018055
:10AF6000013A023055082B4605B3032D01EB01448D
:10AF700002DC06461D4612E003462E46043E032E22
:10AF80001C605C609C60DC6003F11003F6DC043D37
:10AF9000AB085E1C00EB0610A5EB8303E9E71DB1CF
:10AFA00046F8044B013DFAE700EB8300D30748BFA6
:10AFB000018070BD70B52AB1830703D000F8011B72
:10AFC000013AF8E7930801D1024417E04FF0013449
:10AFD00002F003024C43032B054606DD0460446087
:10AFE0008460C460043B1030F5E71E461BB145F891
:10AFF000044B013BFAE700EB8600E5E7904202D004
:10B0000000F8011BFAE770BD0128F7B504460D46AC
:10B0100065DC344B1B6803B19847012D04D0022D29
:10B0200021D0002D5BD135E02F4E56F82470B7B9F2
:10B03000204600F009FA0190002850D0C3680D2185
:10B040005B6A01A898470346002848D00198294622
:10B05000984756F82430013346F8243018E0013779
:10B0600046F824703BE0204600F0EEF901900028FD
:10B0700035D0C3680D215B6A01A8984704460028B3
:10B080002DD01A4B1B6803B1984701980221A047A5
:10B09000002025E0144D55F82430012B01D001206B
:10B0A00015E0204600F0D0F901900028F7D0C368E1
:10B0B0000D215B6A01A8984706460028EFD00B4B8C
:10B0C0001B6803B1984701980021B047002055F84C
:10B0D0002430002B18BF013B45F8243000E001204C
:10B0E00003B0F0BDE0CD0120D8CD0120D4CD0120AA
:10B0F000024B1B680146587CFFF786BFD400002036
:10B1000070B5B2F90030B1F90040B1F90250B1F9AF
:10B110000460B1F906109C42B8BF1C46B2F9023077
:10B120009D42A8BF2B46B2F90450B2F90620AE42A8
:10B13000B8BF3546A4B2ADB29142B8BF0A4604804A
:10B14000858024B22DB29BB292B2A5424380C280C8
:10B1500006DB10B21BB29842B4BF0020012070BDC4
:10B16000002070BD0B8810B5B0F900401AB29442AF
:10B17000B8BF03804B88B0F902401AB29442B8BFFE
:10B1800043808B88B0F904401AB29442C8BF8380D0
:10B19000CB88B0F906101AB29142C8BFC38010BD67
:10B1A00008B5024B1B6803B1984708BDE4CD0120E8
:10B1B000034B1B68D96900B1D8610846704700BFCE
:10B1C000D4000020FFF7B8BEFFF7BEBE70B5084D33
:10B1D0002B68012804465E7C08D800F035F928B1B8
:10B1E0002B685C7400F008F8024B1C60304670BDA0
:10B1F000D4000020680C022008B502F0D5F9FFF752
:10B2000019FABDE80840FEF7DBB8B0F90220B1F941
:10B2100006309A4214DCB1F90220B0F906309A42A5
:10B220000EDCB0F90020B1F904309A4208DCB0F924
:10B230000430B1F900209A42CCBF002001207047B1
:10B2400000207047024B1A6802B91860FFF7A8BFC8
:10B25000E8CD012068B1038889B20B44038083885C
:10B2600019444388818092B213444380C3881A44AE
:10B27000C280704710B538B309B30AB3B1F90040C2
:10B28000B2F900309C42B8BF23460380B1F90240B6
:10B29000B2F902309C42B8BF23464380B1F9044062
:10B2A000B2F90430B1F906109C42A8BF234683804E
:10B2B000B2F906309942A8BF0B46C38010BD1146B3
:10B2C0000B6803604B68436010BD0000054B1B68B2
:10B2D000002B18BF0020044B0129B8BF01211954CD
:10B2E000704700BFECCD0120940C0220024B1B687C
:10B2F0005884998400207047D4000020F8B50B4B87
:10B300001B680546B3F92C0040F002000F461646B4
:10B3100002F0B4FA394604463246284600F008F8EE
:10B320002046BDE8F84002F0A9BA00BFD4000020D2
:10B33000024B1B6859849A8400F002B8D4000020A4
:10B340002DE9F74F0446002879D03E4D00F0E0FB90
:10B350002B688046B3F8229000F0C2FB2B689A8CD1
:10B3600087B2D21B9A842378002B5DD047F6FF71F9
:10B37000204600F003FB06463146204600F02CFB39
:10B380002B689A8D02F00302012A05D0022A14BF0D
:10B39000002290FBF2F200E00246598C8A1A92B227
:10B3A00091B259841FFA80FA9B8CADF800100AF113
:10B3B000FF310A44ADF802301FFA88FB013B5B44C1
:10B3C000ADF80420204631466A46ADF8063000F05C
:10B3D00033FB2B68BDF802209A842046314602F0E8
:10B3E0003BFA235C0A2B04EB000201D00D2B12D197
:10B3F0002B68998D01F00301013901298ABF198C4D
:10B40000A3F82290598411780A290BD1998C8B4486
:10B41000A3F824B006E00B4BBDF800001B68824483
:10B42000A3F822A0137843B92B689A8C17449A8DFD
:10B430009F8422F003029A8501E0541C93E703B035
:10B44000BDE8F08FD4000020012809DC054B53F83B
:10B45000200020B1C3681B681BB10068F9E7704782
:10B4600000207047C40C022000F05ABC012BF8B534
:10B4700006460D4617461C4601DD0020F8BD1C207F
:10B4800000F0AEFD0028F8D00DB1056109E0094BD0
:10B4900053F8241029B10B680BB11946FBE70B696F
:10B4A00003610023836084618782C6600360436018
:10B4B000F8BD00BFC40C0220094B826953F822106A
:10B4C000814204BF016843F8221043680BB102684F
:10B4D0001A60026802B15360002303604360704742
:10B4E000C40C022070B538B38269012A24DC1949E2
:10B4F00051F822300D4613B941F822001AE059687C
:10B5000009B10B46FBE7C1680E68D9680C68B44204
:10B5100003DD1B68002BF8D10EE002D1818A0129DE
:10B5200011D0596899B1086041605860984208BFCD
:10B5300000230360002070BD012070BDCB681B6834
:10B54000A3420B46EDDB19680029F7D1E9E745F87E
:10B550002200EAE7C40C022038B51D46FFF786FF3B
:10B56000044648B1FFF7BEFFE3681B6823B9034BED
:10B5700016351B6843F82540204638BDD40000200E
:10B5800010B5074B07480024214670221C60FFF7C6
:10B5900011FD214604480822BDE81040FFF70ABD0E
:10B5A0006CCE0120F4CD0120C40C022038B5194D19
:10B5B0002B681A1DDA6303F108029B631B64426166
:10B5C0005A7C154B044653F82200C36804F1080165
:10B5D0001B6B9847114B6366114B1B68E3612B682B
:10B5E0000833636101232376FDF78AF9032384F886
:10B5F00068306FF0704323636363A0640020FFF73B
:10B600009BFC6FF07F40FFF79FFC064B064A1A60D9
:10B6100038BD00BFD4000020C40C022068560108C9
:10B62000D8000020BC0C0220207001082DE9F3474F
:10B63000074604209A460E469146FFF75BF9134BE6
:10B640001C68E56C246D2F44264480464D445444C8
:10B650006846ADF80070ADF80450ADF80260ADF882
:10B660000640FDF72FFE28B94046FFF743F902B028
:10B67000BDE8F087384631462A462346FFF796F95B
:10B68000FDF75EFD0028F5D1EEE700BFD4000020F5
:10B6900010B500200146FFF729FE044843F6FF726B
:10B6A00001461346BDE81040FFF7C0BF01C0FFFFD1
:10B6B00080B483B000AF7860054B1A687B685A602D
:10B6C000034B7A681A600C37BD465DF8047B7047FF
:10B6D000F0CD012008B5084B1A6862B901221A6042
:10B6E000F4F770FDF4F798FD0448054B0360BDE8DE
:10B6F0000840FFF7DDBF08BD6CCE012064CE0120FD
:10B7000081B5000890B583B000AF204B1F4A126886
:10B7100022F001021A601E4B01221A601D4B1E4AC4
:10B720001A601C4B1A681D4B9A4200D0FEE7FFF7C7
:10B73000D1FF1B4B2E221A7002F050FA1948FFF766
:10B7400035FFFFF757FB7860FFF75EF80346002BE5
:10B7500004D0FFF75FF80346002B09D1FFF744F848
:10B760000446FFF744F8034620461946FFF742F81F
:10B770000020002102F08CF8FDF782FE0A4B012226
:10B780001A707B6818460C37BD4690BD002000E05B
:10B790000830024000300240C2A507F4CDB5E8B53C
:10B7A000960C0220F4CD0120B40C022038B103889D
:10B7B0008B4202D843888B4201D28068F6E77047FB
:10B7C0002DE9F04F384C2368B3F92A90DB69054620
:10B7D00089B0D8692946FFF7E9FF002861D0B0F8A1
:10B7E00000804768C8EB050807EBC806484696F88E
:10B7F00002B0FFF77FF8256817F83820D5F81CE06D
:10B80000B5F924109EF81AC09EF8183006938246A7
:10B81000B5F92200CDF800C09EF81BE0CDF804E099
:10B820004FF0010ECDF80CB0CDF808E0736804932A
:10B83000AD6B069B0595FFF7C1F92368DA6992F8AD
:10B8400019B0117E8B4520D9B9F1020FD57E1CD0DD
:10B85000079102F03EF8814602F034F8FFF7B4FC9D
:10B86000246817F83870E269B4F92430B4F922007A
:10B87000D27E079907FB020201FB05310BFB053362
:10B88000FFF794F84846FFF79FFC5046FFF732F861
:10B89000054B1B68DA69598C907E727800FB0212A6
:10B8A0005A8409B0BDE8F08FD40000200D4B70B56C
:10B8B0001B68DD6906460C46E8693146FFF776FFEE
:10B8C00070B103884268F61A02EBC6035878AB7E63
:10B8D00010FB03F024B112F8362012FB03F32360AF
:10B8E00070BD00BFD400002001230B80704708B555
:10B8F000C069FFF75BFF003018BF012008BD70472B
:10B9000037B5154602AB1A4A43F8081D0190126874
:10B91000184C6946904723680190586958B901202E
:10B92000FFF7E6FB2368DB695B69BBB19B680198A5
:10B930000099984717E02946FFF767FC0028EED1E9
:10B9400014E001A801F074FF2368DB691B68054659
:10B950009847094B1B680BB128469847009B013B51
:10B96000002B0093EDDA0020FFF7C2FB03B030BDDF
:10B97000DC000020D4000020B00C022037B50D46BA
:10B980000190044698B10B4B1B68DB695B690BB1F6
:10B990005B680BB9002408E0984709E001A801F0B2
:10B9A00047FF20B10A2802D00134AC42F6DB204622
:10B9B00003B030BDD400002013B502A9002441F823
:10B9C000044D00F0B7F8019B8342CCBFC0EB0300ED
:10B9D000204602B010BD000037B5154A019002ABF9
:10B9E000126843F8081D694690470190F0B1114B69
:10B9F0001B68DB695B690BB11B6813B900252C461A
:10BA000002E00099984711E0009B013B002B009356
:10BA100007DB01A801F00CFF054600F081F80444A3
:10BA2000F2E72846FFF7C8FF2044FFE703B030BD28
:10BA3000DC000020D4000020274B1B6873B50546AE
:10BA40000C4663B10020FDF73DFC002841D028469C
:10BA500021466A46FFF754FFFDF772FBF5E71068D1
:10BA600051681E4E6B4603C33368BDF80010B3F82F
:10BA70004C20B3F850301144ADF80010BDF802105E
:10BA80001944ADF80210BDF804100A44ADF80420C2
:10BA9000BDF8062068461344ADF80630FDF712FCE9
:10BAA000336840B9598CDA6C8A1A5A84998C1A6DA9
:10BAB0008A1A9A840DE0BDF800205A84BDF802204D
:10BAC0009A84284621466A46FFF71AFFFDF738FB9D
:10BAD000E6E702B070BD00BF980C0220D400002041
:10BAE0000A4B1B689A8D02F00C02082A07D00C2A18
:10BAF00005D0042A07D1DB69187E01387047DB695D
:10BB0000187E400870470020704700BFD400002016
:10BB1000024B1B68DB69587E704700BFD4000020D1
:10BB200008B5034B1B68DB6900215B68984708BDBB
:10BB3000D400002008B5034B1B68DB695B6898479D
:10BB400008BD00BFD4000020074B5A68596A013273
:10BB500010B55A605A6B02EBC0046160002102F814
:10BB60003010586210BD00BFD40C022038B50B4D08
:10BB7000002405F140002146802285F82840FFF787
:10BB800019FA28462146C022FFF714FA2146044834
:10BB90000C22BDE83840FFF70DBA00BFD40C0220DC
:10BBA00070CE012010B542680F230D4901EBC3048C
:10BBB000246CA24203D213F1FF33F6D210BD0F2B37
:10BBC0000CD80C68A21A0A608268C06802B1506082
:10BBD00008B1026010BD01EBC3035A6410BD00BF81
:10BBE000D40C0220F8B5264EF3685A1EB36B0546F6
:10BBF0001344081898420C4605D84B591BB94368A2
:10BC00001D44FFF7CFFFB36B9C420AD954F8047C64
:10BC1000E71B3B682BB97B6838461D44FFF7C2FF22
:10BC20003C460F2306EBC302126C954203D213F17C
:10BC3000FF33F7D222E00F2B20D8083306EBC302E4
:10BC400061195268A260002084E82100246141F853
:10BC5000045C04F1080102B1516006EBC303E0602B
:10BC60005960336896F82910054A2B44336029B986
:10BC7000D168CB1A9168994238BF93602846F8BDC5
:10BC8000D40C0220254B2DE9F74FDA689C6B013A62
:10BC9000824602EB04099B4694E82800002B33D12E
:10BCA00004EB0508C8452FD254F805C0D8F8046045
:10BCB000BCF1000F28D0DBF83430184F13F83C30BB
:10BCC000012B21D1FB6A20468DE80810FFF76AFF9F
:10BCD000D8F800107A6B02EBC1022046546041464E
:10BCE000324604F003FF9DE808109C4502D17B6BAF
:10BCF0005B1B7B632846A119FFF774FFBAF1000FA5
:10BD000001D0824505D935462C444C45C4D3012089
:10BD100000E0002003B0BDE8F08F00BFD40C02208B
:10BD200028B1034AD36B036003B15860D0637047F6
:10BD3000D40C022028B1034B5B6B03EBC0004068BE
:10BD400008307047D40C0220054BD9690131D96104
:10BD50005B6B13F83010013103F83010FFF7EABFC6
:10BD6000D40C022030B50268094B52F8081C5A6BFB
:10BD700012F83140012C03D9DD690DB1013DDD61BF
:10BD8000013C02F8314000230360184630BD00BF7B
:10BD9000D40C0220024B21F0030118605960704757
:10BDA00070CE012010B5044680B1094B5B6B03EBEC
:10BDB000C00213F83030012B08D151684868FFF7F2
:10BDC00011FF2046BDE81040FFF7BEBE10BD00BF0A
:10BDD000D40C02202DE9F041224CE36A3BB9224BFE
:10BDE0009D685B680835B3FBF5F5023503E0236910
:10BDF0001D1D05EBD305E80000F044F9804660B353
:10BE0000616B2269E76A01EBC003D2005E68083605
:10BE1000304604F0C3FE2269666306EBC201C4F833
:10BE20002C8004311346681E834201F1080103D2BD
:10BE3000013341F8083CF6E706EBC30300265E60D9
:10BE4000636862629B1A2B446360256138463FB188
:10BE5000FFF7A8FF3046BDE8F0810120BDE8F08182
:10BE6000BDE8F081D40C022070CE0120F8B5584E08
:10BE700096F82810002940F0AA80564D6A680123E0
:10BE800086F82830B2F5205F28BF4FF420522B6887
:10BE900094080020A0420CD047184FF0FF0EB7FBCB
:10BEA000FEFECEEB0E2ECEEB070743F820700130DE
:10BEB000F0E70020A04216D047184FF0FF0EB7FB66
:10BEC000FEFECEEB0E2ECEEB070E53F8207077451C
:10BED00007D0AA683F4B002A55D15A6892089A6049
:10BEE00051E00130E6E701310229D2D154080021A6
:10BEF0000020A0420CD047184FF0FF0EB7FBFEFE0B
:10BF0000CEEB0E2ECEEB070723F810700130F0E7D2
:10BF10000020A0420FD047184FF0FF0EB7FBFEFEE7
:10BF2000CEEB0E2ECEEB070733F810C0BFB2BC45E8
:10BF3000CFD10130EDE701310229D9D10021002014
:10BF4000904207D04418FF27B4FBF7F73C441C5439
:10BF50000130F5E7002090420BD04418FF27B4FBD6
:10BF6000F7F73C441F5C04F0FF04A742B1D1013055
:10BF7000F1E701310229E2D100219142A9D000204C
:10BF800058540131F9E71448144B0360FFF790FB54
:10BF90005A2333620023102106EBC3029940013378
:10BFA000102B0B4C1164F6D168682968A163022339
:10BFB0002361A0F114030B4401256363E0605D601D
:10BFC00065626560FFF70EFEFFF704FF2563F8BDAD
:10BFD000D40C022070CE01207CCE01206DBB000865
:10BFE0002DE9F0410546264E0335FFF73FFF25F0CA
:10BFF0000305336CF26B04359D4238BF1D46144671
:10C000002CB154F8043CAB422CD02468F8E7F36818
:10C01000B26B02EB030858F8047CC7EB08073B68D7
:10C0200033B12046FFF72EFE58F8047CC7EB080713
:10C030003B6813BB7B68AB421FDB38461C1DFFF718
:10C04000B1FDF36878685B1BF3607369641B2B4474
:10C05000401B3C44736102D03946FFF7C3FD44F8EE
:10C06000045C0AE023680BB161685960616801B142
:10C070000B60A24201D12368F3632046BDE8F08142
:10C08000D40C02202DE9F843384D0446FFF7EEFEAC
:10C090002F6C2B68BC4224BFE71C27F003070C372A
:10C0A0009F42324C3ED8236B62689A420FD96B682C
:10C0B0006E6A013B6B606B6B4FEAC60903EB0902CA
:10C0C00052686A62012203F8362056B92AE0013B21
:10C0D0002363FFF77FFE236B013323630028E6D041
:10C0E00020E00F2305EBC302126C97420CD213F130
:10C0F000FF33F7D208E094682CB16268974214D9F4
:10C10000A268002AF7D101330F2B03D805EBC30235
:10C11000526CF6E73846FFF7B5FD0028E1D030460F
:10C12000FFF712FD0020BDE8F883D4F804802B6CE3
:10C13000C7EB08020C3320469A4238BF4746FFF748
:10C1400031FD6B6B4B44E1195C60B8454FF0000367
:10C1500084E8C000A360246141F8047C03DDC7EBE0
:10C160000800FFF73FFD3046BDE8F883D40C0220FD
:10C1700008B1FFF787BF704773B50546FFF7F8FFB3
:10C18000064658B1FFF7E0FD02AC002144F8040D6B
:10C190002A46FEF70FFF2046FFF7E4FD304602B0C7
:10C1A00070BD0000C0F3C421064B00F01F02C0F3B5
:10C1B00045109A5C5B5C03EB0243034A105C03EBA3
:10C1C00000207047006E0108C06D0108C0F30741F0
:10C1D000064BC2B2C0F307209A5C5B5C03EBC22340
:10C1E000034A105C03EB4010704700BF206F01084A
:10C1F000206E01084FF6FF7070470000F8B50F4F32
:10C200003F6806460D4614469C460FB1B847F8BD38
:10C2100056F8042B0A49D3B2013CC85CC2F3074369
:10C22000C2F30722CB5C07498A5C03EBC02303EB14
:10C2300042132B806544EBD1F8BD00BF88CE0120AE
:10C24000206F0108206E0108F8B5134E3668844649
:10C2500014461D460EB1B047F8BD501E02F1804293
:10C26000013A03FB00C001EB820102880B4B02F094
:10C270001F06D70A9E5DDB5DC2F3451203EB064342
:10C28000074EB25C013C03EB022341F80439C5EBD5
:10C290000000EAD1F8BD00BF84CE0120006E010885
:10C2A000C06D010870B50D4C2368132B06460D4672
:10C2B00012DCFFF73FFD03696E6043B12268284638
:10C2C0000132226098472368013B236070BD2846F5
:10C2D000BDE87040FDF77CB870BD00BF8CCE01207A
:10C2E00038B5054600F00FF8044654B1AC4207D00B
:10C2F0002046FFF71FFD036AAB4202D01C46F4E75D
:10C300000024204638BD08B5FCF7EAFA18B1FFF75B
:10C3100011FDC06908BD08BD38B505460C4641B1E0
:10C32000FCF7DEFA28B1A5602146BDE83840FFF7EA
:10C33000B9BF38BD024B1A6802601860704700BF71
:10C340007C0C02202DE9F043044687B0002839D048
:10C35000FFF7FAFC0346019003C804AD85E803002B
:10C3600001A81E6AD3F82890FFF7FCFC2046FFF7CF
:10C37000B7FF074630B32046FCF7B2FA19F0020FB8
:10C38000804604D0284641463246FCF798FD2046B8
:10C39000FFF7DAFC01904046FFF7D6FC03903846E1
:10C3A000FFF7D2FC039B019AD969066202901162E1
:10C3B00001A8DC61FFF7D6FC03A8FFF7D3FC02A8B5
:10C3C000FFF7D0FC07B0BDE8F0832DE9F84FDDF8AA
:10C3D00028B0DDF82CA005460E4690461F461446B0
:10C3E000894635F8020BD847D047013C49F8040B81
:10C3F000F7D11F2F06D8304641463A46BDE8F84FE0
:10C4000001F056B9BDE8F88F2DE9F84FDDF828B0F6
:10C41000DDF82CA005460E4690461F468946044688
:10C4200014F8010BD847D0472B1B434449F8040BA1
:10C43000002BF5D11F2F06D8304641463A46BDE8BD
:10C44000F84F01F035B9BDE8F88F00002DE9F04F45
:10C450009DB006460F910D92002800F08683FFF7ED
:10C4600073FC1CAB446943F81C0D1846FFF77AFCBB
:10C470003046FDF78EF80828014602DD002C00F05A
:10C48000C38101224FF0000830461B920B92CDF879
:10C490006880FFF759FC0368DFF80CA61B69B0F948
:10C4A0000A105B680E930DF1700BDAF800304BF850
:10C4B000140D04694569D0F80C90B0F90870587CE7
:10C4C0001291FEF763F9DAF800301090587CFEF70D
:10C4D0007BF9034658460993FFF744FC082C514664
:10C4E0000B9A099B04D9102C8CBF0422022205E070
:10C4F000012C03D111940DF1680800E011920E98FF
:10C50000984200F0E2800B68587CFEF765F91390C2
:10C51000B800FFF72DFE0C90002800F0268330466F
:10C52000FDF728F80646002D00F0BE802846FFF7EC
:10C530000BFCDDF834B018904FF0000A129A9245C7
:10C5400080F2AE80189800231993836819A95B695B
:10C5500052469847B84205462FD10C98FFF7F4FB96
:10C56000082C0146169009D90E9A139B009201934C
:10C5700030463A46109BFFF728FF08E00E98139AC2
:10C580000090019230463A46109BFFF73DFF012391
:10C59000109802901CAD002200930193039255F86D
:10C5A000182D04920F98CDF8148059463A46FEF79C
:10C5B00005FB2846FFF7D6FB60E0012C5CD1002D7F
:10C5C0005CD019980F99CDF80C90082290FBF2F2EC
:10C5D00032440123049200F00702009308440193BF
:10C5E0000293069259462A46CDF81480FEF70AFABD
:10C5F000199B18981D44836819955B6919A95246BF
:10C6000098470546DBE70C98FFF79EFB082C014690
:10C610001690199838D90E9A0092119A139B01938B
:10C6200000FB0260109B2A46FFF7CFFE01230DF1AD
:10C63000700C109800930022019302900F990392BE
:10C6400019985CF8182D049208442A465946CDF8EA
:10C650001480CDF82CC0FEF7B1FADDF82CC060468E
:10C66000FFF780FB199B18981D44836819955B6937
:10C6700019A9524698470546002DC4D14E440AF1E7
:10C68000010A0BF1010B59E70E9B0093119B139AC2
:10C69000019200FB03602A46109BFFF7B5FEC5E739
:10C6A00018A8FFF75FFB0EE00123009301930490AD
:10C6B0000294CDF80C90CDF814800F980D99129B30
:10C6C0003A46FEF77BFA0C984DE23046FCF752FFF3
:10C6D0000646002D00F08A802846FFF735FB00252E
:10C6E0001890129B9D427DDA189800231993836855
:10C6F00019A95B692A469847B842824624D1AA46BE
:10C70000189883680AF1010B5B6919A95A46984782
:10C71000B84201D1DA46F3E7C5EB0A0B0D9904964E
:10C7200001230BF1010B0093019329440294CDF8EE
:10C730000C90CDF814800F983A465B46FEF73EFA0F
:10C7400009FB0B6655464BE0012C27D1BAF1000FCF
:10C7500022D019980F99CDF80C90082290FBF2F294
:10C760003244049200F0070208440D990692012316
:10C7700052460093019302932944CDF81480FEF7AA
:10C7800041F9199B189853441993836819A95B6957
:10C790002A4698478246D9E74E4421E0BAF1000F75
:10C7A000FAD019981199029400FB016204920D9934
:10C7B0000F9ACDF80C900123104400935246019338
:10C7C0002944CDF81480FEF7F9F9199B18985344C1
:10C7D0001993836819A95B692A4698478246DDE761
:10C7E00001357EE718A8FFF7BDFABEE101230093EB
:10C7F000019304900294CDF80C90CDF814800F981A
:10C800000D99129B3A4641E030460A91FFF79CFA97
:10C8100082461CA8BAF80A2040F810ADDAF80040A9
:10C820001092D4F81090BAF808709E4C13B2DAF84F
:10C830000C200B920993FFF795FAD9F804000E909B
:10C8400099480068407C54F820402569D5F800805C
:10C85000FDF79CFF08280FFA87FB0A990B9A099BA2
:10C8600004D910288CBF0424022400E00124A94527
:10C870000FD1012003920AF1180200900190029159
:10C8800004920F980D99002205925A46FEF796F9E8
:10C890006BE1202940F08E800BFB04F0FFF768FC71
:10C8A0000E90002800F06181FFF74EFA1A90304692
:10C8B000FFF74AFA18902B6900F1180A4FEA8B0625
:10C8C0004FEAC409002B2FD0DDF83480022C03D0AE
:10C8D000042C01D0012C06D150462F691A995A46D2
:10C8E0002346B847B244012300221A9900930193CA
:10C8F00003920491059241465A46CDF808900F984C
:10C90000FEF75CF910990D9A08F1010702FA81F31C
:10C91000BB4207D118A8FFF725FA1AA8FFF722FA99
:10C920000E9820E1B846D1E70D9D022C1A9F0ED03B
:10C93000042C18D0012C25D100235AF82300099388
:10C94000C047099BF85401339B45F6D119E00023F9
:10C950005AF823000993C047099B27F813000133B5
:10C960009B45F5D10DE05A4600235AF803000B927F
:10C970000993C0470B9A099B013AF85003F104034D
:10C98000F3D1B244012300221A9900930193039238
:10C99000049105920F98CDF8089029465A46FEF763
:10C9A0000DF910980D996F1C01FA80F3BB42B1D0BC
:10C9B0003D46BAE7102940F0D8800FFA87FA0AFB03
:10C9C00004F0FFF7D5FB1290002800F0CE80FFF7AF
:10C9D000BBF91A903046FFF7B7F918902B6900F1B0
:10C9E000180613B1D9F814302BB9E2003FB21192F6
:10C9F0007F000D9D88E0B0F908008000FFF7B8FBCC
:10CA0000119018B1FFF7A0F9199001E0119B19934B
:10CA1000199B002B00F0A0803FB27F000E97E7002B
:10CA200013970D9F0C97022CDDF8688004D0042C1E
:10CA300007D0012C14D104E0304619995246234600
:10CA400003E01999304652460223D9F81470B847CA
:10CA50002F691998414652462346B8470E9F3E44D7
:10CA60000C9F1A9904910123002207F10108139FDA
:10CA7000009301930297039205920F980C995A46DE
:10CA8000FEF79CF8109F0D9800FA87F3434502D0FB
:10CA9000CDF83080C7E719A8FFF764F91198FFF7C0
:10CAA00081F959E0C40C0220D4000020042C41D0AC
:10CAB000012C11D14A46314631F8020B0A910B92F2
:10CAC0000E9B9847C0470B9A02F8010B09EB0A002E
:10CAD00082420A99F0D13E44012311981A99009399
:10CAE00000220193029003920491059229465A462E
:10CAF0000F98FEF763F810990D9A05F1010902FAF3
:10CB000081F34B4528D04D46022CDDF86890CDD1FD
:10CB10004B463146D94631F8020B0A9109930E9AD9
:10CB20009047C047099B0A9923F8020BB9F1010904
:10CB3000F1D1D0E74B463146D94631F8020B0A9184
:10CB400009930E9A9047C047099B0A9943F8040B32
:10CB5000B9F10109F1D1BEE718A8FFF703F91AA846
:10CB6000FFF700F91298FFF71DF91DB0BDE8F08F2F
:10CB700037B50546FFF7E8F8024602A8948940F861
:10CB8000042D013CA4B29481FFF7ECF814B92846B7
:10CB9000FFF708F903B030BD2DE9F8430546884694
:10CBA00017469946A8684B46466841462846541C95
:10CBB000B047089B3B44A34201D02246F2E7BDE8C0
:10CBC000F88300000248012918BF0020704700BF09
:10CBD000C85601080248162918BF0020704700BF38
:10CBE0004DC40008006808B510B1C3681B6A9847B7
:10CBF00008BD006808B518B1C3689B6A984708BDAE
:10CC00004FF0FF3008BD37B580680C46FFF79CF841
:10CC1000034602A89988DA881D8940F8043D5B899B
:10CC20002180628029441A440139013AA180E280BE
:10CC3000FFF798F803B030BD0E4B1B6873B505467F
:10CC4000186E0E46FFF780F8034602A8B3F90640B7
:10CC500040F8043D03F11801361BDC68B3F90430D9
:10CC600004FB0614ED1AFFF77DF804EB450420469B
:10CC700002B070BDD400002008B508461146FFF789
:10CC8000DBFF008808BD0000144B1B68F7B50746A2
:10CC9000186E15460E46FFF757F8294600903046A5
:10CCA000FFF7CAFF3B6904469B68984723885840B2
:10CCB000009B2080586960B1FFF746F802AC83689A
:10CCC00044F8040D1B6831462A4698472046FFF772
:10CCD00049F86846FFF746F803B0F0BDD4000020DD
:10CCE00073B51C46104B1B68186E0E461546FFF7B1
:10CCF0002BF8294600903046FFF79EFF009B0480EA
:10CD0000586960B1FFF720F802AC836844F8040D5D
:10CD10001B6831462A4698472046FFF723F86846A5
:10CD2000FFF720F802B070BDD40000202DE9F347D2
:10CD30002C4D1E462B688146186E0F461446FFF791
:10CD400003F800904069AA4608B1FEF7FDFF019084
:10CD500021463846FFF770FF009BD3F80C80DAF8C5
:10CD600000301A7CD20705461FD5D9F810309B68D1
:10CD700098471FFA80F8019820B1836839461B68EC
:10CD8000224698472B8888EA03032B80009B0134B6
:10CD9000DB68B4421D44EEDD6846FEF7E3FF019B0D
:10CDA000EBB101A8FEF7DEFF19E0DB6BD3F80090D2
:10CDB000019B63B10198836822461B6839460134A0
:10CDC0009847B442A5F800904544F3DDE4E7341BEE
:10CDD0000134013CA5F800904544FAD1DCE702B0EB
:10CDE000BDE8F087D40000202DE9F04F2A4F14460B
:10CDF0003A689846D36B87B01B6802938246106EE0
:10CE00000E46FEF7A1FF214604903046FFF714FFBF
:10CE1000049A05465069D3680393C6EB080909F1E3
:10CE20000108BB4680B1FEF78FFF109A06AF131BB7
:10CE300047F8040D01330093314622464346FFF77D
:10CE4000ABFE3846FEF78EFF4FEA4906109B9C4228
:10CE50001CDCDBF800301B7CDB070DD5DAF810306A
:10CE60009B689847AA1980B2AB1E5988414023F8A5
:10CE7000021F9342F9D105E0029B284699B242462F
:10CE8000FEF76AF8039A01341544DFE704A8FEF7B9
:10CE900069FF07B0BDE8F08FD400002007B500920D
:10CEA000FFF7A2FF03B05DF804FB00002DE9F04F8F
:10CEB000814C93B09B4623680D90186E07920D46E7
:10CEC000DDF87CA0FEF740FF1090406908B1FEF746
:10CED0003BFF119012A850F8083DDB680993FEF75C
:10CEE00041FF209E11982E44049650B123681B7C6C
:10CEF000990706D11C9F00973146079A5B46FFF7BA
:10CF00004BFE04980799FFF797FE1D9E102E0446CE
:10CF100027D14FEA4B0600251C9FDDF84480BD4217
:10CF20001ADABAF1000F11D084B1204651463246C8
:10CF300003F034FEB8F1000F08D0D8F80830079A93
:10CF40005F68049940462A445B46B8471E9FBA442E
:10CF5000099F01353C44DFE7B8F1000F40F01B8327
:10CF60001CE31D9E172E38DD00261C9F119DBE421E
:10CF700080F29D80079F3744BAF1000F27D034B369
:10CF80003DB1AB680499D3F804C028463A465B46E5
:10CF9000E047A31EAAF104090393D846049B0D9809
:10CFA0005B44C8EB0301036959F8040F1B68029145
:10CFB0009847039B029923F8020F039325B1AB68AE
:10CFC00028461B683A469847B8F10108E6D11E9FEB
:10CFD000BA44099F01363C44C7E71D9E082E00F164
:10CFE00002046BD1079E079F119DF31B1C9FBB4240
:10CFF000A4F102005BDA304B219F1B681B7C67B3F6
:10D0000013F0030304D0022B4BD1A046049F1DE074
:10D010001AF80320219F57F8222020F8132001330B
:10D020005B45F5D13DE0219951F8233028F8023CC9
:10D030002DB1AB6828461B68394632469847049B99
:10D0400001375B44BB4208F102082AD00498C0EBC8
:10D050000A03DB5D002BF2D0E5E713F0030304D0F5
:10D06000022B1ED1A046049F14E051465A4603F0FD
:10D0700095FD16E028F8023C2DB1AB6828461B68E8
:10D08000394632469847049B01375B44BB4208F15E
:10D09000020806D0049AC2EB0A03DB5D002BF2D033
:10D0A000E8E71E9FBA44099F01363C449BE7002DE8
:10D0B00040F0718272E200BFD4000020219EAB4B91
:10D0C000209F0894002E08BF1E462196209E7600C1
:10D0D0000E96BF00079E0F970596089B059E079F1B
:10D0E0009C1EF31B1C9EB34280F253821D9F022F95
:10D0F00000F0D980042F00F07881012F40F03F82AA
:10D10000DFF87092D9F80030186EFEF71DFE9AF81D
:10D110000030974A1090D55CD9F8003020981B7CDD
:10D12000119F03F00303022B5E46C0F1080845FA85
:10D1300000F522D0032B62D0012B60D05246464529
:10D1400038BFB046C8EB06064346214605F001004D
:10D15000219F013B57F8200021F8020B4FEA5505AB
:10D16000F4D104EB4804002E00F0998012F8013F3E
:10D170007F494FF00808CD5CE1E72198DDF8109079
:10D18000B0F804C0CDF818A0464538BFB046C8EB8B
:10D1900006062FB31DB904EB4804C14424E0EA0796
:10D1A0000BD5BB68059A1B68CDF808C038464946C0
:10D1B0009847DDF808C0A4F800C0B8F1010809F1EB
:10D1C000010904F102040FD06D08E3E7EB0748BF43
:10D1D000A4F800C0B8F1010804F1020404D06D08FD
:10D1E000002DF3D104EB4804002E58D00699604A74
:10D1F00011F8013F0691D55C4FF00808C4E70D9A7D
:10D2000013699B689847049B0B9380B20A900AF1BC
:10D210000109464538BFB046C8EB0606A31C1FB33C
:10D22000CDF818800B98069A40440C90811AE807B4
:10D230000DD5BA683846D2F800C0059A0293E04787
:10D24000029B0A9833F8022C424023F8022C0699DC
:10D2500001394FEA550503F102030691E2D10C9B17
:10D260000B9304EB480410E04246E90705D533F878
:10D27000021C0A98414023F8021C013A4FEA550566
:10D2800003F10203F1D104EB480446B199F80030F0
:10D29000374A09F10109D55C4FF00808B9E710A831
:10D2A000FEF760FD6BE1334B209E1B680E9F1B7CDD
:10D2B000DDF84490C6F104059AF8006003F003031A
:10D2C000BE40012BEDB2F6B26AD008D3022B40F07B
:10D2D0005681CDF818A05F46DDF810C03EE05246FA
:10D2E0005B469D42C8BFDDB25B1B294620464FEA24
:10D2F000961C219F013957F82CC020F802CBB600AC
:10D3000011F0FF01F6B2F2D1013DEDB2013504EBAF
:10D310004504002B00F0338112F8016F0425E0E78B
:10D3200016F0C00F08EB0C0126D108F101085FFAD6
:10D3300088F3B6009D42F6B2F2D1013DEDB26B1C0E
:10D3400004EB43040CF1010303EB050C002F00F088
:10D350001681069B13F8016F06930425BD42C8BFD2
:10D36000FDB27F1B4FF00008DAE700BF88560108C6
:10D370005C550108D4000020B309219850F82330EF
:10D3800024F81830B9F1000FCFD0D9F80830059A39
:10D390001B68CDF808C048469847DDF808C0C4E7C8
:10D3A00051465B469D42C8BFDDB25B1BA21C2846AE
:10D3B00016F0C00F05D032F8027C87F0FF0722F884
:10D3C000027C0138B60010F0FF00F6B202F1020252
:10D3D000EED1013DEDB2013504EB4504002B00F028
:10D3E000CE8011F8016F0425DCE76E4A9AF8003010
:10D3F00012680F9F127C119E02F00302BB40012AAB
:10D40000DDB200F0958002D3022A36D0B7E0209E2C
:10D4100066B12D09219F57F8253023800AF10102BA
:10D42000089C9AF801500BF1FF3301E05B4652462D
:10D43000012B19DD5810211D03F0010302EB000C34
:10D440002F09219E05F00F0556F8277056F8255034
:10D4500021F8047C21F8025C12F8015F624501F1B9
:10D460000401EDD104EB8004002B00F088802D092D
:10D47000219F57F82530238081E0209FC7B113F00A
:10D48000F00F0BD02D09219F57F8253023802EB1A6
:10D49000B36804991B68059A304698470498089C1D
:10D4A0009AF80150471C0BF1FF390AF101080FE00F
:10D4B000D946D046049F0BE015F0F00F0CD115F0C3
:10D4C0000F0517D118F8015F04340237A9F10209DA
:10D4D000B9F1010FF0DC1AE02B09219951F8233042
:10D4E0002380002EEBD0B368059A1B68304639467E
:10D4F0009847E4E7219A52F825306380002EE1D066
:10D50000B368059A1B683046791C9847DAE7B9F189
:10D51000000F34D02D0932D0219850F825302380C7
:10D520006EB3B368059A1B6830463946984726E0C3
:10D53000209EC6F10203DBB250465A469342C8BF52
:10D54000D3B2D21AA11C1E4615F0C00F05D031F877
:10D55000027C87F0FF0721F8027C013E2D0116F0C6
:10D56000FF06EDB201F10201EED1013BDBB2013366
:10D5700004EB43041AB110F8015F0223DEE71E9F9B
:10D58000059B099EBA44089F0133374405930897C9
:10D59000A3E5119B13B111A8FEF7E4FB13B0BDE89E
:10D5A000F08F00BFD400002010B50D4B1A68517CDD
:10D5B0000C4A52F821001C4640B1C36813B11B68E5
:10D5C000042B01D00068F7E7FDF776FF23680022FF
:10D5D0001A6603F108025A61BDE81040FDF7FABB74
:10D5E000D4000020C40C022010B5034C2068FEF7C4
:10D5F00097FB0023236010BDC40D022038B5094DF0
:10D600002C685CB9084B18688000FEF7E9FC2860BC
:10D6100030B10648064B0360FEF74AF8002038BDDB
:10D62000012038BDC40D0220E000002090CE012072
:10D63000E9D500082DE9F04700F089FA002480467A
:10D6400044452CDA2046FDF7FFFE30B3154E336813
:10D65000204693F811905C74FDF77EF8082803DDEE
:10D66000336883F8119018E00F4B53F824301A698F
:10D670000E4B9A42F4D02046FDF771F80025824601
:10D680005545EDDAEFB23846FDF70EFC3946024655
:10D690002046FDF729F80135F2E70134D0E7BDE86F
:10D6A000F08700BFD4000020C40C022030700108B5
:10D6B000082A10B50EDD102A0ADC00EB41010346F2
:10D6C00050F8042B23F8022B8B42F9D1012010BD16
:10D6D000002010BD022A6DD0042A54D0012A40F047
:10D6E00095800446036801294FEAC313DBB247D093
:10D6F0004268022902F0010243EA821302D100F1DA
:10D7000008023EE08268032902F0010243EA421364
:10D7100002D100F10C0234E0C268042902F00102D7
:10D7200043EA021302D100F110022AE0026905293E
:10D7300002F0010243EAC20302D100F1140220E028
:10D740004269062902F0010243EA820302D100F194
:10D75000180216E08269073902F0010243EA420327
:10D7600002D100F11C0205E000F12002C06900F0C6
:10D770000100034304F8013B0029A7D01046B1E79C
:10D78000021D0021F6E70246036801294FEA031350
:10D79000DBB202D1041D002106E000F1080440685C
:10D7A00000F00F000343023902F8013B00298DD03D
:10D7B0002046E9E70446036801294FEA8313DBB2F8
:10D7C00021D04268022902F0030243EA021302D187
:10D7D00000F1080218E08268032902F0030243EA1C
:10D7E000820302D100F10C020EE000F11002C068C9
:10D7F00000F003000343043904F8013B00293FF41F
:10D8000065AF1046D7E7021D0021F5E7002350F869
:10D810002320C25401338B42F9D157E70078704777
:10D8200001207047012070470170012070470000FF
:10D83000F8B5084E0468336805461B6820469847CB
:10D84000336807465B68204698472044286038467E
:10D85000F8BD00BFBC0C022070B504460E46002582
:10D8600046B1054B1B6820465B689847013E04445F
:10D870000544F5E7284670BDBC0C0220034B1B682D
:10D88000B3F92C2098851046704700BFD4000020C3
:10D890000A46084910B5088007490A8007490968FF
:10D8A0000346487C064951F82000C1680C6A1946B5
:10D8B000A04710BDAC0C0220A00C0220D400002018
:10D8C000C40C022008B500F051F9BDE80840FDF78E
:10D8D000EBBA08B500F052F9BDE80840FDF7E4BA2C
:10D8E000524B2DE9F04F1B68D9695F8CCC699D8C38
:10D8F000A28990428BB008D3E689864205D3D4F83A
:10D900000090821A4FF0FF3B15E0A268D4F8049013
:10D91000002A00F081801688B0427DD3B2F802C0A0
:10D92000844579D35268801B80B202EB800632F9BD
:10D930002020B6F902B0501C6ED091F81880A17C5E
:10D94000B3F82AA0267C069218FB01F107910FFA82
:10D950008AF108460891FCF7CDFF344909900B681D
:10D96000069AD969887E0090C97E019101210291B1
:10D97000A17C0391079901FB029204929B6B059392
:10D980003FB22DB23846294632464346FDF716F9D6
:10D99000BBF1FF3F1BD04AF0020000B2FCF7AAFF28
:10D9A000224A1368DA69917E0091D27E01920121A8
:10D9B00002910799A27C039201FB0B9204929B6B4C
:10D9C00005933846294632464346FDF7F7F8DFF817
:10D9D0005C80D8F80030DB695A7E1B7E9A4217D9EA
:10D9E000089A022A14D08AF0040000B2FCF782FFE1
:10D9F000D8F80030DB6993F818E0D97E9A7E5B7E18
:10DA000038460EFB015106FB02722B44FCF7CEFF99
:10DA1000099BD8B2FCF76EFF044B617C1B685A8CE3
:10DA20000A445A840BB0BDE8F08F00BFD400002038
:10DA3000044B1B68DB69DB6909B11A7C0A60587CFE
:10DA4000704700BFD400002002230B807047C369D9
:10DA50009A898A4202D8DA898A420FD2986880B1BC
:10DA6000038899420CD342888A4209D3C91A426872
:10DA700032F82100C043C0F3C03070470120704726
:10DA80000020704708B5FCF771FEB0F5807F10D01C
:10DA90007F2810D83F2810D81F2810D80F2810D85A
:10DAA000072810D8032810D8012894BF002001208F
:10DAB0000CE008200AE0072008E0062006E0052028
:10DAC00004E0042002E0032000E00220012303FA26
:10DAD00000F0013808BD38B50446FCF747FE05469E
:10DAE000FCF76AFEAC4203D218B150F8240038BDEE
:10DAF000002038BD2DE9F8438146FCF737FE80460B
:10DB0000FCF75AFE0646D8B1002356F8232091456B
:10DB10001AD001334345F8DB00256FF07F472C46D0
:10DB200056F82410484600F031F8B84238BF254670
:10DB300004F1010428BF3846444502DA0746EFE7FE
:10DB400005462846BDE8F8831846BDE8F88310B5B9
:10DB50000020FDF779FC041C4FF0010018BF0124E0
:10DB6000FDF772FC00B10134204610BD024B1B686A
:10DB70009B6B1868704700BFD4000020024B1B68E5
:10DB8000DB6B1868704700BFD4000020CBB2C2B274
:10DB9000D21A92B293B230B51C0448BF5342C1F3BB
:10DBA0000725C0F30722C5EB020248BF9BB292B221
:10DBB000090C13FB03F4C1EB104193B21D0489B2AD
:10DBC00088B244BF53429BB2020448BF484213FB91
:10DBD000034348BF80B200FB003030BD704700BF38
:10DBE00010B582B000246846009400F0E9F9064BB5
:10DBF00001940246012101A81A6000F0E5F9034BE7
:10DC0000186002B010BD00BF9CCE012098CE01204C
:10DC100010B50446034B4068236000F0F7FF204630
:10DC200010BD00BF5070010810B50446054B406898
:10DC3000236000F0EBFF2046082101F015FD20468F
:10DC400010BD00BF5070010808B54FF0FF3200232F
:10DC5000406800F061FDA0F10100B0FA80F04009D9
:10DC600008BD00BF08B54068002300F055FDA0F1D5
:10DC70000100B0FA80F0400908BD00BF08B5406857
:10DC8000002300F02DFEA0F10100B0FA80F0400961
:10DC900008BD00BF10B50446054B23600846114679
:10DCA000002200F0E7FC034B60602360204610BDBB
:10DCB000507001084415010810B50446034B406834
:10DCC000236000F0A3FF204610BD00BF6C70010868
:10DCD00010B50446054B4068236000F097FF2046CE
:10DCE000082101F0C1FC204610BD00BF6C70010886
:10DCF00008B500230A464068194600F0A9FEA0F1C5
:10DD00000100B0FA80F0400908BD00BF08B500234B
:10DD10001A461946406800F0FFFCA0F10100B0FA75
:10DD200080F0400908BD00BF08B5406800F03AFE29
:10DD3000A0F10100B0FA80F0400908BD10B504461A
:10DD4000044B23600846114600F0C8FC6060204682
:10DD500010BD00BFB015010808B503689B6898475F
:10DD60004FF0100383F31188BFF36F8FBFF34F8F12
:10DD7000FEE700BF10B5034B0360044600F0C8F88F
:10DD8000204610BDA87001082DE9F0410446A446C4
:10DD900018484D6882B04CF8080B0CF10800A060E0
:10DDA0000F2DD1F80080019517461E4612D8012D7F
:10DDB0000DD198F8003023740023E56043552046C8
:10DDC0002784666284F8283002B0BDE8F081002D17
:10DDD000F2D007E06046002201A901F053FC019B4C
:10DDE000A06023612A46414602F0D8FE019DA0684A
:10DDF000E2E700BF7C70010830B5194B1B7887B093
:10DE00000446CBB990F828303BBB012380F828307A
:10DE10000023211D656A228C039302930191A1685E
:10DE200010480095234600F04BFFA0F10100B0FA26
:10DE300080F0400907B030BD0B4905A800F080F81C
:10DE400094F8283033B9012384F8283005A800F06D
:10DE500083F8DDE705A800F07FF8002007B030BDAB
:10DE6000A8CE012059DD0008A0CE012003464FF0C6
:10DE7000FF3210B54260044653F8080F054A22608D
:10DE80000833984203D02169013101F0EDFB2046AF
:10DE900010BD00BF7C70010810B5054B036004463F
:10DEA00000F036F82046082101F0DEFB204610BDC8
:10DEB000A870010808B5054800F036F8BDE808402C
:10DEC000034A04490148F2F7E5BA00BFA0CE012099
:10DED000BD04000875DD000808B500230A46406847
:10DEE000194600F0B5FDA0F10100B0FA80F040093C
:10DEF00008BD00BF08B500231A461946406800F067
:10DF00000BFCA0F10100B0FA80F0400908BD00BF91
:10DF100010B50446034B4068236000F077FE2046AE
:10DF200010BD00BF9070010810B5044B036004469B
:10DF3000012000F0AFFC6060204610BDA870010811
:10DF400010B50A6801600B46044612684FF0FF31B5
:10DF500018469047204610BD10B504460068036877
:10DF60005B689847204610BD38B504461D46FFF74C
:10DF70000BFF06230B49E3620822236321606263DF
:10DF80000021402204F1380002F0C9FD4C22182182
:10DF900004F17800FFF77EFE023D034B204643F874
:10DFA000254038BD60150108ACCE012008B5012917
:10DFB00038BF0121084601F0EFF8002008BD00BF7E
:10DFC000012000F067BC00BF012910B5084604D04D
:10DFD000BDE81040002100F081BB0322002100F0C9
:10DFE00049FB044620B100231A46194600F094FB71
:10DFF000204610BD0A4B1B68013308D04FF01003B8
:10E0000083F31188BFF36F8FBFF34F8FFEE74FF09D
:10E01000100383F31188BFF36F8FBFF34F8FFEE7B9
:10E02000E400002006480068006880F3088862B6B3
:10E0300061B6BFF34F8FBFF36F8F00DF00BF0000EB
:10E0400008ED00E0DFF80C00016841F470010160A8
:10E050007047000088ED00E04FF0807310B440F886
:10E06000043C074C40F80C4C6FF0020340F8081CCD
:10E0700040F8202C40F8243C5DF8044B44387047AD
:10E08000F5DF0008064B19680868B0E8F04F80F328
:10E090000988BFF36F8F4FF0000080F3118870473D
:10E0A0002C0C02204FF0100383F31188BFF36F8F05
:10E0B000BFF34F8F0B4A13680133012B136000D05D
:10E0C00070474FF0E023D3F8043DDBB2002BF7D0CC
:10E0D0004FF0100383F31188BFF36F8FBFF34F8F9F
:10E0E000FEE700BFE4000020084A136843B94FF080
:10E0F000100383F31188BFF36F8FBFF34F8FFEE7D9
:10E10000013B13600BB983F311887047E4000020D2
:10E11000EFF30980BFF36F8F134B1A681EF0100FD7
:10E1200008BF20ED108A20E9F04F106008B44FF0CE
:10E13000100080F31188BFF34F8FBFF36F8F01F092
:10E1400075F84FF0000080F3118808BC1968086862
:10E15000B0E8F04F1EF0100F08BFB0EC108A80F34B
:10E160000988BFF36F8F70472C0C022008B5EFF3BE
:10E1700011834FF0100282F31188BFF36F8FBFF34A
:10E180004F8F00F0CFFE28B14FF0E0234FF08052C8
:10E19000C3F8042D002383F3118808BD064B0749FB
:10E1A0001B68A1FB03134FF0E0229B09013B0721F1
:10E1B00053611161704700BFC4000020D34D62104D
:10E1C00030B54FF0E023344AD3F8001D914283B0BC
:10E1D00059D0D3F8002D314B9A424BD0304B314CB3
:10E1E0001A783148FF21D2B2019219701B78DBB244
:10E1F0008DF803309DF803309DF8032003F01003E1
:10E2000007211206237001600DD506229DF8033008
:10E210005B00DBB28DF803309DF803301B0611461E
:10E2200002F1FF32F2D4019A1D4D0B024FF0E024AF
:10E23000D2B203F4E06303602A70D4F8203D43F4C3
:10E240007003C4F8203DD4F8203D43F07043C4F877
:10E25000203DFFF7A3FF154B00221A60FFF7F2FEE7
:10E26000D4F8343F43F04043C4F8343FFFF7DAFEBC
:10E27000FFF7C0FE4FF0100383F31188BFF36F8FD9
:10E28000BFF34F8FFEE74FF0100383F31188BFF306
:10E290006F8FBFF34F8FFEE771C20F4170C20F4106
:10E2A00000E400E0C0CE0120BCCE0120E40000204C
:10E2B000EFF305830F2B0ED91149124A5B5C1278DC
:10E2C0009A4208D94FF0100383F31188BFF36F8F80
:10E2D000BFF34F8FFEE74FF0E0230B4AD3F80C3D1E
:10E2E000126803F4E063934208D94FF0100383F3FC
:10E2F0001188BFF36F8FBFF34F8FFEE7704700BFEA
:10E30000F0E300E0C0CE0120BCCE012010B4144BDD
:10E310001A461B688342FBD35468416802EB040C25
:10E32000604512D04418A34206D00360824218BF51
:10E3300010605DF8044B70470A4C2468A342F4D087
:10E3400018CB214403604160F0E721445018834218
:10E350005160EED1034800688342EAD01046EFE7EF
:10E36000D4CE0120D0CE01202DE9F8433E4E044604
:10E3700000F0D0FD3368002B58D03C4B1D682C4278
:10E380002ED16CB304F1080160071CBF21F0070116
:10E39000083129B3DFF8E880D8F800708F421FD326
:10E3A0003348046803E0236823B120461C466268B2
:10E3B0008A42F8D33368A34212D0531A2668D0F8A1
:10E3C00000900660102B16D9601842070ED04FF04F
:10E3D000100383F31188BFF36F8FBFF34F8FFEE7F6
:10E3E00000F0CAFE00263046BDE8F8834360616055
:10E3F000FFF78CFF62681F4B1968BF1A8F4238BF46
:10E400001F602A4300232360626009F10806C8F8F0
:10E41000007000F0B1FE7307E5D04FF0100383F3F6
:10E420001188BFF36F8FBFF34F8FFEE7124B134A74
:10E4300010490E4F5D0718BF07330D4D22F007023C
:10E4400018BF23F007032B601846D31A0B600C4942
:10E4500032600B60002169604FF00045C2E9001195
:10E460003D60C0E900238AE7D0CE0120C4CE012060
:10E47000D4CE0120C8CE0120DCCE0120D40A022057
:10E48000CCCE012000B583B0D0B11A4A50F8043C7C
:10E49000126813420BD050F8081CA1B14FF01003C2
:10E4A00083F31188BFF36F8FBFF34F8FFEE74FF0F9
:10E4B000100383F31188BFF36F8FBFF34F8FFEE715
:10E4C00003B05DF804FB23EA020340F8043C01902A
:10E4D00000F020FD084A0198116850F8043C083803
:10E4E0000B441360FFF712FF03B05DF804EB00F07C
:10E4F00043BE00BFC4CE0120CCCE012038B5036C92
:10E50000044615463BB90568002D2CD00020A36BAE
:10E510000133A36338BD6AB91A46806802F03EFB36
:10E52000A368216C62680B449342A360EED3236816
:10E53000A360EBE71A46C06802F030FB226CE36888
:10E5400021689B1A8B42E360C2F1000202D2636829
:10E550001344E360022DD9D1A36B002BD6D0A36B5B
:10E56000013BA363D2E7406800F0CCFF6560CEE7D3
:10E5700038B50446FFF796FDA36C002B12DD04F1BD
:10E58000240505E0A36C013BA364A36C002B09DD0B
:10E59000636A284633B100F0B9FE0028F2D000F0DB
:10E5A00053FFEFE74FF0FF33A364FFF79DFDFFF745
:10E5B00079FD636C002B12DD04F1100505E0636C3E
:10E5C000013B6364636C002B09DD2369284633B18A
:10E5D00000F09CFE0028F2D000F036FFEFE74FF08D
:10E5E000FF336364BDE83840FFF77EBD38B50D46A4
:10E5F0000446C8B1FFF756FD236CE26B2168A160A9
:10E6000003FB02F2D31A0A4462600022A2630B44A5
:10E610004FF0FF326264E360A26475B92369C3B945
:10E62000FFF762FD012038BD4FF0100383F311881E
:10E63000BFF36F8FBFF34F8FFEE704F1100000F0C0
:10E64000C9FF04F1240000F0C5FFFFF74DFD0120D4
:10E6500038BD04F1100000F059FE0128E0D14FF060
:10E66000E0234FF08052C3F8042DBFF34F8FBFF368
:10E670006F8FD5E7F8B50E461746044640B94FF000
:10E68000100383F31188BFF36F8FBFF34F8FFEE743
:10E6900079B95420FFF768FE0546A8B10060EC6325
:10E6A0002E6401212846FFF7A1FF85F85070284607
:10E6B000F8BD01FB00F05530FFF756FE054618B1D6
:10E6C00000F154030360EAE74FF0100383F311886D
:10E6D000BFF36F8FBFF34F8FFEE700BF10B50C463F
:10E6E00040B94FF0100383F31188BFF36F8FBFF36E
:10E6F0004F8FFEE7884208D24FF0100383F3118852
:10E70000BFF36F8FBFF34F8FFEE702220021FFF7A9
:10E71000B1FF846310BD00BFF0B585B00E46019215
:10E720001D460446002877D0002965D0022D0BD164
:10E73000E36B012B08D04FF0100383F31188BFF374
:10E740006F8FBFF34F8FFEE700F084FE00286CD080
:10E75000FFF7A8FCA26BE36B9A4272D3022D70D034
:10E76000002217460EE0FFF7BFFC2046FFF700FF30
:10E7700000F002FDFFF796FCA16BE36B99424FF0AE
:10E7800001025ED30198002872D0002A40D0FFF722
:10E79000ABFC00F0BFFBFFF785FC636C013308BFE7
:10E7A0006764A26C013208BFA764FFF79DFC01A952
:10E7B00002A800F007FE00285ED1FFF773FCA26BF1
:10E7C000E36B9A42CFD1FFF78FFC019904F110005F
:10E7D00000F064FD2046FFF7CBFE00F0CDFC0028E2
:10E7E000C8D14FF0E0234FF08052C3F8042DBFF39F
:10E7F0004F8FBFF36F8FBDE7036C002B96D04FF0A8
:10E80000100383F31188BFF36F8FBFF34F8FFEE7C1
:10E8100002A800F0C1FDBAE74FF0100383F311889E
:10E82000BFF36F8FBFF34F8FFEE7019B002B8FD09D
:10E830004FF0100383F31188BFF36F8FBFF34F8F37
:10E84000FEE72A4631462046FFF758FE636ACBB9F9
:10E8500048B14FF0E0234FF08052C3F8042DBFF3CE
:10E860004F8FBFF36F8FFFF73FFC012005B0F0BD66
:10E87000FFF73AFC0020F9E72046FFF779FE00F0A9
:10E880007BFCF7E704F1240000F040FD0128EAD109
:10E89000DFE700BF70B506465420FFF765FD04466C
:10E8A000D8B100254FF0FF3301228563C263436472
:10E8B0004560836405608560C560056480F85060CC
:10E8C000103000F087FE04F1240000F083FE2B4698
:10E8D0002A4629462046FFF71FFF204670BD00BF8D
:10E8E0002DE9F0410E4617461D460446002841D04A
:10E8F00021B3022D0BD1E36B012B08D04FF0100395
:10E9000083F31188BFF36F8FBFF34F8FFEE7FFF7DD
:10E91000CFFCEFF311884FF0100383F31188BFF39E
:10E920006F8FBFF34F8FA26BE36B9A4212D3022D0E
:10E9300010D0002088F31188BDE8F081036C002B13
:10E94000D7D04FF0100383F31188BFF36F8FBFF35D
:10E950004F8FFEE72A4631462046FFF7CFFDA36CD6
:10E96000013310D0A36C0133A364012088F3118814
:10E97000BDE8F0814FF0100383F31188BFF36F8F70
:10E98000BFF34F8FFEE7636A002BEED004F1240043
:10E9900000F0BCFC0028E8D0002FE6D001233B604B
:10E9A000E3E700BF70B50D46044648B3036C43B1BE
:10E9B0004FF0100383F31188BFF36F8FBFF34F8FB6
:10E9C000FEE703682BB3FFF773FCEFF311864FF0FC
:10E9D000100383F31188BFF36F8FBFF34F8FA26BC8
:10E9E000E36B9A4221D2A36B0133A363A36C01337F
:10E9F0001FD0A36C0133A364012086F3118870BD7E
:10EA00004FF0100383F31188BFF36F8FBFF34F8F65
:10EA1000FEE74368002BD6D04FF0100383F3118834
:10EA2000BFF36F8FBFF34F8FFEE7002086F311888F
:10EA300070BD636A002BDFD004F1240000F066FC97
:10EA40000028D9D0002DD7D001232B60D4E700BFF8
:10EA50002DE9F04184B00D4601921F46044600287E
:10EA600000F0978000297BD000F0F4FC002800F033
:10EA70008380FFF717FBA66B002E53D1019B002B61
:10EA800000F0988002A800F087FC04F124080FE051
:10EA9000FFF72AFB2046FFF76BFD00F06DFBFFF749
:10EAA00001FBA36B002B3DD1019B002B00F082806A
:10EAB000FFF71AFB00F02EFAFFF7F4FA626C01324E
:10EAC00008BF6664A26C013208BFA664FFF70CFBA6
:10EAD00001A902A800F076FC002871D1FFF7E2FA44
:10EAE000A36B002BD4D1FFF7FFFA2368002B59D07A
:10EAF0000199404600F0D2FB2046FFF739FD00F0B7
:10EB00003BFB0028CBD14FF0E0234FF08052C3F8FD
:10EB1000042DBFF34F8FBFF36F8FFFF7C3FAA36BC3
:10EB2000002BC1D0226CE6684AB16368B1189942E3
:10EB3000E16024BF2168E160284602F02FF8002F31
:10EB400044D1A36B2268013BA363002A5AD02369F6
:10EB5000002B50D1FFF7C8FA012004B0BDE8F081C6
:10EB6000036C002B80D04FF0100383F31188BFF3A8
:10EB70006F8FBFF34F8FFEE7019B002B3FF479AF00
:10EB80004FF0100383F31188BFF36F8FBFF34F8FE4
:10EB9000FEE74FF0100383F31188BFF36F8FBFF3CD
:10EBA0004F8FFEE7FFF77EFA606800F063FCFFF727
:10EBB0009BFA9DE7FFF798FA002004B0BDE8F081CA
:10EBC0002046FFF7D5FC00F0D7FAF5E7636AE66068
:10EBD000002BBFD004F1240000F098FB0028B9D02E
:10EBE0004FF0E0234FF08052C3F8042DBFF34F8F56
:10EBF000BFF36F8FAEE704F1100000F087FB012830
:10EC0000A8D1EDE700F0DAFC6060A0E750B10D4953
:10EC1000002351F8332090420DD00133082BF8D156
:10EC2000FFF730BC4FF0100383F31188BFF36F8FF1
:10EC3000BFF34F8FFEE7044A002142F83310FFF77D
:10EC400021BC00BFE40A0220E00A022007484FF07E
:10EC5000E0214FF0805205E0C1F8042DBFF34F8F43
:10EC6000BFF36F8F0368012BF6D8FEE7A00B0220DD
:10EC70000E4B0F4A19681268824210B5044648606C
:10EC800007D90C4A10681968BDE81040043100F03B
:10EC9000BFBC094A10681968043100F0B9FC074B81
:10ECA0001A68944238BF1C6010BD00BF2C0C0220B3
:10ECB000400B0220700B0220740B0220240B022058
:10ECC0002DE9F0470C4616461F460546002800F081
:10ECD0008680089B062B08D94FF0100383F3118818
:10ECE000BFF36F8FBFF34F8FFEE70A9B002B7FD0E0
:10ECF0005C20FFF739FB8046002800F099800A9BD2
:10ED00000363B60032461846A52101F008FFD8F883
:10ED10003090621E08F133030F3412F8011F03F81C
:10ED2000011F09B1A242F8D1089BC8F82C30002479
:10ED300008F1040AC8F84C30504688F84340C8F837
:10ED4000504000F053FC08F1180000F04FFC089B05
:10ED5000C8F85440043EC3F1070309EB0600C8F8A5
:10ED6000183088F85840C8F81080C8F824803A460F
:10ED7000294620F00700FFF76FF9099BC8F800004B
:10ED800013B1099BC3F80080FFF78CF93D4A3E4D53
:10ED90001368013313602B68002B4FD03B4E336850
:10EDA000002B3DD03A4C3B483B4A0368176801337F
:10EDB0000360D8F82C00C8F844300123834000EBEE
:10EDC00080003B43514604EB8000136000F012FCCE
:10EDD000FFF78AF933689BB90120BDE8F0874FF04F
:10EDE000100383F31188BFF36F8FBFF34F8FFEE7DC
:10EDF0009000FFF7B9FA0A9000287FF479AF1AE083
:10EE00002B68089ADB6A9342E6D24FF0E0234FF07A
:10EE10008052C3F8042DBFF34F8FBFF36F8FDBE732
:10EE20002B68089ADB6A934298BFC5F80080B9E75F
:10EE30000A98FFF727FB4FF0FF30CEE7C5F80080B8
:10EE40001368134C012B01D0104EACE7264604F199
:10EE50008C073046143600F0BDFBB742F9D10F4F96
:10EE60000F4E384600F0B6FB304600F0B3FB0D48BD
:10EE700000F0B0FB0C4800F0ADFB0C4B1F600C4BDE
:10EE80001E60E1E7440B02202C0C0220380B02200C
:10EE9000A00B0220280B02203C0B02208C0B02202E
:10EEA000780B02205C0B0220480B0220740B02201E
:10EEB000700B022030B585B000241149114803942D
:10EEC00002940194009423468022FFF7F9FE012862
:10EED00001D005B030BD4FF0100383F31188BFF3AC
:10EEE0006F8FBFF34F8F0849084A094B4FF0FF352A
:10EEF0000D6010601C6005B0BDE83040FFF760B9E0
:10EF0000341501084DEC0008240B0220380B0220B8
:10EF1000400B0220024A136801331360704700BFA0
:10EF2000200B02202DE9F04F4E4B1B6883B0002BC5
:10EF30004AD14D4B1A6801321A601F68002F51D018
:10EF40004A4B0193019B1B68BB4258D8484DDFF8E0
:10EF500038812B68DFF834911C68002C74D0454E42
:10EF6000002423E000F06CFBDBF828200BF11800F4
:10EF70000AB100F065FBDBF82C0033680122824007
:10EF800000EB80001A43514608EB8000326000F02D
:10EF900031FBD9F80030DBF82C20DB6A9A4228BF1D
:10EFA00044F001042B681B68002B4DD02B68DB68F4
:10EFB000D3F80CB0DBF804200BF1040A974250465A
:10EFC000D0D2019B1A601FE02B4A13680133002046
:10EFD00013602A4B1B68002B18BF40F0010003B0E0
:10EFE000BDE8F08F224B1A681268D2B14FF01003BF
:10EFF00083F31188BFF36F8FBFF34F8FFEE7DFF806
:10F000008880DFF888900024D9F80030DB6A03EBB1
:10F01000830358F82330012B94BF204644F00100AD
:10F02000D7E7174A186811681960164910600A680E
:10F0300001320A601A6812685AB90C4B01931A46D9
:10F040004FF0FF3313607DE7019A4FF0FF331360F9
:10F05000DAE71B68054ADB680192DB685B681360CE
:10F0600070E700BF200B0220400B0220240B02207F
:10F07000740B02203C0B0220340B0220300B0220C8
:10F08000700B02202C0B0220A00B02202C0C022063
:10F090002DE9F84FFFF706F82F4B1A68013A1A606E
:10F0A0001B68002B46D12D4B1B68002B42D0DFF88C
:10F0B000BC90DFF8BCA02A4EDFF8B880294F0125AC
:10F0C0001FE0DAF80C30DC6804F1040B04F11800DE
:10F0D00000F0B6FA584600F0B3FAE06A326805FA72
:10F0E00000F300EB80001343594608EB80003360C7
:10F0F00000F080FA3B68E26ADB6A9A4228BFC9F8EE
:10F100000050DAF80030002BDBD1174C23686BB1CC
:10F1100023685BB10125FFF705FF08B1C9F800506E
:10F120002368013B23602368002BF4D1D9F8004009
:10F13000012C05D00024FEF7D7FF2046BDE8F88F4C
:10F140004FF0E0234FF08052C3F8042DBFF34F8FF0
:10F15000BFF36F8FEFE700BF200B0220440B0220AC
:10F160003C0B02202C0C0220340B0220300B02201E
:10F170005C0B0220A00B0220064B1B6843B94FF02A
:10F18000100383F31188BFF36F8FBFF34F8FFEE738
:10F19000FFF77EBF200B022070B550B94FF0E0237F
:10F1A0004FF08052C3F8042DBFF34F8FBFF36F8F22
:10F1B00070BD1A4C236843B14FF0100383F31188DC
:10F1C000BFF36F8FBFF34F8FFEE72368144A154ECE
:10F1D00001332360156805443068043000F030FACC
:10F1E00040B933681049D86A0B680122824023EA8B
:10F1F00002030B602846FFF73BFD236843B94FF03D
:10F20000100383F31188BFF36F8FBFF34F8FFEE7B7
:10F21000FFF73EFF0028C1D070BD00BF200B0220C9
:10F22000400B02202C0C02203C0B0220164B1B68CA
:10F230001BB1164B01221A6070471449144A0B6027
:10F240001368B3FA83F3DBB2C3F11F0303EB830349
:10F2500010499A0001EB8303885840B94FF010031E
:10F2600083F31188BFF36F8FBFF34F8FFEE75868AA
:10F270000832406858600A44904204BF40685860B1
:10F28000054BC2681A607047200B0220300B022029
:10F290003C0B0220A00B02202C0C022038B50C469F
:10F2A000D8B1164D2968183100F0B2F92868043039
:10F2B00000F0C6F940B92B681149D86A0B680122E1
:10F2C000824023EA02030B60631C0FD00D4B1868C9
:10F2D0002044BDE83840FFF7CBBC4FF0100383F368
:10F2E0001188BFF36F8FBFF34F8FFEE72968064881
:10F2F000BDE83840043100F07DB900BF2C0C02207D
:10F300003C0B0220400B0220480B0220C36870B562
:10F31000DC6864B304F11805284600F091F9184B35
:10F320001B6873B11748294600F064F9164BE26A6E
:10F330001B68DB6A9A4283BF144B012018600020CF
:10F3400070BD261D124D304600F07AF9E36AD5F8FB
:10F3500000C0104801229A4003EB830342EA0C02EA
:10F36000314600EB83002A6000F044F9DEE74FF0FD
:10F37000100383F31188BFF36F8FBFF34F8FFEE746
:10F38000200B02205C0B02202C0C0220300B0220F0
:10F390003C0B0220A00B022030B1084A084B126837
:10F3A0001B68C0E9002370474FF0100383F31188F6
:10F3B000BFF36F8FBFF34F8FFEE700BF2C0B022010
:10F3C000400B022070B50D46044618B3C9B1FEF7D4
:10F3D00069FE2B681A4A581C11682CD0DFF864C0EB
:10F3E0002668DCF800E06068764501D0814203D2EF
:10F3F000A1EB000E734516D80124FEF775FE2046DA
:10F4000070BD4FF0100383F31188BFF36F8FBFF30C
:10F410004F8FFEE74FF0100383F31188BFF36F8F18
:10F42000BFF34F8FFEE75B1ADCF80010126803444D
:10F430002B60C4E900120024FEF756FE204670BD82
:10F44000400B02202C0B0220014B01221A60704756
:10F45000300B0220054B1B6833B1054B1868B0FA1E
:10F4600080F040094000704701207047380B0220AF
:10F47000200B0220F8B50446C0B11F4DC36A2A68AC
:10F48000D26A934212D28269002A04DB2A68D26AC5
:10F49000C2F107028261194E626903EB830306EB36
:10F4A00083039A4203D02B68DB6AE362F8BD271D11
:10F4B000384600F0C5F868B9E36A03EB830256F8F2
:10F4C00022203AB90E4A01219940136823EA010328
:10F4D000136000E00A4A2B68D86AE06201231468CE
:10F4E0008340234300EB8000394606EB8000136025
:10F4F000BDE8F84000F07EB82C0C0220A00B0220E2
:10F500003C0B022030B5044683B0A8B1284B1B68E1
:10F51000834208D04FF0100383F31188BFF36F8F3D
:10F52000BFF34F8FFEE71B6D4BB1C16AC26C013B4D
:10F530009142036500D05BB1002003B030BD4FF0B5
:10F54000100383F31188BFF36F8FBFF34F8FFEE774
:10F55000011D0846019100F073F80199B8B11548F2
:10F56000154AE36CD2F800C0E362C3F1070E01252F
:10F57000C4F818E005FA03F403EB830344EA0C042F
:10F5800000EB8300146000F035F82846D5E7E36A05
:10F59000084803EB830250F822200AB1064AE0E74C
:10F5A000054A01259D40136823EA05031360D8E747
:10F5B0002C0C0220A00B02203C0B0220044B1A68EA
:10F5C0001AB119680A6D01320A651868704700BFE0
:10F5D0002C0C022000F108034FF0FF3100224360A1
:10F5E0008160C36003610260704700BF0023036154
:10F5F000704700BF4268036810B494688C600133A0
:10F600004A60616091605DF8044B08610360704777
:10F6100030B40D686B1C10D000F108031C465B6809
:10F620001A68AA42FAD902684B60013299608C606C
:10F630006160086130BC0260704704696368F2E78A
:10F64000034602699968406810B454688160486054
:10F6500010689C4208BF51600138002119615DF8B3
:10F66000044B1060704700BF00F02AB800F028B8C3
:10F67000081E08B501DA00F036F8BDE8084000F0D1
:10F6800021B800000B68B3F1804F10B502D30B48CE
:10F6900000F02CF893420CD9B3EB420F4FEA42042E
:10F6A00007D2B4F1804F2DBF6FF040430C6023466A
:10F6B0000B60591CFFF7DCFF10BD00BFB8700108DC
:10F6C00001F05EB9012838BF012010B5044620467C
:10F6D00001F04EF900B110BD00F00CF808B9F0F7D8
:10F6E000DDFE8047F3E708B5F0F7D8FE08B5F0F780
:10F6F000D5FE0000024B1868BFF35B8F704700BF58
:10F70000300C022053B94AB9002908BF00281CBF99
:10F710004FF0FF314FF0FF3001F028B9ADF1080C88
:10F720006DE904CE00F006F8DDF804E0DDE902231F
:10F7300004B070472DE9F047089D0F4604468C46FB
:10F74000002B48D18A42164661D9B2FA82F34BB1F6
:10F75000C3F1200201FA03FC20FA02F29E4042EAC1
:10F760000C0C9C404FEA164EB7B2BCFBFEF1220CCB
:10F770000EFB11CC42EA0C4201FB07F0904209D982
:10F78000B21801F1FF3C80F0EE80904240F2EB8035
:10F7900002393244121AA4B2B2FBFEF00EFB102260
:10F7A00044EA024400FB07F7A74209D9341900F1E3
:10F7B000FF3280F0DA80A74240F2D780344402382A
:10F7C00040EA0140E41B00211DB1DC400023C5E9F3
:10F7D0000043BDE8F0878B4206D90DB1C5E90001B1
:10F7E00000210846BDE8F087B3FA83F1002948D12B
:10F7F000BB4202D3824200F20781841A67EB030204
:10F8000001209446002DE4D0C5E9004CE1E7002A30
:10F8100000F09280B2FA82F3002B40F0A8808A1A9E
:10F820004FEA164E1FFA86FC0121200CB2FBFEF7B0
:10F830000EFB172240EA02420CFB07F0904207D968
:10F84000B21807F1FF3802D2904200F2E280474638
:10F85000121AA4B2B2FBFEF00EFB102244EA0244DC
:10F860000CFB00FCA44507D9341900F1FF3202D289
:10F87000A44500F2CB801046A4EB0C0440EA0740FC
:10F88000A2E7C1F120068B4022FA06FC4CEA030CE9
:10F8900007FA01F420FA06F3F7404FEA1C49234324
:10F8A00000FA01F81FFA8CFEB7FBF9F01C0C09FBFB
:10F8B000107744EA074400FB0EF7A74202FA01F270
:10F8C0000AD91CEB040400F1FF3A80F09B80A742A8
:10F8D00040F2988002386444E41B9FB2B4FBF9F311
:10F8E00009FB134447EA044403FB0EFEA64509D96D
:10F8F0001CEB040403F1FF3780F08280A6457FD91A
:10F90000023B644443EA0040A4EB0E04A0FB02E780
:10F91000BC427346B94663D360D05DB1B8EB030215
:10F9200064EB090404FA06F622FA01F31E43CC4004
:10F93000C5E9006400214CE76208480842EAC17149
:10F940000B0C43EA00438AB242EA0342B3FBF6F1EE
:10F95000E407B4463746B6461F23B0FBF6F0D21B89
:10F9600041EA004161E7614614E7104628E7C3F128
:10F97000200120FA01F29E4027FA01F19F403A430C
:10F980004FEA164E1FFA86FCB1FBFEF70EFB17106E
:10F99000110C41EA004107FB0CF8884504FA03F416
:10F9A0003AD9711807F1FF3001D288451FD8A1EB71
:10F9B0000801B1FBFEF808FB0CF70EFB181192B220
:10F9C00042EA0142BA422FD2B21808F1FF31C6D240
:10F9D000BA42C4D2A8F102013244C0E7F0459CD239
:10F9E000BEEB020367EB0C070138B94695E7A6EBBF
:10F9F00008084144B81EB1FBFEF808FB0CF7DCE731
:10FA00003B467FE7504667E70846FBE6344402384A
:10FA100032E7023F32441BE7A1EB08013846B1FB55
:10FA2000FEF808FB0CF7C8E7414698E703685A0060
:10FA30004CBF43F0004323F000431844704700BF1D
:10FA40002DE9F04759B301F1FF3805461646474600
:10FA50004FF0000A0AEB070101EBD171491005EBE9
:10FA6000C1094846FFF7E2FF88454FEAC104034653
:10FA700010D004F10800B342284407D8FFF7D6FF9E
:10FA80000138B04208D201F1010AE3E78A4506D005
:10FA90004F1EDFE7B042F9D84846BDE8F0874FF087
:10FAA00000094846BDE8F087012806D0022802D0A8
:10FAB00028B904487047044870470448704700203C
:10FAC000704700BF99010108A9010108A1010108BF
:10FAD00030B5224B83B004468D1E43B301A928469E
:10FAE000AFF30080F0B101992A46FFF7A9FF014664
:10FAF000C0B1FFF79BFFA0644B68012B2BD0002BFC
:10FB000001F1040025DBFFF791FF00232365036863
:10FB1000E064002B12DBFFF789FF0346002023611E
:10FB200003B030BD00230920236103B030BD0C4B6E
:10FB30000C49C91AC91018460191D5E7C3F30360EF
:10FB4000FFF7B2FF031E0CBF09200020236103B0A2
:10FB500030BD0123DAE700230520E0E700000000C4
:10FB6000280D0108201301080368DA0710B50446C0
:10FB700006D49B0700F1500009D500F0A3FC2368D0
:10FB8000590709D51A070ED5DB0613D510BD00F0AD
:10FB900091FC23685907F5D404F1D80000F09AFCD1
:10FBA00023681A07F0D404F5AC7000F09BFC2368BE
:10FBB000DB06EBD404F5EC70BDE8104000F0D6BCD9
:10FBC0000346006800B11844704700BF704700BF8B
:10FBD00070B504460E46316C2046FFF779FF0546A6
:10FBE00088B9326C62612369324621460120984708
:10FBF0000828F0D0072806D12846316CFFF7E6FF29
:10FC0000301D00F04BFCF0F749FC00BF2DE9F04F30
:10FC10000D1DD0F80C90D0F818A0074614460FCD53
:10FC2000ADF5777D0DF10C0CACE80F000FCDACE815
:10FC30000F000FCDACE80F0095E80F0002AE4FF0BB
:10FC4000000E8CE80F000DF5F878C6F800E021E012
:10FC5000336C7B614FF4F4723146404600F09EFFF6
:10FC60003B694246394658469847D8F83830B3641D
:10FC70002146CDE9006A05463B4601203A46C84781
:10FC8000044618BB4FF4F4724146304600F086FF3C
:10FC9000082D19D1316C3846FFF71AFF0934054693
:10FCA0005FFA84FB0028D3D0B36BB3643A46CDE946
:10FCB000006A3B464BF010010120C84730B9284686
:10FCC0000DF5777DBDE8F08F072D05D00925284675
:10FCD0000DF5777DBDE8F08F2046316CFFF776FF9C
:10FCE00003A800F0DBFB00BFF0B5CB6BFBB001F16C
:10FCF000040C0B640F460546BCE80F0001AC0FC4B2
:10FD0000BCE80F000FC4BCE80F000FC49CE80F0054
:10FD10004FF0FF3E84E80F006E46CDF800E006E0AD
:10FD20002B693246294698470828044608D1316C89
:10FD30002846FFF7CDFE0028F2D009207BB0F0BDA9
:10FD40003046FFF711FF062CF7D139462846FFF75A
:10FD50003FFF00BFC1608261DA6B1A64194600225E
:10FD6000FFF754BF436970B50B64C668AEB9036949
:10FD70000A4604460D46014602209847072805D04A
:10FD800008280FD129462046FFF722FF3046296C6C
:10FD9000FFF71CFF281D00F081FB0122FFF736FF53
:10FDA000F0F77CFBF0F77AFBC26808B532B1CA6B9A
:10FDB0000A64BDE808400022FFF728BFFFF794FF60
:10FDC000092008BD052915D8DFE801F00A0314034E
:10FDD000030501207047009A436C136000207047B0
:10FDE00043B90F2A06D800EB820200205368009A1C
:10FDF000136070470220704700B585B00A460023A3
:10FE000003A900911946FFF7DDFF039805B05DF8DF
:10FE100004FB00BF052915D8DFE801F00A0314032D
:10FE2000030501207047009B1B6843640020704756
:10FE300043B90F2A06D8009B00EB82021B6853606F
:10FE4000002070470220704710B584B0002303AC37
:10FE5000039200940A461946FFF7DCFF04B010BD78
:10FE60002DE9F041D36BADF5107D02F1040C136464
:10FE700007460E46BCE80F000DF15C0EAEE80F0021
:10FE8000BCE80F00AEE80F00BCE80F00AEE80F00C2
:10FE90009CE80F0016AC4FF0FF388EE80F006D465F
:10FEA000C4F8008010E0FFF7CFFF31462046B84786
:10FEB000034622460820294683B92B69984705281E
:10FEC00080460DD0092809D0216C2846FFF700FE96
:10FED00003460C212A462046002BE4D04FF00908A7
:10FEE0002046FFF741FE40460DF5107DBDE8F0814C
:10FEF0002DE9F04F1646CA6C89B00D4652F8041B26
:10FF0000069200F0030CE3B10C0C8DF81D400904BF
:10FF1000E4B2059102EB840202218DF81C10296DD8
:10FF2000BCF1020F08BFAA6B11F001080FD005A9A0
:10FF3000304600F09BFB002839D1082009B0BDE80D
:10FF4000F08F090205918DF81D300321E5E7176850
:10FF5000002FECD000F008010191E346CDF80880B5
:10FF60009A46BAF1020F26D01788548802F1040984
:10FF7000AA6C24F001030F21304603EB0208FFF7BF
:10FF80003BFF804515D827F0010202EB08038342AE
:10FF900094BF00230123640004F0020407F001076A
:10FFA0002743012F0BD0022F50D0002F45D009201E
:10FFB000C4E70023EFE7546802F10809D8E7BBF172
:10FFC000000F73D1CBB1D9F80430D9F80020991CB7
:10FFD0004FEAD272EBD005F158040133049400F0DB
:10FFE000CC8009F10400FFF7EBFD04AB0146284685
:10FFF000AFF30080002840F0978009F108021768ED
:020000040801F1
:10000000002FAED105A93046DDF8088000F02EFBA8
:100010000028CCD1B8F1000F8FD00F213046FFF768
:10002000EBFE0E2102463046FFF70EFF594A0F2124
:100030003046FFF709FF072080E7BBF1000F02D031
:10004000002B40F0878009F10402D8E7D9F800407E
:1000500024F00048BBF1000F0FD12BB1019B002B06
:100060003CD0B8F1000F39D0002C01DA09F10409B5
:1000700008F1010209EB8202C1E70D213046FFF7CA
:10008000BBFE2F6A8742EFD1AB6A9945ECD10024C1
:100090000423C5E90B434B44C5F828806B63D9F8AA
:1000A0000030A34270DB01230293E1E70D213046CB
:1000B000FFF7A2FE2C6A84429FD1AB6A99459CD17E
:1000C0004846FFF7B3FC0F2102463046FFF7BCFE5F
:1000D0002A4600213046FFF7B7FEACE705F158038A
:1000E000CDF80CB009F10407B34600241E460BE01E
:1000F00038460496FFF764FD0022014604AB28460B
:10010000AFF300800437F8B9444504F10104EFD19E
:100110000D215846FFF770FE049BC5F82890024653
:10012000C5E90823062009E704460D213046FFF7FC
:1001300063FE049E2862022C04BFEE6205F12C06C9
:10014000C5E909690620F9E65E46D9F80040DDF800
:100150000CB089E74846FFF769FC09F1040304463F
:10016000AB632846AFF3008000283FF420AF22465F
:100170000F213046FFF768FE5DE730460D21FFF79F
:100180003BFE26462862DBE708F1010209EB82000C
:1001900097E700BF000000000023FFF7A9BE00BFE3
:1001A0000123FFF7A5BE00BF0223FFF7A1BE00BFDA
:1001B0002DE9F0410646C4B01446052908D8DFE809
:1001C00001F016300773980B3A19102A40F2B780E5
:1001D000022044B0BDE8F081836B002CF8D153F8C5
:1001E000042B42648363002044B0BDE8F081002BFF
:1001F000EED1856B1FFA84FC012006F1040E00FA93
:1002000003F111EA0C0F2A4604D052F8041B4EF8F1
:10021000231015460133102BF1D1A004E3D4B563AC
:10022000E1E7012B4FEA1447A4B2CDD0052BCFD183
:1002300007EB0408B8F1200FCAD80F2F40F2BD8099
:10024000002CD0D002685107A04600F11B81019319
:1002500002AC204600F042F9D6F838C0019B102FBE
:100260004FF0FF3239464FF0020E38BF102118FB15
:100270000E2E04EBC10184397246604650F8045BCF
:1002800041F8045F013A551CF8D10CF1040C012B24
:100290000CEB8E0200F0D5800F2FB26340F2FA8093
:1002A000204600F017F99EE7032B91D1A7B207EB88
:1002B0001443102B4FEA14448AD80368190700F13D
:1002C000A38022AD284600F02FF97A00B06B05EB31
:1002D000C404531E42B1011B625844F8042B013B75
:1002E0005A1CF9D100EBC700B063284600F0FAF8B9
:1002F00079E7002B7FF46CAF102C3FF669AF0368F1
:10030000D80679D422AD284600F03AF9B76B2946D1
:1003100000234FF0010C0CFA03F22242384603F19D
:10032000010303D050F8042B0A600746042B01F1A7
:100330000401F0D1B763284600F018F953E7102FF5
:100340003FF446AF0268D10708D5304622F00302D9
:1003500040F8502B019300F0B1F8019B019322ADBE
:10036000284600F0ABF8D6F838C0002C6BD0019BC3
:100370004FF0000802214FF0FF3214FB012E05EB75
:10038000C70104397246604650F8044B41F8044FE7
:10039000013A541CF8D10CF1040C0CEB8E0CB8F1A2
:1003A000000F39D1012B4ED00F2FC6F838C03FF6C1
:1003B0001AAF284600F086F815E70268B8F1100F6A
:1003C00002F001012AD851B1304622F0010242F078
:1003D000020240F8502B019300F078F8019B019342
:1003E00022AD284600F072F8019B002CE1D0D6F82F
:1003F00038C04FF00008BDE723F01003336006F566
:10040000EC7000F0BDF87DE723F00803036000F511
:10041000AC7000F089F854E702AC20E7D1B9550779
:1004200026D422AD2846019300F050F802A800F02F
:1004300055F8A8F11008D6F838C0019BC7F1100490
:1004400098E7944622AD0CF10403B363284600F00C
:1004500031F8C8E622F0010242F0020240F8502BC7
:10046000019300F033F83268019B12F0040FD8D0EA
:10047000304622F0040240F8D82B019300F02EF809
:10048000019BCEE722F0040240F8D82B019300F044
:1004900025F8DDE622A800F015F801E700F13401A7
:1004A00091E838009C46A6464CF8045D90E8FF0FA2
:1004B000E54600BD90EC210B704700BF80EC210B9E
:1004C000704700BF90EC200B704700BF80EC200B02
:1004D000704700BFD0EC200B704700BFC0EC200B72
:1004E000704700BFF0EC0201F0EC0211F0EC0221C9
:1004F000F0EC0231F0EC0241F0EC0251F0EC026160
:10050000F0EC0271F0EC0281F0EC0291F0EC02A14F
:10051000F0EC02B1F0EC02C1F0EC02D1F0EC02E13F
:10052000F0EC02F1704700BFE0EC0201E0EC0211D8
:10053000E0EC0221E0EC0231E0EC0241E0EC02519F
:10054000E0EC0261E0EC0271E0EC0281E0EC02918F
:10055000E0EC02A1E0EC02B1E0EC02C1E0EC02D17F
:10056000E0EC02E1E0EC02F1704700BFB0FC018179
:10057000B0FC0191B0FC01A1B0FC01B1704700BF1B
:10058000A0FC0181A0FC0191A0FC01A1A0FC01B193
:10059000704700BFEC4600B52DE900502DE9FF1F64
:1005A0004FF000030CB401A9FFF79EFBDDF840E01B
:1005B00012B07047EC4600B52DE900502DE9FF1F41
:1005C0004FF000030CB401A9FFF7CCFBDDF840E0CD
:1005D00012B07047EC4600B52DE900502DE9FF1F21
:1005E0004FF000030CB401A9FFF7DEFBDDF840E09B
:1005F00012B07047EC4600B52DE900502DE9FF1F01
:100600004FF000030CB401ABFFF7A4FBDDF840E0B2
:1006100012B07047EC4600B52DE900502DE9FF1FE0
:100620004FF000030CB401AAFFF71AFCDDF840E01C
:1006300012B07047027A03467AB9427AA2B1416891
:10064000013A10B44272086803220C1D1A720202A9
:100650005C60000E10BC1A6070470068013A1A72A4
:1006600002021A60000E7047B02070472DE9F04377
:10067000064685B00D4600272846FFF7DBFFB02869
:10068000044600F0218103065ED500F0F003A02BA4
:100690001DD033D8802B00F08780902B2AD100F01A
:1006A0000D030D2B26D00DF10808002300F00F02DA
:1006B0001946CDF800803046FFF784FB0023CDF8C3
:1006C00000800D2219463046FFF7A4FBD4E7C34350
:1006D00003F007034FF47F621A41010702F47F62BF
:1006E00001D542F48042002319463046FFF760FDF1
:1006F0000028C1D0092005B0BDE8F083B02B68D038
:10070000C02B3FD1C62800F0CC80C72800F0DF8086
:1007100000F0F803C02B00F0EC80C82800F0F78050
:10072000C928E7D12846FFF785FF020300F00F0034
:1007300002F4702201300243012105233046FFF705
:1007400037FD002898D0D5E78300DBB203F1040819
:100750000DF1080900231946CDF800900D2230460E
:10076000FFF730FB029ACDF8009060064CBFA2EB79
:10077000080242440023029219460D223046FFF738
:1007800049FB79E700F0F803D02BB3D100F0070262
:100790000132052342F4002201213046FFF708FD13
:1007A00000283FF469AFA5E72846FFF743FF24027E
:1007B0002043B0F5004F9DD004010023A2B219469A
:1007C0003046FFF7F5FC002894D1C4F3C03007434E
:1007D00052E7A0F1B103042B00F2B580DFE803F08B
:1007E0005729160C030003AA0023009219460D2274
:1007F0003046FFF7E7FA3FE700231A460521304667
:10080000FFF7D6FC00283FF437AF73E72846FFF721
:1008100011FF020300F00F00013002F470220123E7
:10082000024319463046FFF7C3FC00283FF424AFCB
:1008300060E700230DF108090D221946CDF800905C
:100840003046FFF7BFFA2846FFF7F4FE0206029C87
:100850004FF002080CD500F07F0000FA08F00444C5
:1008600028460294FFF7E6FE030608F10708F2D4D3
:1008700000FA08F004F50174204400230290CDF83A
:1008800000900D2219463046FFF7C4FAF4E62846D8
:10089000FFF7D0FE431EDBB20E2B02467FF623AFDE
:1008A00028E72846FFF7C6FE020300F00F000130DC
:1008B00002F470220323024319463046FFF778FC06
:1008C00000283FF4D9AE15E76FB3002013E72846A0
:1008D000FFF7B0FE431EDBB20E2B02463FF60AAF17
:1008E000002304213046FFF763FC00283FF4C4AE28
:1008F00000E700F00F020132032342F420221946E0
:100900003046FFF755FC00283FF4B6AEF2E6284625
:10091000FFF790FE00F0F00200F00F0310320133F9
:1009200043EA023208E702AC3B46394600940E2205
:100930003046FFF747FA0F2200943B4639463046CF
:10094000FFF768FAC1E700F0FC03B42B3FF4D2AE26
:1009500000F007020132012342F40022194630461A
:10096000FFF726FC00283FF487AEC3E6704700BFC0
:10097000024B0146186800F02DB800BFE8000020C7
:10098000024B0146186800F01FB900BFE8000020C4
:1009900070B50F4E0C463168054611B900F0C8F825
:1009A00030602146284600F0C3F8431C03D14FF0C5
:1009B000FF34204670BDC41C24F00304A042F8D0CC
:1009C000211A284600F0B4F80130F2D1EFE700BF59
:1009D000340C02202DE9F843CD1C25F00305083521
:1009E0000C2D38BF0C25002D064601DBA94204D989
:1009F0000C2333600020BDE8F883DFF8D48000F0DA
:100A000069F8D8F800301C4644BB29463046FFF749
:100A1000BFFF431C044658D1D8F800402746002F9A
:100A200043D1002C4BD023683946304604EB0309F0
:100A300000F07EF8814542D121686D1A2946304682
:100A4000FFF7A6FF01303AD023682B442360D8F883
:100A500000305A6862BBC8F800700FE02268521B71
:100A600020D40B2A17D96119A342256018BF5960F9
:100A7000636808BFC8F8001062514B60304600F050
:100A80002FF804F10B00231D20F00700C21A1CBF31
:100A90001B1AA350AFE76268A3420CBFC8F800203E
:100AA0005A60EBE723466468AEE73C467F68B6E7EA
:100AB0001A465B68A342FBD100235360DEE70C2398
:100AC0003360304600F00CF894E70560D6E700BFCD
:100AD000380C0220014800F05FB800BF3C0C022037
:100AE000014800F05AB800BF3C0C0220884210B503
:100AF00001EB020402D98442234607D8431EA142D7
:100B000007D011F8012B03F8012FF8E702448242C5
:100B100000D110BD13F8011D02F8011DF7E70244D2
:100B20000346934200D1704703F8011BF9E7000028
:100B300038B5064D0023044608462B60EFF7B0FC9D
:100B4000431C02D12B6803B1236038BD3CB901209E
:100B500070B50D4B0D4D5B1B9C100026A64209D1B4
:100B6000EFF79AFC0A4D0B4B5B1B9C100026A6422C
:100B700005D170BD55F8043B98470136EEE755F8AE
:100B8000043B98470136F2E7D0700108D0700108A5
:100B9000D0700108E4700108704770470A44914220
:100BA00000F1FF3300D1704710B511F8014B03F885
:100BB000014F9142F9D110BD034613F8012B002AD1
:100BC000FBD1181A0138704738B50546002941D0C5
:100BD00051F8043C0C1F002BB8BFE418FFF77AFF54
:100BE0001D4A136833B9636014602846BDE8384075
:100BF000FFF776BFA34208D9206821188B4201BFB6
:100C000019685B6809182160EDE71A465B680BB14B
:100C1000A342FAD911685018A0420BD120680144B0
:100C2000501883421160E0D118685B685360084433
:100C30001060DAE702D90C232B60D6E72068211870
:100C40008B4204BF19685B68636004BF09182160A8
:100C50005460CAE738BD00BF380C022008B10181DA
:100C6000B0B000840000000008B10181B0B0008481
:100C70000000000008B10181B0B000840000000055
:100C800008B10181B0B000840000000008B101810A
:100C9000B0B000840000000008B10181B0B0008451
:100CA0000000000008B10181B0B000840000000025
:100CB00008B10181B0B000840000000008B10181DA
:100CC000B0B000840000000008B10181B0B0008421
:100CD0000000000008B10181B0B0008400000000F5
:100CE00008B10181B0B000840000000008B10181AA
:100CF000B0B000840000000008B10181B0B00084F1
:100D00000000000008B10181B0B0008400000000C4
:100D100008B10181B0B000840000000008B1018179
:080D2000B0B0008400000000E7
:100D28009CF4FE7F01000000E8F4FE7FB0A920805B
:100D380070F5FE7F0100000070F5FE7FB0A90A8003
:100D4800F8F5FE7F01000000FC0DFF7F08FFFF7F24
:100D5800000EFF7F01000000FC0DFF7F04FFFF7FF6
:100D6800080EFF7F08FFFF7F200EFF7FB0AA0180DB
:100D7800780EFF7FA908B180A00EFF7FAD08B18073
:100D8800000FFF7FA908B180340FFF7FB0AF02804A
:100D9800F40FFF7FB0AF06807011FF7FB0AF048003
:100DA8002012FF7FB0A90280AC13FF7F0100000072
:100DB8001414FF7FC4FEFF7F2414FF7FC8FEFF7F4B
:100DC8003014FF7FCCFEFF7F4814FF7FB0AA01805C
:100DD8009C14FF7FB0B0A880AC14FF7FB0B0AA808D
:100DE800CC14FF7FB0AF02803815FF7FB0AF06800C
:100DF800A816FF7FA908B180DC16FF7FB0AF04807A
:100E08007017FF7FB0AA0380FC18FF7FB0A902808B
:100E18005419FF7F010000008024FF7FB0A90A80D9
:100E2800A425FF7F01000000E425FF7FB0AD0C8002
:100E3800EC26FF7FB0B0AA801027FF7FB0A82D80D6
:100E48001428FF7F010000003428FF7FB0B0A8807D
:100E58007428FF7FB0A805805C29FF7FB0A80380B5
:100E6800C429FF7F38FEFF7FCC29FF7F3CFEFF7F30
:100E7800D429FF7F01000000F029FF7FB0AF068072
:100E8800DC2AFF7FB0B0AE80E02BFF7FB0B0AC8033
:100E98001C2CFF7FB0AF0680342DFF7FB0AF0280DF
:100EA800082EFF7FB0B0AA80D82EFF7FB0A914808B
:100EB800302FFF7FB0A81380A42FFF7FB0AA09802E
:100EC8009430FF7FB0AA0F80BC31FF7FB0B0AA80FA
:100ED8000C32FF7FB0AF0280F832FF7F00840880B9
:100EE8004033FF7FD0FDFF7F6833FF7F01000000A4
:100EF8006833FF7FB0B0A8807433FF7FB0A801804B
:100F0800B433FF7FB0AA01800C34FF7F01000000DA
:100F18006037FF7FA908B180A037FF7F010000007C
:100F2800BC37FF7FA908B180D837FF7F01000000D8
:100F38009839FF7FA908B180B83AFF7F0100000007
:100F4800283BFF7FB0B0AA80B03BFF7F01000000C4
:100F5800CC3BFF7FB0AB0280703DFF7F01000000FB
:100F6800BC3FFF7F5CFDFF7FCC3FFF7FAD08B180BA
:100F7800E840FF7FB0B0AA804041FF7F0100000039
:100F8800B041FF7FB0B0AA809042FF7FB0AE018031
:100F98008043FF7FB0AE0380BC44FF7F01000000A8
:100FA800B844FF7FB0B0AA803846FF7F0100000038
:100FB8003446FF7FB0B0A8806046FF7FB0AF0280A4
:100FC800AC47FF7FB0AF0680384AFF7F01000000C2
:100FD800584AFF7FA908B180004BFF7FB0B0A880B6
:100FE800584CFF7FB0AA0B808855FF7FB0AB0280BA
:100FF8001857FF7F01000000A858FF7FB0B0AA80F3
:101008007C59FF7F010000007859FF7FB0B0A880AD
:101018009859FF7FAD08B1806C5AFF7FAF08B18047
:101028006C5BFF7FB0B0AA802C5CFF7FAD08B180FD
:10103800645EFF7FB0AA0780FC5EFF7F01000000AE
:10104800685FFF7FB0B0AC809460FF7F0100000054
:101058001C61FF7FB0AC01803467FF7F0100000096
:101068003067FF7FB0B0A8805C67FF7F0100000099
:101078005867FF7FA908B1802868FF7F010000003A
:101088003868FF7FB0B0AC80D868FF7FB0A9048013
:101098003869FF7FB0A90280A869FF7F01000000BE
:1010A800A469FF7FB0B0AA80FC6AFF7FA908B1805D
:1010B800186CFF7F01000000186CFF7F10FCFF7F99
:1010C8001C6CFF7F01000000186CFF7F0CFCFF7F89
:1010D8001C6CFF7F01000000186CFF7F08FCFF7F7D
:1010E8001C6CFF7F01000000186CFF7F04FCFF7F71
:1010F800346CFF7FB0A902809C6CFF7FB0AA01808E
:10110800EC6DFF7FB0A904805C6FFF7FF0FBFF7F71
:10111800646FFF7F01000000606FFF7FB0B0AA809E
:10112800B06FFF7F010000000C70FF7FB0B0A88097
:101138005871FF7F010000003072FF7FB0B0A880B7
:101148006072FF7F010000006072FF7FA908B18014
:101158004073FF7F010000003C73FF7FA908B18046
:101168009473FF7F010000009473FF7FB0B0A880E4
:101178000874FF7F010000000474FF7FB0B0AA80EC
:10118800AC75FF7F84FBFF7FB475FF7F0100000013
:1011980048CAFF7FB0A8018070CAFF7F0100000025
:1011A80020CEFF7FB0B0A88044CEFF7F01000000B2
:1011B800B0D1FF7FAD08B180C4D2FF7F0084028028
:1011C80034D3FF7FA908B180A4D4FF7FAB08B180D6
:1011D80004D5FF7FB0B0A88038D5FF7FB0AB0480BE
:1011E800ACD6FF7FB0B0AA80F0D6FF7FB0B0AC809D
:1011F800ACD7FF7FB0B0AA8050D8FF7FB0AC0380D7
:1012080004DAFF7F0100000060DAFF7FB0B0A88039
:10121800A8DAFF7FB0B0AE8094DCFF7FB0A904806D
:10122800ECDCFF7F01000000F4DCFF7FB0AF028040
:1012380058DEFF7FAF08B18038DFFF7F0100000074
:1012480050DFFF7FB0B0AA80DCDFFF7F0100000025
:1012580044E0FF7FA908B180ACE0FF7FB0B0AA806E
:1012680030E1FF7F0100000054E1FF7FB0B0AA80A9
:10127800D0E1FF7F01000000F4E1FF7FAB08B180FF
:101288007CE2FF7FB0A902802CE3FF7F0100000011
:1012980038E8FF7FB0A90280C8E8FF7FB0B0A88017
:1012A80018E9FF7F0100000020E9FF7FB0B0AA80A5
:1012B80054E9FF7FAF76B28028EAFF7FAB3F3A80E0
:1012C8008CEAFF7F0100000094EAFF7FB0B0AA809B
:1012D800D0EAFF7F40FAFF7FE4EAFF7F01000000C9
:1012E80078EBFF7FAC0FB28000ECFF7FB0AF0880D7
:1012F800A0EEFF7F01000000B0EEFF7FAC3F03804F
:1013080094F1FF7F010000005CF3FF7FB0AD048023
:0813180054F6FF7F0100000004
:1013200053746172742076616E2067656D696464C0
:10133000656C646520776161726465206170706CB2
:10134000696B617469652E0A00000000476562726E
:1013500075696B2053656767657220525454206F1E
:101360006D206865742066696C7465726765647267
:10137000616720746520646562756767656E2C20FF
:10138000696E6469656E206E6F6469672E0A00007D
:10139000455345204453504553454C20707261637A
:1013A000746963756D0000006573650031363A3508
:1013B000363A31372033312D30312D32303236004C
:1013C0004F70647261636874203241004472756BBF
:1013D0002022557022206F6D207465206265676938
:1013E0006E6E656E000000004F7064726163687419
:1013F0002032000046696C74657220697320616B4D
:10140000746965662100000047656D20576161724F
:101410006465205461736B004C454420426C696ED6
:101420006B207461736B00005465726D696E616C42
:1014300020627566666572004C6F6767696E67202B
:1014400042756666657200002853544D3332426F10
:10145000617264436F6E74726F6C6C65723A3A536A
:10146000544D3332426F617264436F6E74726F6CAD
:101470006C65722920536567676572205254542049
:101480006F7065726174696F6E65656C2E0A00001D
:10149000546F75636873637265656E0043616C6950
:1014A00062726174696F6E004552524F52000000C3
:1014B000546F75636873637265656E2063616E6EE9
:1014C0006F742062652063616C6962726174656427
:1014D00000000000546F75636873637265656E2069
:1014E000756E646566696E6564206572726F720000
:1014F000546F75636873637265656E2054696D65BA
:101500006F757400546F75636873637265656E20E0
:101510004E6F7420466F756E640000005465726DE6
:10152000696E616C000000005254540053454747F7
:101530004552000049444C450000000000000000F6
:1015400000000000C1040008D504000849DC0008C0
:1015500065DC00087DDC00080000000000000000E1
:1015600000000000000000009104000800000000DE
:1015700000000000000000000000000091040008CE
:1015800000000000000000002D05000851050008C3
:1015900075060008000000000000000009050008B2
:1015A0007D0500082507000800000000000000007D
:1015B000450800085908000800000000000000006D
:1015C0000000000000000100000101000000000018
:1015D00001000000020000000300000000010203FF
:1015E0000000000060EA3075983A88131400DC00AF
:1015F00006072828060000000100020000800040C5
:1016000001000000000002400018024000140240E7
:101610000014024000180240010000000200000017
:1016200004000000080000000000000000000000AE
:10163000000000000010101010100000100000004A
:10164000006C48480000000000000000001414284E
:101650007C287C28505000000010384040384870EA
:1016600010100000002050200C700814080000002A
:101670000000001820205448340000000010101012
:1016800010000000000000000008081010101010EA
:10169000100808000020201010101010102020004A
:1016A00000107C102828000000000000000010102E
:1016B00010FE1010100000000000000000000018D4
:1016C0001030200000000000007C0000000000003E
:1016D000000000000000003030000000000404089A
:1016E0000810102020400000003844444444444482
:1016F0003800000000301010101010107C000000A6
:1017000000384404081020447C00000000384404E1
:101710001804044438000000000C141424447E040F
:101720000E000000003C2020380404443800000073
:10173000001C20407844444438000000007C4404ED
:10174000080808101000000000384444384444449D
:101750003800000000384444443C04087000000095
:1017600000000030300000303000000000000018A1
:10177000180000183020000000000C10608060107D
:101780000C000000000000007C007C000000000055
:101790000000C02018041820C00000000000182419
:1017A00004081000300000003844444C54544C40AD
:1017B000443800000030102828287C44EE00000047
:1017C00000F8444478444444F8000000003C44409D
:1017D000404040443800000000F04844444444483D
:1017E000F000000000FC445070504044FC00000039
:1017F000007E22283828202070000000003C444051
:10180000404E44443800000000EE44447C444444CC
:10181000EE000000007C1010101010107C00000082
:10182000003C0808084848483000000000EE4448E2
:1018300050704844E600000000702020202024243E
:101840007C00000000EE6C6C54544444EE00000038
:1018500000EE64645454544CEC00000000384444DE
:1018600044444444380000000078242424382020D4
:10187000700000000038444444444444381C0000D4
:1018800000F8444444784844E200000000344C40EE
:10189000380404645800000000FE9210101010106C
:1018A0003800000000EE4444444444443800000042
:1018B00000EE4444282828101000000000EE4444A4
:1018C000545454542800000000C6442810102844E2
:1018D000C600000000EE4428281010103800000058
:1018E000007C4408101020447C00000000382020B8
:1018F0002020202020203800004020202010100828
:101900000808000000380808080808080808380017
:10191000001010284400000000000000000000003B
:1019200000000000000000FE0010080000000000A1
:101930000000000000000038443C44443E00000029
:1019400000C0405864444444F80000000000003CDB
:101950004440404438000000000C04344C444444EB
:101960003E00000000000038447C40403C00000085
:10197000001C207C202020207C000000000000367D
:101980004C4444443C04380000C04058644444443F
:10199000EE00000000100070101010107C0000001D
:1019A00000100078080808080808700000C0405CB3
:1019B00048705048DC00000000301010101010106B
:1019C0007C000000000000E854545454FE00000065
:1019D000000000D864444444EE00000000000038D9
:1019E0004444444438000000000000D864444444A7
:1019F0007840E000000000364C4444443C040E00B3
:101A00000000006C302020207C0000000000003C22
:101A100044380444780000000000207C202020226C
:101A20001C000000000000CC4444444C3600000080
:101A3000000000EE4444282810000000000000EEE2
:101A40004454545428000000000000CC4830304872
:101A5000CC000000000000EE44242818101078008C
:101A60000000007C481020447C000000000810109A
:101A7000101020101010080000101010101010107E
:101A8000101000000020101010100810101020007E
:101A900000000000002458000000000000000000CA
:101AA0000000000000000000000000000000000036
:101AB0000000000000000000000000000000000026
:101AC00000000000000007000700070007000700F3
:101AD00007000700020002000000000007000700E6
:101AE00000000000000000000000000000000000F6
:101AF0001CE01CE01CE0084008400840000000001A
:101B000000000000000000000000000000000000D5
:101B1000000000000CC00CC00CC00CC00CC03FF09A
:101B20003FF00CC00CC03FF03FF00CC00CC00CC02C
:101B30000CC00CC000000000000000000300030007
:101B400007E00FE0186018001F000FC000E01860E9
:101B500018601FC01F800300030003000000000086
:101B60000000000000001C002200220022001C6077
:101B700001E00F803C0031C002200220022001C0A1
:101B80000000000000000000000000000000000055
:101B9000000003E00FE00C000C0006000F301FF007
:101BA00019E018C01FF007B000000000000000009E
:101BB000000000000000000003800380038001009B
:101BC0000100010000000000000000000000000013
:101BD000000000000000000000000000000000C045
:101BE00000C00180018001800300030003000300A6
:101BF0000300030001800180018000C000C00000DC
